:020000040800F2
:1000000000060020E1010008E3010008E301000808
:10001000E3010008E3010008E3010008E301000830
:10002000E3010008E3010008E30100089D2F000838
:10003000E3010008E3010008E3010008E301000810
:10004000E3010008E3010008E3010008E301000800
:10005000E3010008E3010008453200086D320008A2
:1000600095320008BD320008E5320008E3010008BF
:10007000E3010008E3010008E3010008E3010008D0
:10008000E3010008E3010008E3010008E3010008C0
:10009000E3010008E3010008E30100080D33000854
:1000A000E3010008E3010008E3010008E3010008A0
:1000B000E1330008E3010008E3010008E301000860
:1000C000E3010008E3010008E3010008E301000880
:1000D000E3010008E3010008E3010008E301000870
:1000E00071330008E3010008E3010008E3010008A0
:1000F000E3010008E3010008E3010008E301000850
:10010000E3010008E3010008E3010008E30100083F
:10011000E3010008E3010008E3010008E30100082F
:10012000E3010008E3010008E3010008E30100081F
:10013000E3010008E3010008E3010008E30100080F
:10014000E3010008E3010008E3010008512700086B
:10015000E3010008E3010008E3010008E3010008EF
:10016000E3010008E3010008E3010008E3010008DF
:10017000E3010008E3010008E3010008E3010008CF
:10018000E3010008E3010008E3010008E3010008BF
:10019000E3010008E3010008E3010008E3010008AF
:1001A000E3010008E3010008E3010008E30100089F
:1001B000E3010008E3010008E3010008E30100088F
:1001C000E3010008E3010008E3010008E30100087F
:1001D000E3010008E3010008E3010008E30100086F
:1001E00002E000F000F8FEE772B6374880F30888B6
:1001F000364880F3098836483649086040F20000E6
:10020000CCF200004EF63471CEF200010860BFF36C
:100210004F8FBFF36F8F40F20000C0F2F0004EF638
:100220008851CEF200010860BFF34F8FBFF36F8F8C
:100230004FF00000E1EE100A4EF63C71CEF20001E4
:100240000860062080F31488BFF36F8F01F048FF29
:1002500002F042FE4FF055301F491B4A91423CBF0D
:1002600041F8040BFAE71D49184A91423CBF41F896
:10027000040BFAE71A491B4A1B4B9A423EBF51F83E
:10028000040B42F8040BF8E700201849184A914281
:100290003CBF41F8040BFAE701F026FF02F070FEC4
:1002A000144C154DAC4203DA54F8041B8847F9E7A7
:1002B00000F042F8114C124DAC4203DA54F8041B22
:1002C0008847F9E701F00EBF000600200022002059
:1002D0000000000808ED00E00000002000060020FB
:1002E000A8370008002200204022002040220020E1
:1002F000602E0020E0010008E0010008E001000895
:10030000E00100082DE9F04F2DED108AC1F80CD066
:10031000C3689D46BDEC108ABDE8F08F002383F3CF
:1003200011882846A047002001F08AFAFEE701F074
:1003300019FA00DFFEE7000038B500F0BFFB01F05E
:100340009FFE054601F0C2FE0446C8B90E4B9D4211
:1003500018D001339D4218BF044641F2883504BFCE
:1003600001240025002001F095FE0CB100F074F886
:1003700000F018FD284600F0C3F800F06DF8F9E72A
:100380000025EFE70546EDE7010007B008B500F0EE
:1003900067FBA0F120035842584108BD07B541F260
:1003A0001203022101A8ADF8043000F077FB03B07E
:1003B0005DF804FB38B5302383F3118817480368D0
:1003C0000BB101F009FB164A144800234FF47A716F
:1003D00001F0F8FA002383F31188124C236813B15B
:1003E0002368013B2360636813B16368013B63606A
:1003F0000D4D2B7833B963687BB9022000F034FCD3
:10040000322363602B78032B07D163682BB902205A
:1004100000F02AFC4FF47A73636038BD402200205C
:10042000B50300086023002058220020084B1870F4
:1004300003280CD8DFE800F008050208022000F0CD
:1004400003BC022000F0F0BB024B00225A60704750
:100450005822002060230020244B254A10B51C465A
:100460001968013140D004339342F9D16268214BBD
:100470009A4239D9204B9B6803F1006303F580331E
:100480009A4231D2002000F033FB0220FFF7CEFF6A
:100490001A4B1A6C00221A64196E1A66196E596C7E
:1004A0005A64596E5A665A6E5A6942F080025A610D
:1004B0005A6922F080025A615A691A6942F0005260
:1004C0001A611A6922F000521A611B6972B64FF064
:1004D000E0233021C3F8084DD4E9003281F31188BC
:1004E0009D4683F30888104710BD00BF0000010837
:1004F00020000108FFFF0008002200200038024011
:100500002DE9F04F93B0AA4B00902022FF210AA8BA
:100510009D6800F0F1FBA74A1378A3B9A648012112
:1005200003601170302383F3118803680BB101F06D
:1005300053FAA24AA04800234FF47A7101F042FA1C
:10054000002383F31188009B13B19D4B009A1A601E
:100550009C4A009C1378032B1EBF00231370984AFB
:100560004FF0000A18BF5360D3465646D1460120CB
:1005700000F06AFB24B1924B1B68002B00F0118243
:10058000002000F06DFA0390039B002BF2DB0120AA
:1005900000F04AFB039B213B162BE8D801A252F83E
:1005A00023F000BF0106000829060008BD06000868
:1005B0006F0500086F0500086F0500084707000871
:1005C000170900083108000893080008BB08000854
:1005D000E10800086F050008F30800086F0500082F
:1005E00065090008A10600086F050008A9090008B0
:1005F0000D060008A10600086F0500089308000812
:100600000220FFF7C3FE002840F0F581009B022185
:10061000BAF1000F08BF1C4605A841F21233ADF82D
:10062000143000F03BFAA2E74FF47A7000F018FAA9
:10063000071EEBDB0220FFF7A9FE0028E6D0013FF2
:10064000052F00F2DA81DFE807F0030A0D101336F8
:1006500005230593042105A800F020FA17E054486B
:100660000421F9E758480421F6E758480421F3E744
:100670004FF01C08404600F03DFA08F104080590D0
:10068000042105A800F00AFAB8F12C0FF2D10120DC
:1006900000FA07F747EA0B0B5FFA8BFB4FF00009F4
:1006A00000F076FB26B10BF00B030B2B08BF0024E8
:1006B000FFF774FE5BE746480421CDE7002EA5D086
:1006C0000BF00B030B2BA1D10220FFF75FFE0746B7
:1006D00000289BD0012000F00BFA0220FFF7A6FEB5
:1006E00000261FFA86F8404600F012FA044690B140
:1006F0000021404600F01CFA01360028F1D1BA462C
:10070000044641F21213022105A8ADF814303E460A
:1007100000F0C4F92BE70120FFF788FE2546244BA3
:100720009B68AB4207D9284600F0E4F9013040F05D
:1007300067810435F3E7234B00251D70204BBA4633
:100740005D603E46ACE7002E3FF460AF0BF00B035C
:100750000B2B7FF45BAF0220FFF768FE322000F026
:100760007FF9B0F10008FFF651AF18F003077FF4EE
:100770004DAF0F4A926808EB050393423FF646AF30
:10078000B8F5807F3FF742AF124B0193B84523DDA8
:100790004FF47A7000F064F90390039A002AFFF690
:1007A00035AF019B039A03F8012B0137EDE700BF3A
:1007B000002200205C23002040220020B503000816
:1007C000602300205822002004220020082200205C
:1007D0000C2200205C220020C820FFF7D7FD07462E
:1007E00000283FF413AF1F2D11D8C5F12002424558
:1007F0000AAB25F0030028BF424683490192184402
:1008000000F054FA019A8048FF2100F075FA4FEA8F
:10081000A8037D490193C8F38702284600F074FAC3
:10082000064600283FF46DAF019B05EB830537E7D3
:100830000220FFF7ABFD00283FF4E8AE00F0A4F97A
:1008400000283FF4E3AE0027B846704B9B68BB42DC
:1008500018D91F2F11D80A9B01330ED027F003039C
:1008600012AA134453F8203C05934046042205A9DC
:1008700000F0C2FA04378046E7E7384600F03AF95C
:100880000590F2E7CDF81480042105A800F006F9E0
:1008900006E70023642104A8049300F0F5F800287B
:1008A0007FF4B4AE0220FFF771FD00283FF4AEAE36
:1008B000049800F051F90590E6E70023642104A8AC
:1008C000049300F0E1F800287FF4A0AE0220FFF7C7
:1008D0005DFD00283FF49AAE049800F04DF9EAE778
:1008E0000220FFF753FD00283FF490AE00F05CF9C2
:1008F000E1E70220FFF74AFD00283FF487AE05A993
:10090000142000F057F904210746049004A800F0D1
:10091000C5F83946B9E7322000F0A2F8071EFFF605
:1009200075AEBB077FF472AE384A926807EB0903D5
:1009300093423FF66BAE0220FFF728FD00283FF4FC
:1009400065AE27F003074F44B9453FF4A9AE4846CA
:1009500000F0D0F80421059005A800F09FF809F1F7
:100960000409F1E74FF47A70FFF710FD00283FF417
:100970004DAE00F009F9002844D00A9B01330BD09A
:1009800008220AA9002000F0BFF900283AD020224E
:10099000FF210AA800F0B0F9FFF700FD1C4800F0A5
:1009A00055FF13B0BDE8F08F002E3FF42FAE0BF0D3
:1009B0000B030B2B7FF42AAE0023642105A80593BB
:1009C00000F062F8074600287FF420AE0220FFF70F
:1009D000DDFC804600283FF419AEFFF7DFFC41F252
:1009E000883000F033FF059800F004FA464600F026
:1009F000CFF93C46BBE5064652E64FF0000905E656
:100A0000BA467EE637467CE65C22002000220020C3
:100A1000A086010070B50F4B1B780133DBB2012BB0
:100A20000C4611D80C4D29684FF47A730E6AA2FB5C
:100A30000332014622462846B047844204D1074B80
:100A400000221A70012070BD4FF4FA7000F0FEFE13
:100A50000020F8E710220020082600209423002020
:100A600007B50023024601210DF107008DF807307C
:100A7000FFF7D0FF20B19DF8070003B05DF804FB3D
:100A80004FF0FF30F9E700000A4608B50421FFF7F0
:100A9000C1FF80F00100C0B2404208BD30B4054C37
:100AA0002368DD69044B0A46AC460146204630BC4B
:100AB000604700BF08260020A086010070B501F045
:100AC000E5F9094E094D30800024286833888342B7
:100AD00008D901F0D5F92B6804440133B4F5803FFF
:100AE0002B60F2D370BD00BF962300206823002046
:100AF00001F07ABA00F1006000F5803000687047BC
:100B000000F10060920000F5803001F005BA0000AD
:100B1000054B1A68054B1B889B1A834202D9104467
:100B200001F0AEB900207047682300209623002012
:100B300038B5084D044629B128682044BDE838403E
:100B400001F0BEB92868204401F0A2F90028F3D0D2
:100B500038BD00BF6823002010F003030AD1B0F5B0
:100B6000047F05D200F10050A0F51040D0F8003805
:100B7000184670470023FBE700F10050A0F5104035
:100B8000D0F8100A70470000064991F8243033B1BC
:100B90000023086A81F824300822FFF7B1BF012042
:100BA000704700BF6C230020014B1868704700BFDE
:100BB000002004E070B5194B1D68194B0138C5F3CE
:100BC0000B0408442D0C04221E88A6420BD15C683D
:100BD0000A46013C824213460FD214F9016F4EB10E
:100BE00002F8016BF6E7013A03F10803ECD1814208
:100BF0000B4602D22C2203F8012B0A4A0524168840
:100C0000AE4204D1984284BF967803F8016B013C50
:100C100002F10402F3D1581A70BD00BF002004E0B5
:100C2000C4340008B0340008022804D1054B4FF04A
:100C300080429A6170470128FCD1024B4FF000526C
:100C4000F7E700BF00000240022804D1054B4FF433
:100C500080429A6170470128FCD1024B4FF4005248
:100C6000F7E700BF00000240022805D1064A536999
:100C700083F48043536170470128FCD1024A5369D1
:100C800083F40053F6E700BF0000024070B504464D
:100C90004FF47A764CB1412C254628BF412506FBFE
:100CA00005F000F0D3FD641BF4E770BD10B5002320
:100CB000934203D0CC5CC4540133F9E710BD00006B
:100CC00010B5013810F9013F3BB191F900409C4249
:100CD00003D11AB10131013AF4E71AB191F90020B8
:100CE000981A10BD1046FCE703460246D01A12F9C6
:100CF000011B0029FAD1704702440346934202D0F7
:100D000003F8011BFAE770472DE9F8431F4D14461D
:100D100095F824200746884652BBDFF870909CB3B4
:100D200095F824302BB92022FF2148462F62FFF787
:100D3000E3FF95F82400C0F10802A24228BF224632
:100D4000D6B24146920005EB8000FFF7AFFF95F861
:100D50002430A41B1E44F6B2082E17449044E4B27B
:100D600085F82460DBD1FFF70FFF0028D7D108E01A
:100D70002B6A03EB82038342CFD0FFF705FF0028E5
:100D8000CBD10020BDE8F8830120FBE76C230020D5
:100D9000024B1A78024B1A70704700BF9423002050
:100DA0001022002010B5104C104800F0B5F8214674
:100DB0000E4800F0DDF82468626DD2F8043843F084
:100DC0000203C2F804384FF47A70FFF75FFF084956
:100DD000204600F0D3F9626DD2F8043823F0020304
:100DE000C2F8043810BD00BF903500080826002066
:100DF000983500087047000030B5094D0A4491420B
:100E00000DD011F8013B5840082340F30004013B8A
:100E10002C4013F0FF0384EA5000F6D1EFE730BD19
:100E20002083B8ED026843681143016003B118479D
:100E30007047000013B5446BD4F894341A681178E5
:100E4000042915D1217C022912D119791289012393
:100E50008B4013420CD101A904F14C0001F0F8FEC3
:100E6000D4F89444019B21790246206800F0D0F91F
:100E700002B010BD143001F07BBE00004FF0FF3314
:100E8000143001F075BE00004C3001F04DBF000081
:100E90004FF0FF334C3001F047BF0000143001F039
:100EA00049BE00004FF0FF31143001F043BE000096
:100EB0004C3001F019BF00004FF0FF324C3001F010
:100EC00013BF00000020704710B5D0F894341A68A2
:100ED00011780429044617D1017C022914D15979CB
:100EE000528901238B4013420ED1143001F0DCFDF6
:100EF000024648B1D4F894444FF480736179206875
:100F0000BDE8104000F072B910BD0000406BFFF763
:100F1000DBBF0000704700007FB5124B0360002369
:100F20004360C0E90233012502260F4B05740446D5
:100F30000290019300F18402294600964FF48073D9
:100F4000143001F08DFD094B0294CDE9006304F5E6
:100F500023724FF48073294604F14C0001F054FED3
:100F600004B070BDE43400080D0F0008350E000811
:100F70000B68302282F311880A7903EB82029061B8
:100F80004A79093243F822008A7912B103EB8203CD
:100F900098610223C0F894140374002080F3118830
:100FA0007047000038B5037F044613B190F8543001
:100FB000ABB9201D01250221FFF734FF04F1140015
:100FC00025776FF0010100F069FC84F8545004F1BA
:100FD0004C006FF00101BDE8384000F05FBC38BD47
:100FE00010B5012104460430FFF71CFF00232377CE
:100FF00084F8543010BD000038B504460025143084
:1010000001F046FD04F14C00257701F015FE201D8E
:1010100084F854500121FFF705FF2046BDE8384011
:10102000FFF752BF90F8443003F06003202B07D144
:1010300090F84520212A4FF0000303D81F2A06D834
:1010400000207047222AFBD1C0E90E3303E0034A97
:1010500082630722C26303640120704711220020CB
:1010600037B5D0F894341A681178042904461AD197
:10107000017C022917D11979128901238B4013426F
:1010800011D100F14C05284601F096FE58B101A996
:10109000284601F0DDFDD4F89444019B21790246F5
:1010A000206800F0B5F803B030BD0000F0B500EBEB
:1010B000810385B09E6904460D46FEB1302383F35B
:1010C000118804EB8507301D0821FFF7ABFEFB6894
:1010D0005B691B6806F14C001BB1019001F0C6FD75
:1010E000019803A901F0B4FD024648B1039B2946CB
:1010F000204600F08DF8002383F3118805B0F0BD81
:10110000FB685A691268002AF5D01B8A013B13401C
:10111000F1D104F14402EAE7093138B550F8214031
:10112000DCB1302383F31188D4F894241368527906
:1011300003EB8203DB689B695D6845B1042160189D
:10114000FFF770FE294604F1140001F0B7FC2046B9
:10115000FFF7BAFE002383F3118838BD7047000003
:1011600001F016B8012303700023C0E90133C36105
:1011700083620362C36243620363704738B5044607
:10118000302383F311880025C0E90355C0E90555D4
:10119000416001F00DF80223237085F31188284681
:1011A00038BD000070B500EB810305465069DA6078
:1011B0000E46144618B110220021FFF79DFDA069CC
:1011C00018B110220021FFF797FD31462846BDE8EF
:1011D000704001F0B7B80000826802F0011282602E
:1011E0000022C0E90422826101F038B9F0B400EBBA
:1011F00081044789E4680125A4698D403D43458108
:1012000023600023A2606360F0BC01F053B90000CA
:10121000F0B400EB81040789E468012564698D401E
:101220003D43058123600023A2606360F0BC01F0B0
:10123000CDB9000070B50223002504460370C0E953
:101240000255C0E90455C564856180F8345001F049
:1012500015F863681B6823B129462046BDE8704035
:10126000184770BD0378052B10B504460AD080F8E6
:1012700050300523037043681B680BB10421984765
:101280000023A36010BD00000178052906D190F865
:101290005020436802701B6803B118477047000074
:1012A00070B590F83430044613B1002380F8343020
:1012B00004F14402204601F0F3F863689B68B3B977
:1012C00094F8443013F0600535D00021204601F039
:1012D00093FB0021204601F085FB63681B6813B176
:1012E000062120469847062384F8343070BD2046F6
:1012F00098470028E4D0B4F84A30E26B9A4288BF9D
:10130000E36394F94430E56B002B4FF0300380F237
:101310000381002D00F0F280092284F8342083F349
:1013200011880021D4E90E232046FFF771FF002326
:1013300083F31188DAE794F8452003F07F0343EA4A
:10134000022340F20232934200F0C58021D8B3F567
:10135000807F48D00DD8012B3FD0022B00F0938026
:10136000002BB2D104F14C02A2630222E263236497
:10137000C1E7B3F5817F00F09B80B3F5407FA4D136
:1013800094F84630012BA0D1B4F84C3043F002035E
:1013900032E0B3F5006F4DD017D8B3F5A06F31D060
:1013A000A3F5C063012B90D8636894F846205E686B
:1013B00094F84710B4F848302046B047002884D04D
:1013C0004368A3630368E3631AE0B3F5106F36D094
:1013D00040F6024293427FF478AF5C4BA363022352
:1013E000E3630023C3E794F84630012B7FF46DAF2D
:1013F000B4F84C3023F00203C4E90E55A4F84C3085
:10140000256478E7B4F84430B3F5A06F0ED194F8B2
:10141000463084F84E30204600F088FF63681B6831
:1014200013B1012120469847032323700023C4E908
:101430000E339CE704F14F03A3630123C3E7237832
:10144000042B10D1302383F311882046FFF7C4FE0C
:1014500085F311880321636884F84F5021701B685D
:101460000BB12046984794F84630002BDED084F824
:101470004F300423237063681B68002BD6D00221F1
:1014800020469847D2E794F848301D0603F00F0134
:1014900020460AD500F0F6FF012804D002287FF488
:1014A00014AF2B4B9AE72B4B98E700F0DDFFF3E7E7
:1014B00094F84630002B7FF408AF94F8483013F0CE
:1014C0000F01B3D01A06204602D501F0A9FAADE704
:1014D00001F09CFAAAE794F84630002B7FF4F5AEB1
:1014E00094F8483013F00F01A0D01B06204602D517
:1014F00001F082FA9AE701F075FA97E7142284F86E
:10150000342083F311882B462A4629462046FFF7CC
:101510006DFE85F31188E9E65DB1152284F834206B
:1015200083F311880021D4E90E232046FFF75EFEE5
:10153000FDE60B2284F8342083F311882B462A46DB
:1015400029462046FFF764FEE3E700BF1435000894
:101550000C3500081035000838B590F834300446D2
:10156000002B3ED0063BDAB20F2A34D80F2B32D8EC
:10157000DFE803F037313108223231313131313196
:1015800031313737C56BB0F84A309D4214D2C36849
:101590001B8AB5FBF3F203FB12556DB9302383F3BD
:1015A00011882B462A462946FFF732FE85F311881B
:1015B0000A2384F834300EE0142384F834303023C6
:1015C00083F3118800231A4619462046FFF70EFEC2
:1015D000002383F3118838BD036C03B198470023BF
:1015E000E7E70021204601F007FA0021204601F03C
:1015F000F9F963681B6813B1062120469847062352
:10160000D7E7000010B590F83430142B044629D0E9
:1016100017D8062B05D001D81BB110BD093B022BF2
:10162000FBD80021204601F0E7F90021204601F017
:10163000D9F963681B6813B1062120469847062331
:1016400019E0152BE9D10B2380F83430302383F3D4
:10165000118800231A461946FFF7DAFD002383F3A9
:101660001188DAE7C3689B695B68002BD5D1036CEE
:1016700003B19847002384F83430CEE70023037584
:10168000826803691B6899689142FBD25A680360BB
:1016900042601060586070470023037582680369D8
:1016A0001B6899689142FBD85A68036042601060D9
:1016B0005860704708B50846302383F311880B7DC6
:1016C000032B05D0042B0DD02BB983F3118808BD53
:1016D0008B6900221A604FF0FF338361FFF7CEFF62
:1016E0000023F2E7D1E9003213605A60F3E700000B
:1016F000FFF7C4BF054BD9680875186802681A60FF
:10170000536001220275D860FEF7FCBD98230020CB
:1017100030B50C4BDD684B1C87B004460FD02B4610
:10172000094A684600F04EF92046FFF7E3FF009BA8
:1017300013B1684600F050F9A86907B030BDFFF753
:10174000D9FFF9E798230020B5160008044B1A6862
:10175000DB6890689B68984294BF00200120704726
:1017600098230020084B10B51C68D86822681A60BE
:10177000536001222275DC60FFF78EFF0146204690
:10178000BDE81040FEF7BEBD9823002038B5074CD9
:1017900007490848012300252370656001F044FBD8
:1017A0000223237085F3118838BD00BF0026002076
:1017B0001C3500089823002000F044B9034A516802
:1017C00053685B1A9842FBD8704700BF001000E0D6
:1017D0008B60022308618B82084670478368A3F1FF
:1017E000840243F8142C026943F8442C426943F8FC
:1017F000402C094A43F8242CC26843F8182C0222D2
:1018000003F80C2C002203F80B2C044A43F8102C8C
:10181000A3F12000704700BF1D030008982300209B
:1018200008B5FFF7DBFFBDE80840FFF761BF000028
:10183000024BDB6898610F20FFF75CBF9823002004
:10184000302383F31188FFF7F3BF000008B501468A
:10185000302383F311880820FFF75AFF002383F316
:10186000118808BD064BDB6839B1426818605A60C0
:10187000136043600420FFF74BBF4FF0FF30704709
:10188000982300200368984206D01A6802605060CE
:1018900099611846FFF72CBF7047000038B5044621
:1018A0000D462068844200D138BD036823605C6027
:1018B0008561FFF71DFFF4E710B503689C68A2423D
:1018C0000CD85C688A600B604C6021605960996834
:1018D0008A1A9A604FF0FF33836010BD1B68121B99
:1018E000ECE700000A2938BF0A2170B504460D460E
:1018F0000A26601901F092FA01F07EFA041BA54253
:1019000003D8751C2E460446F3E70A2E04D9BDE819
:101910007040012001F0C8BA70BD0000F8B5144B4A
:101920000D46D96103F1100141600A2A19698260EC
:1019300038BF0A22016048601861A818144601F0F7
:101940005FFA0A2701F058FA431BA342064606D362
:101950007C1C281901F062FA27463546F2E70A2F67
:1019600004D9BDE8F840012001F09EBAF8BD00BFDF
:1019700098230020F8B506460D4601F03DFA0F4ABF
:10198000134653F8107F9F4206D12A46014630463F
:10199000BDE8F840FFF7C2BFD169BB68441A2C19F3
:1019A00028BF2C46A34202D92946FFF79BFF2246B7
:1019B00031460348BDE8F840FFF77EBF982300207A
:1019C000A823002010B4C0E9032300235DF8044BD2
:1019D0004361FFF7CFBF000010B5194C236998424F
:1019E0000DD0D0E90032816813605A609A680A44C9
:1019F0009A60002303604FF0FF33A36110BD2346BC
:101A0000026843F8102F53600022026022699A4254
:101A100003D1BDE8104001F0FBB9936881680B4425
:101A2000936001F0E9F92269E1699268441AA242DF
:101A3000E4D91144BDE81040091AFFF753BF00BFB5
:101A4000982300202DE9F047DFF8BC8008F110074B
:101A50002C4ED8F8105001F0CFF9D8F81C40AA68E5
:101A6000031B9A423ED81444D5E900324FF00009D6
:101A7000C8F81C4013605A60C5F80090D8F81030C0
:101A8000B34201D101F0C4F989F31188D5E90331DA
:101A900028469847302383F311886B69002BD8D0F0
:101AA00001F0AAF96A69A0EB04094A4582460DD201
:101AB000022001F0F9F90022D8F81030B34208D121
:101AC00051462846BDE8F047FFF728BF121A2244C6
:101AD000F2E712EB090938BF4A4629463846FFF7B4
:101AE000EBFEB5E7D8F81030B34208D01444211A01
:101AF000C8F81C00A960BDE8F047FFF7F3BEBDE8D9
:101B0000F08700BFA8230020982300200020704702
:101B1000FEE70000704700004FF0FF307047000004
:101B200002290CD0032904D00129074818BF00203E
:101B30007047032A05D8054800EBC20070470448E7
:101B400070470020704700BFF435000820220020B5
:101B5000A835000870B59AB00546084601A9144694
:101B600000F0C2F801A8FFF7BFF8431C5B00C5E90D
:101B700000340022237003236370C6B201AB023429
:101B80001046D1B28E4204F1020401D81AB070BDE1
:101B900013F8011B04F8021C04F8010C0132F0E7F1
:101BA00008B5302383F311880348FFF759FA00235F
:101BB00083F3118808BD00BF0826002090F8443048
:101BC00003F01F02012A07D190F845200B2A03D108
:101BD0000023C0E90E3315E003F06003202B08D189
:101BE000B0F848302BB990F84520212A03D81F2A95
:101BF00004D8FFF717BA222AEBD0FAE7034A826328
:101C00000722C26303640120704700BF182200202E
:101C100007B5052917D8DFE801F0191603191920AF
:101C2000302383F31188104A01900121FFF7BAFA9B
:101C300001980E4A0221FFF7B5FA0D48FFF7DCF9CB
:101C4000002383F3118803B05DF804FB302383F392
:101C500011880748FFF7A6F9F2E7302383F31188CC
:101C60000348FFF7BDF9EBE7483500086C3500087D
:101C70000826002038B50C4D0C4C0D492A4604F1BD
:101C80000800FFF767FF05F1CA0204F110000949D7
:101C9000FFF760FF05F5CA7204F118000649BDE8B8
:101CA0003840FFF757BF00BFD02A00202022002075
:101CB00028350008323500083D35000870B5044667
:101CC00008460D46FFF710F8C6B2204601340378E7
:101CD0000BB9184670BD32462946FEF7F1FF0028C1
:101CE000F3D10120F6E700002DE9F04705460C4648
:101CF000FEF7FAFF2B49C6B22846FFF7DFFF08B10F
:101D00000A36F6B228492846FFF7D8FF08B1103640
:101D1000F6B2632E0BD8DFF88C80DFF88C90234F5F
:101D2000DFF894A02E7846B92670BDE8F0872946E2
:101D30002046BDE8F04701F09DBB252E2ED107229D
:101D400041462846FEF7BCFF70B9194B224603F105
:101D5000100153F8040B42F8040B8B42F9D11B78A5
:101D6000137007351134DDE7082249462846FEF78F
:101D7000A7FF98B90F4BA21C197809090232C95D57
:101D800002F8041C13F8011B01F00F015345C95D53
:101D900002F8031CF0D118340835C3E704F8016BCE
:101DA0000135BFE7143600083D3500082E3600081F
:101DB0001C360008107AFF1F1C7AFF1FBFF34F8FDD
:101DC000024AD368DB03FCD4704700BF003C0240EA
:101DD00008B5094B1B7873B9FFF7F0FF074B1A6979
:101DE000002ABFBF064A5A6002F188325A601A6858
:101DF00022F480621A6008BD2E2D0020003C0240B3
:101E00002301674508B50B4B1B7893B9FFF7D6FF45
:101E1000094B1A6942F000421A611A6842F4805272
:101E20001A601A6822F480521A601A6842F48062BA
:101E30001A6008BD2E2D0020003C02400B28F0B592
:101E400016D80C4C0C4923787BB90C4D0E460C234C
:101E50004FF0006255F8047B46F8042B013B13F069
:101E6000FF033A44F6D10123237051F82000F0BD5E
:101E70000020FCE7602D0020302D002040360008B7
:101E8000014B53F820007047403600080C20704783
:101E90000B2810B5044601D9002010BDFFF7CEFF76
:101EA000064B53F824301844C21A0BB90120F4E74A
:101EB00012680132F0D1043BF6E700BF403600085B
:101EC0000B2810B5044621D8FFF778FFFFF780FFF5
:101ED0000F4AF323D360C300DBB243F4007343F033
:101EE00002031361136943F480331361FFF766FF44
:101EF000FFF7A4FF074B53F8241000F0D9F8FFF7C1
:101F000081FF2046BDE81040FFF7C2BF002010BD92
:101F1000003C024040360008F8B512F001031446B8
:101F200042D18218B2F1016F57D82D4B1B6813F0C4
:101F3000010352D02B4DFFF74BFFF323EB60FFF76C
:101F40003DFF40F20127032C15D824F00104661848
:101F5000244C401A40F20117B142236900EB0105FD
:101F600024D123F001032361FFF74CFF0120F8BDCA
:101F7000043C0430E7E78307E7D12B6923F440737F
:101F80002B612B693B432B6151F8046B0660BFF357
:101F90004F8FFFF713FF03689E42E9D02B6923F0B0
:101FA00001032B61FFF72EFF0020E0E723F44073CD
:101FB000236123693B4323610B882B80BFF34F8F41
:101FC000FFF7FCFE2D8831F8023BADB2AB42C3D027
:101FD000236923F001032361E4E71846C7E700BF44
:101FE00000380240003C0240084908B50B7828B18F
:101FF0001BB9FFF7EDFE01230B7008BD002BFCD0D1
:10200000BDE808400870FFF7FDBE00BF2E2D002080
:1020100010B50244064BD2B2904200D110BD441C10
:1020200000B253F8200041F8040BE0B2F4E700BF1F
:10203000502800400F4B30B51C6F240407D41C6F90
:1020400044F400741C671C6F44F400441C670A4C81
:10205000236843F4807323600244084BD2B2904259
:1020600000D130BD441C00B251F8045B43F820504D
:10207000E0B2F4E700380240007000405028004011
:1020800007B5012201A90020FFF7C2FF019803B0A4
:102090005DF804FB13B50446FFF7F2FFA04205D03C
:1020A000012201A900200194FFF7C4FF02B010BD76
:1020B00070470000034B1A681AB9034AD2F8742813
:1020C0001A607047642D00200030024008B5FFF709
:1020D000F1FF024B1868C0F3407008BD642D00206A
:1020E00070470000FEE700000A4B0B480B4A904285
:1020F0000BD30B4BDA1C121AC11E22F003028B42C7
:1021000038BF00220021FEF7F7BD53F8041B40F84A
:10211000041BECE7E8370008602E0020602E00204A
:10212000602E002070B5D0E915439E6800224FF064
:10213000FF3504EB42135101D3F800090028BEBF5C
:10214000D3F8000940F08040C3F80009D3F8000B31
:102150000028BEBFD3F8000B40F08040C3F8000B4E
:10216000013263189642C3F80859C3F8085BE0D2FD
:102170004FF00113C4F81C3870BD0000890141F014
:102180002001016103699B06FCD41220FFF716BBF6
:1021900010B5054C2046FEF7E5FF4FF0A043636500
:1021A000024BA36510BD00BF682D002094360008C7
:1021B00070B50378012B054650D12A4B446D9842E7
:1021C0001BD1294B5A6B42F080025A635A6D42F080
:1021D00080025A655A6D5A6942F080025A615A6902
:1021E00022F080025A610E2143205B6900F022FC3C
:1021F0001E4BE3601E4BC4F800380023C4F8003EB9
:10220000C02323606E6D4FF40413A3633369002B66
:10221000FCDA012333610C20FFF7D0FA3369DB07C6
:10222000FCD41220FFF7CAFA3369002BFCDA00262F
:10223000A6602846FFF776FF6B68C4F81068DB6875
:10224000C4F81468C4F81C684BB90A4BA3614FF07A
:10225000FF336361A36843F00103A36070BD064BC5
:10226000F4E700BF682D0020003802404014004011
:1022700003002002003C30C0083C30C0F8B5446D7B
:10228000054600212046FFF779FFA96D00234FF096
:1022900001128F68C4F834384FF00066C4F81C2867
:1022A0004FF0FF3004EB431201339F42C2F8006944
:1022B000C2F8006BC2F80809C2F8080BF2D20B682A
:1022C0006A6DEB65636210231361166916F01006E0
:1022D000FBD11220FFF772FAD4F8003823F4FE6322
:1022E000C4F80038A36943F4402343F01003A3610A
:1022F0000923C4F81038C4F814380A4BEB604FF0C7
:10230000C043C4F8103B084BC4F8003BC4F8106944
:10231000C4F80039EB6D03F1100243F48013EA6551
:10232000A362F8BD7036000840800010426D90F83E
:102330004E10D2F8003823F4FE6343EA0113C2F8CA
:10234000003870472DE9F84300EB8103456DDA68EA
:10235000166806F00306731E022B05EB41130C46AC
:1023600080460FFA81F94FEA41104FF00001C3F89F
:10237000101B4FF0010104F1100398BFB60401FADD
:1023800003F391698EBF334E06F1805606F5004681
:1023900000293AD0578A04F15801490137436F5058
:1023A000D5F81C180B43C5F81C382B180021C3F8AE
:1023B000101953690127611EA7409BB3138A928BA2
:1023C0009B08012A88BF5343D8F85C20981842EA3A
:1023D000034301F1400205EB8202C8F85C0021468C
:1023E00053602846FFF7CAFE08EB8900C3681B8AC2
:1023F00043EA8453483464011E432E51D5F81C38F7
:102400001F43C5F81C78BDE8F88305EB4917D7F8DA
:10241000001B21F40041C7F8001BD5F81C1821EA65
:102420000303C0E704F13F0305EB83030A4A5A6044
:1024300028462146FFF7A2FE05EB4910D0F80039E7
:1024400023F40043C0F80039D5F81C3823EA070705
:10245000D7E700BF0080001000040002826D126800
:10246000C265FFF75FBE00005831436D49015B58FC
:1024700013F4004004D013F4001F0CBF022001200D
:10248000704700004831436D49015B5813F4004028
:1024900004D013F4001F0CBF02200120704700007D
:1024A00000EB8101CB68196A0B6813604B685360BD
:1024B0007047000000EB810330B5DD68AA6913683E
:1024C000D36019B9402B84BF402313606B8A146812
:1024D000426D1C44013CB4FBF3F46343033323F02B
:1024E000030302EB411043EAC44343F0C043C0F886
:1024F000103B2B6803F00303012B09B20ED1D2F875
:10250000083802EB411013F4807FD0F8003B14BF71
:1025100043F0805343F00053C0F8003B02EB4112FC
:10252000D2F8003B43F00443C2F8003B30BD00004A
:102530002DE9F041244D6E6D06EB40130446D3F8AF
:10254000087BC3F8087B38070AD5D6F81438190772
:1025500006D505EB84032146DB6828465B6898476F
:10256000FA071FD5D6F81438DB071BD505EB840313
:10257000D968CCB98B69488A5A68B2FBF0F600FB7F
:1025800016228AB91868DA6890420DD2121AC3E985
:102590000024302383F311880B482146FFF78AFF7C
:1025A00084F31188BDE8F081012303FA04F26B89FA
:1025B00023EA02036B81CB68002BF3D0214602484B
:1025C000BDE8F041184700BF682D002000EB8103F3
:1025D00070B5DD68436D6C692668E6604A0156BBDC
:1025E0001A444FF40020C2F810092A6802F00302CE
:1025F000012A0AB20ED1D3F8080803EB421410F4F2
:10260000807FD4F8000914BF40F0805040F00050A3
:10261000C4F8000903EB4212D2F8000940F004406C
:10262000C2F80009D3F83408012202FA01F101438B
:10263000C3F8341870BD19B9402E84BF4020206003
:1026400020682E8A8419013CB4FBF6F440EAC440A9
:1026500040F000501A44C6E72DE9F8433B4D6E6D3B
:1026600006EB40130446D3F80889C3F8088918F02C
:10267000010F4FEA40171AD0D6F81038DB0716D5ED
:1026800005EB8003D9684B691868DA68904230D24C
:10269000121A4FF000091A60C3F80490302383F334
:1026A000118821462846FFF791FF89F3118818F019
:1026B000800F1CD0D6F834380126A640334216D0FD
:1026C00005EB84036D6DD3F80CC0DCF814200134E5
:1026D000E4B2D2F800E005EB04342F4451687145B0
:1026E00015D3D5F8343823EA0606C5F83468BDE8B2
:1026F000F883012303FA04F22B8923EA02032B81D6
:102700008B68002BD3D0214628469847CFE7BCF8EA
:102710001000AEEB0103834228BF0346D7F8180927
:1027200080B2B3EB800FE2D89068A0F1040959F8A9
:10273000048FC4F80080A0EB09089844B8F1040F96
:10274000F5D818440B4490605360C7E7682D00200B
:102750002DE9F74FA24C656D6E69AB691E4016F40A
:1027600080586E6107D02046FEF764FD03B0BDE8D7
:10277000F04F00F047BC002E12DAD5F8003E984822
:102780009B071EBFD5F8003E23F00303C5F8003EAB
:10279000D5F8043823F00103C5F80438FEF774FDBA
:1027A000370505D58E48FFF7BDFC8D48FEF75AFD6D
:1027B000B0040CD5D5F8083813F0060FEB6823F4F5
:1027C00070530CBF43F4105343F4A053EB60310734
:1027D0001BD56368DB681BB9AB6923F00803AB61E9
:1027E0002378052B0CD1D5F8003E7D489A071EBFF3
:1027F000D5F8003E23F00303C5F8003EFEF744FD84
:102800006368DB680BB176489847F30274D4B7026B
:1028100027D5D4F85490DFF8C8B100274FF0010A4B
:1028200009EB4712D2F8003B03F44023B3F5802FA5
:1028300011D1D2F8003B002B0DDA62890AFA07F3B6
:1028400022EA0303638104EB8703DB68DB6813B1CF
:10285000394658469847A36D01379B68FFB29F429F
:10286000DED9F00617D5676D3A6AC2F30A1002F096
:102870000F0302F4F012B2F5802F00F08580B2F55C
:10288000402F08D104EB83030022DB681B6A07F5A5
:10289000805790426AD13003D5F8184813D5E10328
:1028A00002D50020FFF744FEA20302D50120FFF766
:1028B0003FFE630302D50220FFF73AFE270302D54D
:1028C0000320FFF735FE75037FF550AFE00702D513
:1028D0000020FFF7C1FEA10702D50120FFF7BCFED3
:1028E000620702D50220FFF7B7FE23077FF53EAF50
:1028F0000320FFF7B1FE39E7636DDFF8E4A0019331
:1029000000274FF00109A36D9B685FFA87FB9B4589
:102910003FF67DAF019B03EB4B13D3F8001901F495
:102920004021B1F5802F1FD1D3F8001900291BDAFF
:10293000D3F8001941F09041C3F80019D3F80019F9
:102940000029FBDB5946606DFFF718FC218909FA65
:102950000BF321EA0303238104EB8B03DB689B6801
:1029600013B15946504698470137CCE7910708BF45
:10297000D7F80080072A98BF03F8018B02F1010203
:1029800098BF4FEA182884E7023304EB830207F567
:1029900080575268D2F818C0DCF80820DCE9001C27
:1029A000A1EB0C0C002188420AD104EB830463687C
:1029B0009B699A6802449A605A6802445A606AE7BE
:1029C00011F0030F08BFD7F800808C4588BF02F8CC
:1029D000018B01F1010188BF4FEA1828E3E700BF2E
:1029E000682D0020436D03EB4111D1F8003B43F407
:1029F0000013C1F8003B7047436D03EB4111D1F860
:102A0000003943F40013C1F800397047436D03EBFC
:102A10004111D1F8003B23F40013C1F8003B70478B
:102A2000436D03EB4111D1F8003923F40013C1F8D1
:102A30000039704700F1604303F561430901C9B2F1
:102A400083F80013012200F01F039A4043099B0002
:102A500003F1604303F56143C3F880211A607047B6
:102A600030B5039C0172043304FB0325C0E906530F
:102A7000049B03630021059BC160C0E90000C0E91D
:102A80000422C0E90842C0E90A11436330BD0000D6
:102A9000416A0022C0E90411C0E90A22C2606FF055
:102AA0000101FEF7FBBE0000D0E90432934201D1E0
:102AB000C2680AB9181D7047002070470369196081
:102AC000C2680132C260C2691344826903619342E1
:102AD00024BF436A03610021FEF7D4BE38B5044623
:102AE0000D46E3683BB16269131D1268A36213448B
:102AF000E362002007E0237A33B929462046FEF737
:102B0000B1FE0028EDDA38BD6FF00100FBE70000F0
:102B1000C368C269013BC36043691344826943616E
:102B2000934224BF436A436100238362036B03B172
:102B30001847704770B53023044683F31188866ABE
:102B40003EB9FFF7CBFF054618B186F3118828463A
:102B500070BDA36AE26A13F8015BA362934202D3D9
:102B60002046FFF7D5FF002383F31188EFE700002D
:102B70002DE9F84F04460E46174698464FF03009A7
:102B800089F311880025AA46D4F828B0BBF1000FBC
:102B900009D141462046FFF7A1FF20B18BF31188F0
:102BA0002846BDE8F88FD4E90A12A7EB050B521AA4
:102BB000934528BF9346BBF1400F1BD9334601F123
:102BC000400251F8040B43F8040B9142F9D1A36A77
:102BD00040334036A3624035D4E90A239A4202D3F7
:102BE0002046FFF795FF8AF31188BD42D8D289F3BA
:102BF0001188C9E730465A46FEF758F8A36A5B4485
:102C00005E44A3625D44E7E710B5029C01720433A1
:102C100003FB0421C0E906130023C0E90A33039B28
:102C20000363049BC460C0E90000C0E90422C0E95A
:102C30000842436310BD0000026AC260426AC0E9F4
:102C400004220022C0E90A226FF00101FEF726BE2D
:102C5000D0E904239A4201D1C26822B9184650F83B
:102C6000043B0B60704700231846FAE7C368C2694B
:102C70000133C3604369134482694361934224BFB3
:102C8000436A43610021FEF7FDBD000038B50446EC
:102C90000D46E3683BB123691A1DA262E269134441
:102CA000E362002007E0237A33B929462046FEF785
:102CB000D9FD0028EDDA38BD6FF00100FBE7000018
:102CC00003691960C268013AC260C269134482692B
:102CD0000361934224BF436A036100238362036B51
:102CE00003B118477047000070B530230D46044605
:102CF000114683F31188866A2EB9FFF7C7FF10B11A
:102D000086F3118870BDA36A1D70A36AE26A01335D
:102D10009342A36204D3E16920460439FFF7D0FF50
:102D2000002080F31188EDE72DE9F84F04460D46A9
:102D3000904699464FF0300A8AF311880026B34630
:102D4000A76A4FB949462046FFF7A0FF20B187F395
:102D500011883046BDE8F88FD4E90A073A1AA8EB83
:102D60000607974228BF1746402F1BD905F140039D
:102D700055F8042B40F8042B9D42F9D1A36A403347
:102D8000A3624036D4E90A239A4204D3E16920467B
:102D90000439FFF795FF8BF311884645D9D28AF3A2
:102DA0001188CDE729463A46FDF780FFA36A3B44E8
:102DB0003D44A3623E44E5E7D0E904239A4217D19B
:102DC000C3689BB1836A8BB1043B9B1A0ED013601E
:102DD000C368013BC360C3691A44836902619A42B4
:102DE00024BF436A036100238362012318467047AE
:102DF0000023FBE700F030B94FF08043586A70477A
:102E00004FF08043002258631A610222DA60704753
:102E10004FF080430022DA60704700004FF080439B
:102E200058637047FEE7000070B51B4B0163002537
:102E3000044686B0586085620E4600F0BFF804F183
:102E40001003C4E904334FF0FF33C4E90635C4E985
:102E50000044A560E562FFF7CFFF2B460246C4E9B8
:102E6000082304F134010D4A256580232046FEF72E
:102E7000AFFC0123E0600A4A037500927268019278
:102E8000B268CDE90223074B6846CDE90435FEF769
:102E9000C7FC06B070BD00BF00260020A0360008A9
:102EA000A5360008252E0008024AD36A1843D062CE
:102EB000704700BF982300204B6843608B68836095
:102EC000CB68C3600B6943614B6903628B694362E2
:102ED0000B6803607047000008B5264B26481A6946
:102EE00040F2FF110A431A611A6922F4FF7222F0BC
:102EF00001021A611A691A6B0A431A631A6D0A43AE
:102F00001A651E4A1B6D1146FFF7D6FF02F11C0120
:102F100000F58060FFF7D0FF02F1380100F5806016
:102F2000FFF7CAFF02F1540100F58060FFF7C4FF0C
:102F300002F1700100F58060FFF7BEFF02F18C0125
:102F400000F58060FFF7B8FF02F1A80100F580608E
:102F5000FFF7B2FF02F1C40100F58060FFF7ACFF9C
:102F600002F1E00100F58060FFF7A6FFBDE8084030
:102F700000F0EEB80038024000000240AC36000815
:102F800008B500F059FAFEF701FCFFF793F8BDE829
:102F90000840FEF76FBE000070470000EFF30983A2
:102FA00005494A6B22F001024A63683383F30988BA
:102FB000002383F31188704700EF00E0302080F396
:102FC000118862B60C4B0D4AD96821F4E0610904FE
:102FD000090C0A43DA60D3F8FC20094942F08072F8
:102FE000C3F8FC200A6842F001020A602022DA7766
:102FF00083F82200704700BF00ED00E00003FA05EF
:10300000001000E010B5302383F311880E4B5B688D
:1030100013F4006314D0F1EE103AEFF30984683C26
:103020004FF08073E361094BDB6B236684F30988FF
:10303000FEF78CFB10B1064BA36110BD054BFBE7FF
:1030400083F31188F9E700BF00ED00E000EF00E036
:103050002F030008320300080F4B1A6C42F00102E4
:103060001A641A6E42F001021A660C4A1B6E9368CB
:1030700043F0010393604FF0804353229A624FF074
:10308000FF32DA6200229A615A63DA605A600122E2
:103090005A611A60704700BF00380240002004E007
:1030A0004FF0804208B51169D3680B40D9B2C943CB
:1030B0009B07116107D5302383F31188FEF77CFB52
:1030C000002383F3118808BD1F4B1A696FEAC252AF
:1030D0006FEAD2521A611A69C2F308021A614FF0FC
:1030E000FF301A695A69586100215A6959615A6951
:1030F0001A6A62F080521A621A6A02F080521A62E8
:103100001A6A5A6A58625A6A59625A6A1A6C42F0C2
:1031100080521A641A6E42F080521A661A6E0B4A76
:10312000106840F480701060186F00F44070B0F5C3
:10313000007F1EBF4FF4803018671967536823F46F
:103140000073536000F054B9003802400070004032
:10315000334B4FF080521A64324A4FF440411160B1
:103160001A6842F001021A601A689107FCD59A6841
:1031700022F003029A602A4B9A6812F00C02FBD1EB
:10318000196801F0F90119609A601A6842F48032F6
:103190001A601A689203FCD55A6F42F001025A670E
:1031A0001F4B5A6F9007FCD51F4A5A601A6842F0AD
:1031B00080721A601B4A53685904FCD5184B1A6870
:1031C0009201FCD5194A9A60194B1A68194B9A4218
:1031D000194B21D1194A1168194A91421CD140F268
:1031E00005121A60144A136803F00F03052BFAD175
:1031F0000B4B9A6842F002029A609A6802F00C0245
:10320000082AFAD15A6C42F480425A645A6E42F447
:1032100080425A665B6E704740F20572E1E700BF7C
:10322000003802400070004008544007009488387D
:10323000002004E011640020003C024000ED00E0AA
:1032400041C20F41074A08B5536903F001035361B6
:1032500023B1054A13680BB150689847BDE8084090
:10326000FFF7D0BE003C0140E02D0020074A08B522
:10327000536903F00203536123B1054A93680BB10C
:10328000D0689847BDE80840FFF7BCBE003C01404D
:10329000E02D0020074A08B5536903F00403536189
:1032A00023B1054A13690BB150699847BDE808403E
:1032B000FFF7A8BE003C0140E02D0020074A08B5FA
:1032C000536903F00803536123B1054A93690BB1B5
:1032D000D0699847BDE80840FFF794BE003C014024
:1032E000E02D0020074A08B5536903F0100353612D
:1032F00023B1054A136A0BB1506A9847BDE80840EC
:10330000FFF780BE003C0140E02D0020164B10B5B9
:103310005C6904F478725A61A30604D5134A936A6F
:103320000BB1D06A9847600604D5104A136B0BB1F5
:10333000506B9847210604D50C4A936B0BB1D06BA8
:103340009847E20504D5094A136C0BB1506C9847B5
:10335000A30504D5054A936C0BB1D06C9847BDE822
:103360001040FFF74FBE00BF003C0140E02D0020A1
:10337000194B10B55C6904F47C425A61620504D5AE
:10338000164A136D0BB1506D9847230504D5134AA7
:10339000936D0BB1D06D9847E00404D50F4A136EBE
:1033A0000BB1506E9847A10404D50C4A936E0BB133
:1033B000D06E9847620404D5084A136F0BB1506F62
:1033C0009847230404D5054A936F0BB1D06F9847F3
:1033D000BDE81040FFF716BE003C0140E02D002084
:1033E00008B5FFF75DFEBDE80840FFF70BBE000023
:1033F000062108B50846FFF71DFB06210720FFF749
:1034000019FB06210820FFF715FB06210920FFF70D
:1034100011FB06210A20FFF70DFB06211720FFF7FD
:1034200009FB06212820FFF705FBBDE8084007211E
:103430001C20FFF7FFBA000008B5FFF745FE00F0BB
:103440000BF8FDF78DFEFDF765FDFFF7A5FDBDE867
:103450000840FFF7CFBC00000023054A194601339E
:10346000102BC2E9001102F10802F8D1704700BF29
:10347000E02D0020034611F8012B03F8012B002A50
:10348000F9D1704753544D3332463F3F3F005354B8
:103490004D3332463430780053544D333246343253
:1034A000780053544D3332463434365858000000B7
:1034B000012033000010410001105A000310590090
:1034C00007103100000000008434000813040000DD
:1034D0008E3400081904000098340008210400000C
:1034E000A234000800000000910E00087D0E0008C4
:1034F000B90E0008A50E0008B10E00089D0E0008C8
:10350000890E0008750E0008C50E000800000000B6
:1035100001000000000000006330000018350008C2
:10352000F0230020002600204172647550696C6F02
:10353000740025424F415244252D424C00255345ED
:103540005249414C2500000002000000000000002C
:10355000AD1000081911000840004000A02A00200A
:10356000B02A00200200000000000000030000005C
:10357000000000005D1100080000000010000000C5
:10358000C02A002000000000010000000000000030
:10359000682D002001010200111C0008211B0008F9
:1035A000BD1B0008A11B000843000000B035000847
:1035B00009024300020100C03209040000010202B6
:1035C0000100052400100105240100010424020269
:1035D0000524060001070582030800FF0904010015
:1035E000020A0000000705010240000007058102F1
:1035F0004000000012000000FC350008120110011C
:1036000002000040091241570002010203010000BC
:103610000403090425424F41524425005370656557
:1036200064794265654634303557494E470030313C
:103630003233343536373839414243444546000049
:10364000004000000040000000400000004000007A
:103650000000010000000200000002000000020063
:103660000000020000000200000002000000020052
:1036700000000000A11200085915000805160008F6
:1036800040004000C82D0020C82D0020010000008F
:10369000D82D002080000000400100000300000041
:1036A0006D61696E0069646C650000000001801640
:1036B00000000000AAAAAAAA00010000FF9F0000C3
:1036C0000000000000A00A0000000001000000004F
:1036D000AAAAAAAA00000001FFFF00000000000043
:1036E000000000000000001000000000AAAAAAAA22
:1036F00000000010FFFF00000000000000000000BC
:103700000000000000000000AAAAAAAA0000000011
:10371000FFFF0000000000000000000000000000AB
:1037200000000000AAAAAAAA00000000FFFF0000F3
:103730000000000000000000000000000000000089
:10374000AAAAAAAA00000000FFFF000000000000D3
:10375000000000000000000000000000AAAAAAAAC1
:1037600000000000FFFF000000000000000000005B
:1037700000000000000000000A000000000000003F
:103780000300000000000000000000000000000036
:103790000000000000000000000000000000000029
:1037A00000000000000000005204000000000000C3
:1037B00000000F0000000000FF009600000000085D
:1037C0000096000000000800040000001036000809
:1037D00000000000000000000000000000000000E9
:1037E0000000000000000000FFFFFFFFFFFFFFFFE1
:1037F000FFFFFFFFFFFFFFFFFFFFFFFFFFFFFFFFD9
:10380000FFFFFFFFFFFFFFFFFFFFFFFFFFFFFFFFC8
:10381000FFFFFFFFFFFFFFFFFFFFFFFFFFFFFFFFB8
:10382000FFFFFFFFFFFFFFFFFFFFFFFFFFFFFFFFA8
:020000040801F1
:100000000006002099120108491C0708A51B0708D3
:10001000111C0708A51B0708DD1B07089B12010818
:100020009B1201089B1201089B120108C195090847
:100030009B1201089B1201089B1201089B120108E8
:100040009B1201089B1201089B1201089B120108D8
:100050009B1201089B12010859A1090881A10908F6
:10006000A9A10908D1A10908F9A109084D45090864
:1000700075450908A1450908CD450908F94509084C
:10008000214609084D460908D14409089B12010878
:100090009B1201089B1201089B12010821A209086A
:1000A0006DA3090881A3090895A3090899A3090864
:1000B0009DA30908B1A30908C5A30908D94B0908DC
:1000C000814D09089B1201089B1201089B1201082F
:1000D0009B120108F5A2090809A309081DA3090834
:1000E00085A209089B1201089B120108E9A30908CF
:1000F000EDA3090801A4090805A40908794609081F
:100100009B1201089B120108D9A309089B12010840
:1001100031A3090845A309089B1201089B12010895
:10012000A5460908CD460908F946090825470908E2
:10013000514709089B1201089B1201089B120108F4
:100140009B1201089B1201089B120108ED9C0908F3
:1001500079470908A5470908D147090859A309089B
:100160009B1201089B1201089B1201089B120108B7
:100170009B1201089B1201089B1201089B120108A7
:100180009B1201089B1201089B1201089B12010897
:100190009B1201089B1201089B1201089B12010887
:1001A0009B1201089B1201089B1201089B12010877
:1001B0009B1201089B1201089B1201089B12010867
:1001C0009B1201089B1201089B1201089B12010857
:1001D0009B1201089B1201089B1201089B12010847
:1001E00071250108F1AD0108259904083DBA0408FC
:1001F00019240508DD2B0508152F0508A59305080A
:10020000E9B00508B53D060861530608B96006085F
:10021000150D0708B912070821C10708DD030808F2
:10022000B9240808B1720808C999080885B00808F7
:10023000E9DF080815E608080000000000000000DB
:1002400081F0004102E000BF83F0004330B54FEA87
:1002500041044FEA430594EA050F08BF90EA020FF4
:100260001FBF54EA000C55EA020C7FEA645C7FEA87
:10027000655C00F0E2804FEA5454D4EB5555B8BFAA
:100280006D420CDD2C4480EA020281EA030382EA1B
:10029000000083EA010180EA020281EA0303362DAD
:1002A00088BF30BD11F0004F4FEA01314FF4801C80
:1002B0004CEA113102D0404261EB410113F0004F92
:1002C0004FEA03334CEA133302D0524263EB430349
:1002D00094EA050F00F0A780A4F10104D5F1200EE7
:1002E0000DDB02FA0EFC22FA05F2801841F1000142
:1002F00003FA0EF2801843FA05F359410EE0A5F116
:1003000020050EF1200E012A03FA0EFC28BF4CF046
:10031000020C43FA05F3C01851EBE37101F00045FC
:1003200007D54FF0000EDCF1000C7EEB00006EEB09
:100330000101B1F5801F1BD3B1F5001F0CD3490893
:100340005FEA30004FEA3C0C04F101044FEA4452EA
:1003500012F5800F80F09A80BCF1004F08BF5FEA71
:10036000500C50F1000041EB045141EA050130BD51
:100370005FEA4C0C404141EB0101013C28BFB1F563
:10038000801FE9D291F0000F04BF01460020B1FAAE
:1003900081F308BF2033A3F10B03B3F120020CDA81
:1003A0000C3208DD02F1140CC2F10C0201FA0CF05F
:1003B00021FA02F10CE002F11402D8BFC2F1200CC4
:1003C00001FA02F120FA0CFCDCBF41EA0C0190407A
:1003D000E41AA2BF01EB0451294330BD6FEA0404C3
:1003E0001F3C1CDA0C340EDC04F11404C4F12002AE
:1003F00020FA04F001FA02F340EA030021FA04F3C0
:1004000045EA030130BDC4F10C04C4F1200220FA16
:1004100002F001FA04F340EA0300294630BD21FA54
:1004200004F0294630BD94F0000F83F4801306BF1A
:1004300081F480110134013D4EE77FEA645C18BF0E
:100440007FEA655C29D094EA050F08BF90EA020FA5
:1004500005D054EA000C04BF1946104630BD91EA9D
:10046000030F1EBF0021002030BD5FEA545C05D1A0
:100470004000494128BF41F0004130BD14F58004DF
:100480003CBF01F5801130BD01F0004545F0FE4153
:1004900041F470014FF0000030BD7FEA645C1ABF88
:1004A000194610467FEA655C1CBF0B46024650EABF
:1004B000013406BF52EA033591EA030F41F40021EB
:1004C00030BD00BF90F0000F04BF0021704730B571
:1004D0004FF4806404F132044FF000054FF0000146
:1004E00050E700BF90F0000F04BF0021704730B507
:1004F0004FF4806404F1320410F0004548BF4042DC
:100500004FF000013EE700BF42004FEAE2014FEA30
:1005100031014FEA02701FBF12F07F4393F07F4F0B
:1005200081F06051704732F07F4208BF704793F00E
:100530007F4F04BF41F40021704730B54FF4607421
:1005400001F0004521F000411CE700BF50EA010224
:1005500008BF704730B54FF000050AE050EA0102CD
:1005600008BF704730B511F0004502D5404261EB3D
:1005700041014FF4806404F132045FEA915C3FF47E
:10058000D8AE4FF003025FEADC0C18BF03325FEA1B
:10059000DC0C18BF033202EBDC02C2F1200300FACC
:1005A00003FC20FA02F001FA03FE40EA0E0021FAF1
:1005B00002F11444BDE600BF70B54FF0FF0C4CF4DF
:1005C000E06C1CEA11541DBF1CEA135594EA0C0F91
:1005D00095EA0C0F00F0DEF82C4481EA030621EACC
:1005E0004C5123EA4C5350EA013518BF52EA033507
:1005F00041F4801143F4801338D0A0FB02CE4FF0B9
:100600000005E1FB02E506F00042E0FB03E54FF0E8
:100610000006E1FB03569CF0000F18BF4EF0010EE0
:10062000A4F1FF04B6F5007F64F5407404D25FEADC
:100630004E0E6D4146EB060642EAC62141EA55518F
:100640004FEAC52040EA5E504FEACE2EB4F1FD0CD1
:1006500088BFBCF5E06F1ED8BEF1004F08BF5FEA4F
:10066000500E50F1000041EB045170BD06F0004601
:1006700046EA010140EA020081EA0301B4EB5C04AE
:10068000C2BFD4EB0C0541EA045170BD41F48011A6
:100690004FF0000E013C00F3AB8014F1360FDEBFCB
:1006A000002001F0004170BDC4F10004203C35DAA7
:1006B0000C341BDC04F11404C4F1200500FA05F32A
:1006C00020FA04F001FA05F240EA020001F00042CB
:1006D00021F0004110EBD37021FA04F642EB060141
:1006E0005EEA430E08BF20EAD37070BDC4F10C046B
:1006F000C4F1200500FA04F320FA05F001FA04F22F
:1007000040EA020001F0004110EBD37041F100011A
:100710005EEA430E08BF20EAD37070BDC4F1200525
:1007200000FA05F24EEA020E20FA04F301FA05F28D
:1007300043EA020321FA04F001F0004121FA04F235
:1007400020EA020000EBD3705EEA430E08BF20EA05
:10075000D37070BD94F0000F0FD101F0004640003F
:1007600041EB010111F4801F08BF013CF7D041EAC1
:10077000060195F0000F18BF704703F000465200C5
:1007800043EB030313F4801F08BF013DF7D043EA96
:100790000603704794EA0C0F0CEA135518BF95EA4C
:1007A0000C0F0CD050EA410618BF52EA4306D1D1D3
:1007B00081EA030101F000414FF0000070BD50EAF2
:1007C000410606BF1046194652EA430619D094EA7C
:1007D0000C0F02D150EA013613D195EA0C0F05D166
:1007E00052EA03361CBF104619460AD181EA0301BA
:1007F00001F0004141F0FE4141F470014FF0000072
:1008000070BD41F0FE4141F4780170BD70B54FF00C
:10081000FF0C4CF4E06C1CEA11541DBF1CEA13558C
:1008200094EA0C0F95EA0C0F00F0A7F8A4EB05046E
:1008300081EA030E52EA03354FEA013100F0888065
:100840004FEA03334FF0805545EA131343EA12632E
:100850004FEA022245EA111545EA10654FEA0026E3
:100860000EF000419D4208BF964244F1FD0404F59C
:10087000407402D25B084FEA3202B61A65EB0305F8
:100880005B084FEA32024FF480104FF4002CB6EBB5
:10089000020E75EB030E22BFB61A754640EA0C0035
:1008A0005B084FEA3202B6EB020E75EB030E22BF75
:1008B000B61A754640EA5C005B084FEA3202B6EBB6
:1008C000020E75EB030E22BFB61A754640EA9C0075
:1008D0005B084FEA3202B6EB020E75EB030E22BF45
:1008E000B61A754640EADC0055EA060E18D04FEA03
:1008F000051545EA16754FEA06164FEAC30343EAA3
:1009000052734FEAC2025FEA1C1CC0D111F4801F6F
:100910000BD141EA00014FF000004FF0004CB6E768
:1009200011F4801F04BF01430020B4F1FD0C88BF07
:10093000BCF5E06F3FF6AFAEB5EB030C04BFB6EB12
:10094000020C5FEA500C50F1000041EB045170BD05
:100950000EF0004E4EEA113114EB5C04C2BFD4EB32
:100960000C0541EA045170BD41F480114FF0000EB6
:10097000013C90E645EA060E8DE60CEA135594EA32
:100980000C0F08BF95EA0C0F3FF43BAF94EA0C0F35
:100990000AD150EA01347FF434AF95EA0C0F7FF4AA
:1009A00025AF104619462CE795EA0C0F06D152EAFE
:1009B00003353FF4FDAE1046194622E750EA4106E2
:1009C00018BF52EA43067FF4C5AE50EA41047FF4F3
:1009D0000DAF52EA43057FF4EBAE12E74FF0FF3C58
:1009E00006E000BF4FF0010C02E000BF4FF0010C29
:1009F0004DF804CD4FEA410C7FEA6C5C4FEA430CA2
:100A000018BF7FEA6C5C1BD001B050EA410C0CBFF0
:100A100052EA430C91EA030F02BF90EA020F002052
:100A2000704710F1000F91EA030F58BF994208BFB9
:100A300090422CBFD8176FEAE37040F00100704776
:100A40004FEA410C7FEA6C5C02D150EA013C07D1CD
:100A50004FEA430C7FEA6C5CD6D152EA033CD3D018
:100A60005DF8040B704700BF8446104662468C4612
:100A70001946634600E000BF01B5FFF7B7FF002845
:100A800048BF10F1000F01BD4DF808EDFFF7F4FF6E
:100A90000CBF012000205DF808FB00BF4DF808EDF9
:100AA000FFF7EAFF34BF012000205DF808FB00BF1C
:100AB0004DF808EDFFF7E0FF94BF012000205DF83E
:100AC00008FB00BF4DF808EDFFF7CEFF94BF0120F3
:100AD00000205DF808FB00BF4DF808EDFFF7C4FFEC
:100AE00034BF012000205DF808FB00BF4FEA410C35
:100AF0007FEA6C5C02D150EA013C0AD14FEA430C18
:100B00007FEA6C5C02D152EA033C02D14FF0000054
:100B100070474FF0010070474FEA410212F5001292
:100B200015D211D56FF47873B3EB625212D94FEA34
:100B3000C12343F0004343EA505311F0004F23FA1E
:100B400002F018BF404270474FF00000704750EA73
:100B5000013005D111F0004008BF6FF00040704730
:100B60004FF00000704700BF4A0011D212F500128A
:100B700011D20DD56FF47873B3EB62520ED44FEAF5
:100B8000C12343F0004343EA505323FA02F0704775
:100B90004FF00000704750EA013002D14FF0FF30B3
:100BA00070474FF0000070474FEA4102B2F1E04356
:100BB00024BFB3F5001CDCF1FE5C0DD901F0004C44
:100BC0004FEAC0024CEA5070B2F1004F40EB830094
:100BD00008BF20F00100704711F0804F21D113F1C0
:100BE0003872BCBF01F00040704741F480114FEAF9
:100BF0005252C2F11802C2F1200C10FA0CF320FA82
:100C000002F018BF40F001004FEAC1234FEAD3239E
:100C100003FA0CFC40EA0C0023FA02F34FEA430308
:100C2000CCE77FEA625307D150EA01331EBF4FF091
:100C3000FE4040F44000704701F0004040F0FE40AC
:100C400040F40000704700BF80F0004002E000BFA9
:100C500081F0004142001FBF5FEA410392EA030FA7
:100C60007FEA226C7FEA236C6AD04FEA1262D2EBF1
:100C70001363C1BFD218414048404140B8BF5B42F6
:100C8000192B88BF704710F0004F40F4000020F08F
:100C90007F4018BF404211F0004F41F4000121F0A5
:100CA0007F4118BF494292EA030F3FD0A2F10102EF
:100CB00041FA03FC10EB0C00C3F1200301FA03F12D
:100CC00000F0004302D5494260EB4000B0F5000F50
:100CD00013D3B0F1807F06D340084FEA310102F10F
:100CE0000102FE2A51D2B1F1004F40EBC25008BFC1
:100CF00020F0010040EA03007047490040EB00008B
:100D0000013A28BFB0F5000FEDD2B0FA80FCACF18B
:100D1000080CB2EB0C0200FA0CF0AABF00EBC250B8
:100D200052421843BCBFD0401843704792F0000FA6
:100D300081F4000106BF80F400000132013BB5E7F9
:100D40004FEA41037FEA226C18BF7FEA236C21D06F
:100D500092EA030F04D092F0000F08BF08467047D4
:100D600090EA010F1CBF0020704712F07F4F04D1A2
:100D7000400028BF40F00040704712F100723CBFB5
:100D800000F50000704700F0004343F0FE4040F4DF
:100D9000000070477FEA226216BF08467FEA23639D
:100DA0000146420206BF5FEA412390EA010F40F488
:100DB000800070474FF0000304E000BF10F00043D4
:100DC00048BF40425FEA000C08BF704743F09643BB
:100DD00001464FF000001CE050EA010208BF7047D6
:100DE0004FF000030AE000BF50EA010208BF70475D
:100DF00011F0004302D5404261EB41015FEA010C72
:100E000002BF84460146002043F0B64308BFA3F169
:100E10008053A3F50003BCFA8CF2083AA3EBC2534B
:100E200010DB01FA02FC634400FA02FCC2F120026A
:100E3000BCF1004F20FA02F243EB020008BF20F0A1
:100E40000100704702F1200201FA02FCC2F1200207
:100E500050EA4C0021FA02F243EB020008BF20EAFC
:100E6000DC7070477BB972B90029BEBF00204FF01B
:100E7000004106E008BF00281CBF6FF000414FF0A2
:100E8000FF3000F007BAADF1080C6DE904CE00297F
:100E900009DB002B1ADB00F095F8DDF804E0DDE952
:100EA000022304B07047404261EB4101002B1BDB81
:100EB00000F088F8DDF804E0DDE9022304B04042E8
:100EC00061EB4101524263EB43037047524263EBD3
:100ED000430300F077F8DDF804E0DDE9022304B015
:100EE000404261EB41017047524263EB430300F023
:100EF00069F8DDF804E0DDE9022304B0524263EB57
:100F00004303704753B94AB9002908BF00281CBFE2
:100F10004FF0FF314FF0FF3000F0BCB9ADF1080CDD
:100F20006DE904CE00F04EF8DDF804E0DDE90223BF
:100F300004B07047430803F05533C01A830803F028
:100F4000333300F03330184400EB101000F00F3052
:100F500000EB002000EB0040000E704707EE900A07
:100F6000F5EEC07AF1EE10FA01D400F00BB8F1EE14
:100F7000677A08B517EE900A00F004F8404261EB7A
:100F8000410108BDD0B5FFF7BFFA0C4B0022064661
:100F90000F46FFF711FBFFF7E7FD0446FFF792FA54
:100FA000074B0022FFF708FB02460B463046394646
:100FB000FFF74AF9FFF7D8FD2146D0BD0000F03D0C
:100FC0000000F0412DE9F047089D04468E46002BB5
:100FD0004DD18A42944669D9B2FA82F252B101FAED
:100FE00002F3C2F1200120FA01F10CFA02FC41EAFD
:100FF000030E94404FEA1C48210CBEFBF8F61FFA82
:101000008CF708FB16E341EA034306FB07F199421C
:101010000AD91CEB030306F1FF3080F01F819942CF
:1010200040F21C81023E63445B1AA4B2B3FBF8F0A9
:1010300008FB103344EA034400FB07F7A7420AD930
:101040001CEB040400F1FF3380F00A81A74240F258
:1010500007816444023840EA0640E41B00261DB1C3
:10106000D4400023C5E900433146BDE8F0878B42F8
:1010700009D9002D00F0EF800026C5E900013046B7
:101080003146BDE8F087B3FA83F6002E4AD18B4291
:1010900002D3824200F2F980841A61EB030301203B
:1010A0009E46002DE0D0C5E9004EDDE702B9FFDE27
:1010B000B2FA82F2002A40F09280A1EB0C014FEAD2
:1010C0001C471FFA8CFE0126200CB1FBF7F307FB2F
:1010D000131140EA01410EFB03F0884208D91CEBD2
:1010E000010103F1FF3802D2884200F2CB8043466F
:1010F000091AA4B2B1FBF7F007FB101144EA01444E
:101100000EFB00FEA64508D91CEB040400F1FF31DC
:1011100002D2A64500F2BB800846A4EB0E0440EACA
:1011200003409CE7C6F12007B34022FA07FC4CEAD3
:10113000030C20FA07F401FA06F31C43F9404FEAC6
:101140001C4900FA06F3B1FBF9F8200C1FFA8CFEDB
:1011500009FB181140EA014108FB0EF0884202FA2F
:1011600006F20BD91CEB010108F1FF3A80F08880F0
:10117000884240F28580A8F102086144091AA4B2AD
:10118000B1FBF9F009FB101144EA014100FB0EFE2E
:101190008E4508D91CEB010100F1FF346CD28E455D
:1011A0006AD90238614440EA0840A0FB0294A1EBEE
:1011B0000E01A142C846A64656D353D05DB1B3EB4B
:1011C000080261EB0E0101FA07F722FA06F3F1407B
:1011D0001F43C5E9007100263146BDE8F087C2F122
:1011E0002003D8400CFA02FC21FA03F3914001439A
:1011F0004FEA1C471FFA8CFEB3FBF7F007FB1036D3
:101200000B0C43EA064300FB0EF69E4204FA02F47E
:1012100008D91CEB030300F1FF382FD29E422DD9D1
:10122000023863449B1B89B2B3FBF7F607FB163306
:1012300041EA034106FB0EF38B4208D91CEB010186
:1012400006F1FF3816D28B4214D9023E6144C91A06
:1012500046EA004638E72E46284605E70646E3E616
:101260001846F8E64B45A9D2B9EB020864EB0C0E20
:101270000138A3E74646EAE7204694E74046D1E72F
:10128000D0467BE7023B614432E7304609E76444DD
:10129000023842E7704700BF02E000F000F8FEE7C6
:1012A00072B6374880F30888364880F30988364894
:1012B0003649086040F20000CCF200004EF634716E
:1012C000CEF200010860BFF34F8FBFF36F8F40F283
:1012D0000000C0F2F0004EF68851CEF20001086026
:1012E000BFF34F8FBFF36F8F4FF00000E1EE100A96
:1012F0004EF63C71CEF200010860062080F314889F
:10130000BFF36F8F88F0BAF987F022FA4FF05530AB
:101310001F491B4A91423CBF41F8040BFAE71D49A3
:10132000184A91423CBF41F8040BFAE71A491B4A9C
:101330001B4B9A423EBF51F8040B42F8040BF8E7EE
:1013400000201849184A91423CBF41F8040BFAE7C3
:1013500088F098F987F050FA144C154DAC4203DA36
:1013600054F8041B8847F9E701F0F2F8114C124DCC
:10137000AC4203DA54F8041B8847F9E788F080B9D7
:1013800000060020002200200000010808ED00E017
:101390000000002000060020C8BD0B08002200202D
:1013A000A8250020A825002018350120E00101080B
:1013B0003802010838020108380201082DE9F04F0F
:1013C0002DED108AC1F80CD0C3689D46BDEC108A83
:1013D000BDE8F08F002383F311882846A047002042
:1013E00086F03CFFFEE786F099FD00DFFEE7000097
:1013F00001F0FF01102A2BDB10F0070F08D010F8C6
:10140000013B013A8B422DD010F0070F42B3F6D1C9
:10141000F0B441EA012141EA014122F007047FF0E2
:1014200000070023F0E80256083C85EA010586EA39
:10143000010685FA47F5A3FA87F586FA47F6A5FA75
:1014400087F68EB9EED1F0BC01F0FF0102F0070281
:1014500032B110F8013B013A83EA010313B1F8D12C
:101460000020704701387047002D06BF354603380D
:10147000073815F0010F07D1013015F4807F02BF46
:10148000013015F4C03F0130F0BC0138704700BF97
:1014900010F8012B11F8013B012A28BF9A42F7D01E
:1014A000D01A7047034613F8012B002AFBD1181AF3
:1014B0000138704738B50022002304460D46FFF777
:1014C000EDFA28B920462946BDE8384000F00AB8B0
:1014D000204605F1004100F005F8404261EB410172
:1014E00038BD00BFD0B50C4B002206460F46FFF7B3
:1014F00063F8FFF739FB0446FEF7E4FF074B0022D1
:10150000FFF75AF802460B4630463946FEF79CFE76
:10151000FFF72AFB2146D0BD0000F03D0000F0415E
:10152000036800221B6818470120704737B50191F6
:10153000202104465DF08CFCD0B10E4B93F9B21221
:10154000A1B1B3F9B412D3F8843A019AB3F90A50AD
:1015500001F10A039D4203DD40F28D33994205DC1F
:101560002046054B20215DF07BFC002003B030BD00
:101570000120FBE7B0450020C8180A0807B5044859
:101580005EF0DEFE00F0010003B05DF804FB00BF7A
:101590004C5900202DE9F0438FB00E46054605F06A
:1015A00061FD002780462E22394602A801978BF064
:1015B000ABFF322301AA3946404605F09DF80446A8
:1015C00048B9184A01AB314628465DF051FE204625
:1015D0000FB0BDE8F083DFF85890D9F8B008036881
:1015E0009B6898470028F2D0A9F5405003F038FDD9
:1015F000814630B90C4A314628465DF039FE4C46EA
:10160000E5E76946404604F0CDFE0028DFD09DF8AE
:1016100001305B06DBD5054A314628465DF028FEE1
:101620003C46D4E7DC180A08E5180A08FC180A0842
:10163000B055002008B5064B93F8193D9B0704D51B
:10164000044A5DF015FE002008BD0120FCE700BF44
:10165000B04500200C190A0870B50C4C0546D4F8AA
:10166000B0080368DB680E46984710B10124204695
:1016700070BDA4F5405003F011FD04460028F5D1DB
:10168000034A314628465DF0F3FDF0E7B0550020EF
:101690001C190A082DE97043264BD3F81C3D1D7B0D
:1016A000804689465DB9244B1B68986A03685B6B6A
:1016B000984738B9214A494640465DF0D9FD284649
:1016C000BDE8708348F0B2F8202149F029F838B11C
:1016D00048F0ACF81F2149F023F808B1184AEAE7AE
:1016E000D8F808303BB9D8F80030494640465B6B23
:1016F000BDE87043184749464046FFF717FF494683
:10170000064640465EF04AFA2021064040465DF01B
:101710009FFB49464046FFF78DFFF5B2054049461D
:101720004046FFF799FF4946054040465EF00CFCF5
:101730000540C4E7B0450020685F002030190A0862
:1017400047190A0808B5FFF7A5FF054A92F8081DD2
:1017500060F3410182F8081D024A907108BD00BF84
:10176000B0450020F55F0020F7B505460F465DF057
:10177000ABFB044678B1022128465DF069FB0646C2
:1017800048B114485EF0DCFDC205C0F30723C0F386
:10179000002403D53446204603B0F0BD9B07F9D59D
:1017A0000C485EF0D7FD0C4BD3EDA97AF8EEE77A42
:1017B00030EE670ADFED097AB0EEC00AB4EEE70A50
:1017C000F1EE10FAE6DD064B3A46022128465DF0BE
:1017D00047FBE0E74C590020B05500200000C8420C
:1017E00064190A08F8B504460F465DF0D3FD1021D0
:1017F000054620465DF02CFB58B12046FFF7BEFEA3
:10180000064630B9044B3A46102120465DF028FBCD
:1018100035462846F8BD00BF78190A0870B5054658
:101820000E465DF0BDFA044678B1802128465DF091
:101830000FFB50B1094B93F8A13243B1084B32462C
:10184000802128465DF00CFB0024204670BD314607
:101850002846BDE870405DF065BF00BFB055002070
:101860008C190A082DE9F04180460E46FFF792FEDA
:101870001A4F044610B90024FC710AE0184D05F512
:101880004053D3F8B00803689B68984720B90123F8
:10189000FB712046BDE8F081082140465DF0D8FA92
:1018A0000028F4D095F81434B02202FB035305F558
:1018B0000055B3F81E22B5F9B0329A4206DD094B45
:1018C0003246082140465DF0CBFAD4E73146404627
:1018D0005DF0F2FB0028DAD1CDE700BFF55F002014
:1018E000B0250020A0190A085EF01CB870B50546A6
:1018F0000E46FFF74FFE084B0446D8713146284686
:10190000FFF7AAFE31460028284608BF00245EF0F3
:10191000CBF9204070BD00BFF55F00202DE9F843F2
:10192000414F3B788146002B7BD1404CD4F81C5D65
:101930002D7B01263E701DB13B702846BDE8F88323
:101940005EF0BCFB054630B9394A3870137843F075
:1019500001031370F1E7DFF8F4803CF013F831462F
:101960003AF0FCFF88F804600B2634F05BFA013E85
:1019700034F00EFA16F0FF06F7D12E4948465EF015
:10198000B7FA05F06FFBD0F80022C4F82C2D90F8C0
:101990007C32DA0733D404F015FF3BF0F3FF3C212F
:1019A0003BF088FD04F6145300221A60224B1B689A
:1019B000D86A036801211B689847D4F81C2D137B53
:1019C0001BB90123137388F804303BF0DBFF94F854
:1019D0000D2D94F80C1D3BF09DF938F0B7FF38F051
:1019E000F7FA00233B7060F065F9144BC3F8A008C8
:1019F00094F8093D43F0200384F8093D9DE79B07D7
:101A0000D4D431460E4802F089F90E485EF0A2FCAB
:101A1000DFED0D7A20EE270A04F6145383ED000A59
:101A2000C4E7002589E700BFA8250020B0450020B5
:101A300014600020B0190A08685F0020B05500202B
:101A4000B02500204C5900200AD7233CF55F002028
:101A50002DE9F0432B4DD5F81C3D1B7B87B0064686
:101A6000002B4CD05EF0E0FB0446002843D0264912
:101A700030465EF03DFA05F0F5FA074609F036FF0C
:101A80008046384604F05AF9D8B198F92430022B30
:101A900017D100264FF00009F1B203AA3846019190
:101AA000CDF80C90CDF81090CDF8149004F0C0FC57
:101AB000019918B103AA404609F024FC0136032E0F
:101AC000EAD1D5F81C2D137B1BB1002313730F4AE9
:101AD00013713BF057FF00213AF040FF0C4B1B689D
:101AE000D86A036800211B68984795F8093D6FF391
:101AF000451385F8093D204607B0BDE8F083012471
:101B0000F9E700BFB0450020C0190A08F55F0020C2
:101B1000685F002008B500F5005090F8083DC3F359
:101B200080028A420BD061F3820380F8083D31B114
:101B30003BF028FFBDE808400F213BF0BBBC08BDCF
:101B400010B500F500520C4692F8193D03F0010162
:101B5000A14209D064F3000382F8193DDB0704D4E5
:101B600002F028FB024B9C7210BD02F0D7FBF9E794
:101B7000F55F002000F5005090F8193D61F3410336
:101B800080F8193D014B1973704700BFF55F0020C5
:101B900000207047002070470020704700207047E9
:101BA00000207047002070470020704700207047D9
:101BB00000207047002070470020704770470000E9
:101BC00000F50B50704700000048704768460A084F
:101BD00000F5005090F80C0D7047000003480860B5
:101BE0001D21117008221A60704700BF9C1C0A0852
:101BF00038F0F6BD18F0F4B83BF032B847F062BAEE
:101C000045F098BB02F0F6BA02F028BA02F050B9DB
:101C100034F0BEB84CF0CAB903F00AB847F054BD6E
:101C200012F08ABB02F068B802F028BD02F0DEB9FB
:101C300002F07CBC02F0E6BF18F0F0BB03F046BA3D
:101C400002F00EBB02F0C6BB70B51F4B036000F57F
:101C500000530446D3F89C0C1C4AC3F8E02A08B190
:101C600009F0D8F81A4B236004F5805393F8142F29
:101C700042B9D3F8105F2DB1284616F0F1FE284680
:101C800009F0C4F804F58A501C305CF03DFB04F503
:101C9000895049F0DDFB04F6F44504F69446B5425C
:101CA00004D0183D284616F04BFBF8E7094BC4F862
:101CB000C83804F6C4103DF0FDFF04F513603DF094
:101CC000F9FF204670BD00BFEC1E0A0854FB0A084D
:101CD00028D90A08DCAE0A0838B54C4B044640F84F
:101CE000043B4AF0E9FC04F1100008F07BFC04F12D
:101CF000680038F003FB04F5907010F07FFF04F5E6
:101D00008C6007F0DBF904F2845009F085F804F6E2
:101D1000C80017F009FF04F547604AF055FC04F5C8
:101D2000546037F09FFF04F57F603AF067FD04F5DB
:101D30008850043050F0C8F904F5895049F070FB20
:101D400004F58A501C305CF0CBFA04F58B50183047
:101D500038F096FE04F58E500C304BF08BFE04F5F7
:101D6000805300252A4A83F8F05104F58F5310332D
:101D700004F59050136033F07FFE04F5925029462D
:101D8000103003F0D7FC04F5C55056F0D7FB04F52E
:101D9000ED50043059F0DCFA04F5F5501C305BF0DE
:101DA000F9FB04F5F9505CF02FF804F5FB501830FE
:101DB00003F020FB04F50350183057F0B3F804F596
:101DC00004501449303037F041F804F5055008301C
:101DD00050F01EFC04F5085004305CF01DFE04F5C4
:101DE000005304F5095083F85C520B4D34305CF01D
:101DF00035FF2B6813B109485FF02AFF20460849D8
:101E000037F024F82C60204638BD00BF28D90A08D6
:101E10007C69002090660B08CC600020141A0A0828
:101E200040D80A0810B503F041F847F0FFFC0368FA
:101E3000BDE810405B681847FFF7F4BF38B500F500
:101E4000345530350446284608F0A6FA09F04EFD10
:101E500090F92130D3B190F84033BBB1284600212E
:101E600008F02EF8DFED0A7A04F2DC7393ED287A9D
:101E700020EE270ADFED077AA7EE270A04F2845046
:101E800083ED280ABDE8384009F040BC38BD00BFEA
:101E9000CDCCCC3D6666663FFFF7D0BF10B50121C3
:101EA000044603F037F910B1204601F0C1F84FF4B1
:101EB0008051204603F02EF920B12046BDE81040A5
:101EC00001F078B810BD0000FFF7E8BF13B502219C
:101ED000044603F01FF938B10121204603F01AF936
:101EE00010B9204601F0A4F80221204603F012F9AF
:101EF00050B3204601F0AAF84021204603F00AF929
:101F000060B104F57F6001903AF076F804F58053F3
:101F1000019893F920310BB13AF0B0F94FF4806198
:101F2000204603F0F7F818B104F57F603AF0FEF8A8
:101F30008021204603F0EEF868B119F0B1FA02B042
:101F4000BDE8104017F036BC0121204603F0E2F84E
:101F50000028CED1D0E74FF48021204603F0DAF8F4
:101F60000028EAD14FF40021204603F0D3F80028DE
:101F7000E3D102B010BD0000FFF7A8BF10B50121EA
:101F8000044603F0C7F810B1204601F05FF8802145
:101F9000204603F0BFF828B119F082FABDE81040DE
:101FA00017F0E4BB10BD0000FFF7E8BF38B54FF6EF
:101FB000FF71044603F0AEF804F5005528B1D5F8DA
:101FC000082D0721204601F049F849F087F848F02C
:101FD0002BFE95F8083D074A83F01003C3F3001366
:101FE000537138F0B3FC38F01BF9BDE838400248B3
:101FF00055F082BDF55F0020685D0020FFF7D6BF79
:10200000F0B52DED028B00F5925410349FB00546CB
:102010000121204604F0ACFF05F54B510431204668
:1020200004F032FE05F54B511C31204603F028FF29
:1020300005F5AC5104F5457008311CF0C9F805F5FB
:10204000405405F54B50D4F8C422D4F8C83284ED7E
:10205000BA0A1CA930301C921D933EF071FD05F5A3
:102060004B5105F54C500C313430B0EE608AF0EE37
:10207000408A3EF0E7FB05F54B5105F54D50283100
:10208000C4EDB48A84EDB58A84EDB60A28303EF0FA
:10209000D9FB84EDBB0A3BF075FC05465FF012FEF0
:1020A0002A4B074618680E46FEF72EFACDE91801AE
:1020B000D4F8E402FEF728FACDE91601D4F8E002DC
:1020C000FEF722FACDE91401D4F8DC02FEF71CFA7F
:1020D000CDE91201D4F8EC02FEF716FACDE91001B1
:1020E000D4F8E802FEF710FACDE90E01D4F8D802D0
:1020F000FEF70AFACDE90C01D4F8CC02FEF704FA97
:10210000CDE90A01D4F8D402FEF7FEF9CDE90801C1
:10211000D4F8C802FEF7F8F9CDE90601D4F8D002E8
:10212000FEF7F2F9CDE90401D4F8C402FEF7ECF9A8
:10213000CDE90076CDE90201054B064A064928465D
:102140003BF04CF81FB0BDEC028BF0BD0C3A002008
:10215000281A0A08361A0A08631A0A08FFF750BF35
:1021600010B5044602F014FF1021204602F0D2FF01
:1021700028B119F095F9BDE8104017F0E9BB10BD82
:10218000FFF7EEBF00F5A553D3ED005AD3ED036A78
:10219000D1ED017A91ED006A26EEE77A67EEA57A35
:1021A000A6EE257AE6EE267A81ED007AC1ED017A77
:1021B0007047000000F5A553D3ED005AD3ED036A34
:1021C000D1ED017A91ED006A27EEA67A67EEA57A45
:1021D000A6EE257AE6EE667A81ED007AC1ED017A07
:1021E000704700002DE9F0432DED028B044687B0C7
:1021F000FFF772FDBE4B236004F50B50343001F045
:1022000011FC04F5005504F50A53383304F52A5639
:102210001436C5F88C3A062385F8903A30465CF0BF
:10222000CBFD0DF11008B34BC5F8943A301D0123D6
:10223000414604F52B578DF81030203737F0DEFB80
:10224000AD4BC5F8E03A07F114005EF0E7FB04F58A
:102250002C5604F52D59183609F13C093046143630
:1022600043F02CF94E45F9D10723C5F8A03C0023D3
:10227000A5F8A43C4FF4CB7008F0C6FDC5F89C0C43
:1022800004F5325028305EF0C9FB04F533502C3091
:102290005EF0C4FB994B1A6802B91F60984BC5F8F1
:1022A000E03A04F534500123A5F80C3D0E305DF002
:1022B000DBFF944B0593944B0494009304F5345046
:1022C00098E80C004FF40071303007F0A1FC04F5E1
:1022D0004A5003A9F7EE008A2830CDED038A3EF07C
:1022E0006DF804F54A50343008F08EFA9FED878A75
:1022F0009FED872A04F5405504F592531033B0EE54
:10230000083A04F54E50C5F8B433F0EE432AF0EE27
:10231000420AB0EE430AF0EE481AB0EE481A85EDD4
:10232000B18A85EDB28A85EDB38A85EDB48A85EDF3
:10233000B58A85EDB68A85EDB78A85EDB88A85EDD3
:10234000B98A85EDC58A85EDC68A85EDC78A85ED92
:10235000C88A85EDC98A85EDCA8A85EDCB8A85ED67
:10236000CC8A85EDE78A85EDE88A85EDE98A85EDF9
:10237000EA8A85EDEB8A85EDEC8A383055F05AFD16
:10238000B0EE083A04F55450F0EE432AB0EE682A55
:10239000F0EE481AB0EE481AF7EE080AB1EE0C0A51
:1023A000043055F02BFFB0EE083A04F55550F0EE2E
:1023B000432AB0EE430A9FED562ADFED560AF0EEAF
:1023C000481AB0EE481A3C3055F018FFB0EE083A03
:1023D00004F55750F0EE432A9FED4F2ADFED4F0AE8
:1023E000F0EE481AB0EE481AB0EE680A343055F0F4
:1023F00021FDB0EE083AF0EE432A9FED490AB0EE17
:10240000482AF0EE481AB0EE481AF0EE480A04F5F1
:102410005D5055F0F3FEF0EE083A04F55E509FED86
:10242000410AB0EE485AF0EE684AB0EE484AB0EEC3
:10243000633AF0EE632AB0EE002AF0EE481AB0EEEE
:10244000481AF6EE000A383055F006FB3649374890
:102450000860002304F5625285F8A5382C32142751
:102460009EB207FB06010133097C0029F8D1304BED
:102470001E80304B196811B12F485FF0E9FB04F55D
:1024800062503430C5F8B0081A6002F0B1F82B4B36
:10249000C5F8B43804F56350243002F0A9F8284B8D
:1024A000C5F8E43804F56450143002F0A1F8254B67
:1024B000C5F8143904F56550043002F099F8224B40
:1024C000C5F8443904F5665005F6741383ED008AA7
:1024D00083ED018A83ED028A043002F089F81B4BF8
:1024E000C5F88439204607B0BDEC028BBDE8F08307
:1024F000EC1E0A08DC190A0854FB0A0810640020C4
:10250000A41F0A08451C0108E01E0A08000000007C
:10251000CDCC4C3ECDCCCC3ECDCCCC3DCDCC4C3D31
:102520003333333F9A99993F906000204C580A0802
:102530008E6000204C600020681A0A08E0610A08DA
:1025400028610A088C620A0884610A082C620A0859
:1025500038B5054B1C6823680A461D68034B0146C5
:102560002046A847002038BD685F0020B025002025
:1025700010B55EF09DFE064C064B18602046FFF736
:1025800031FE2046044A0549BDE8104088F08EBA65
:10259000B0250020685F0020F8C10020491C010818
:1025A00010B504460180024936F050FC204610BDAB
:1025B0006C1F0A0810B500234FF07C52274C0365AE
:1025C0004FF07E51C0F88030C0F89030C0F8A03095
:1025D000C0F8C0304365C0F88430C0F89430C0F80B
:1025E000A430C0F8C43083668367C0F89830C0F860
:1025F000A830C0F8B830C366C367C0F89C30C0F8D4
:10260000AC30C0F8BC304FF03F430267C0F8B02098
:102610004267C0F8B420C0F88820C0F8C820C0F8CD
:102620008C20016644668465C165C0F8CC304FF4E7
:102630007A71212048F080FA4FF47A71222048F014
:102640007BFA4FF47A71232048F076FABDE8104007
:102650004FF47A71242048F06FBA00BF000080BFA9
:10266000F8B52DED068B037B044643B90023C0F873
:10267000D430C0F8D830C0F8E030C0F8DC30D4ED49
:10268000371A94ED381AD4ED360A94ED350A854898
:10269000DFED858A00F022FC5820B7EE001AFFEE2D
:1026A000000A94ED350A19F0D3FB592084ED350A60
:1026B000B7EE001AFFEE000A94ED360A19F0C8FBD7
:1026C0005A2084ED360AB7EE001AFFEE000A94EDA8
:1026D000380A19F0BDFB5B2084ED380AB7EE001A0A
:1026E000FFEE000A94ED370A19F0B2FB84ED370AC9
:1026F0005FF0D4FA07EE900A9FED6C7AF8EE677AF5
:1027000004F1100567EE877A2126C4ED027A2F4680
:10271000F7EE009A94ED35AAD5ED100AB0EE680AEE
:102720006AEE200A88F06EFB94ED368AD5ED140A25
:10273000B0EE409A68EE200AB0EE680A88F062FBBC
:10274000D4ED385AD5ED186A94ED376A95ED1C7AB8
:1027500065EEA66A79EE007AF0EEE66A26EE077A72
:1027600077EEA67AB0EEC77A77EE877AB5EEC09AA2
:10277000E5EC017A95ED235AC5ED079A28EE058A16
:1027800095ED1F5AAAEE058A95ED275AA5EE858A82
:10279000D5ED2B5AA6EE258AF1EE10FACCBF012317
:1027A0000023B5EEC00A85ED038AF1EE10FA84F835
:1027B000D030C8BF94F8D030F5EEC06AC4BF013342
:1027C00084F8D030F1EE10FAC8BF94F8D030B5EEEE
:1027D000C07AC4BF013384F8D030F1EE10FAC2BF22
:1027E00094F8D030013384F8D03094F9D030002BF5
:1027F000C1BF07EE103AB8EEC77AC8EE076AC5ED5A
:10280000036A95ED038AB0EEC87A77EE877AF4EE24
:10281000E97AF1EE10FAC4BF79EEC77A45ED017A94
:1028200094F9E83015ED019A83B1DFED217AB4EE29
:10283000E79AF1EE10FA09D8DFED1E7AB4EEE77AE6
:10284000F1EE10FAA4BF4FF08043EB6194ED390A2A
:10285000D5ED077A20EE270AD4ED027A20EE270A7A
:10286000DFED157A30EE000A20EE270A88F044FAF0
:10287000A9EE008A30B201369FED100A85ED0B8A71
:1028800028EE000AB6B248F033F9252E7FF442AFA5
:10289000BDEC068B04F1200239460248BDE8F84041
:1028A00000F04EBBB025002000000000BD3786358B
:1028B0009A99193FCDCCCC3EDB0F494000007A44B9
:1028C0000022C0F8D420C0F8D820C0F8E020C0F81A
:1028D000DC20FFF7C5BE00000020704700207047D5
:1028E0000120704790F89C308B4286BF283150F809
:1028F000210000207047000090F89C308B4286BF7A
:10290000283150F82100002070470000FA2070475D
:10291000014B93F8A2027047B0450020D0E90B327A
:1029200042F4E0520263426B43F4F84342F4E05253
:102930004263C36270470000014802F005BC00BF5B
:10294000B025002013B54FF44470CDE9002108F004
:1029500055FA044628B1DDE9002145F091FC024B0F
:102960002360204602B010BD8C210A087047000089
:10297000704700000020704770470000002070473B
:102980007047000070470000032070470820704720
:10299000064BD3F81C3D3BB11B7B002B0CBF5020DA
:1029A000D02040F0010070475020FAE7B0450020E9
:1029B00070470000014B93F8A4027047B045002017
:1029C000034B93F9F802003818BF0120704700BF8D
:1029D000B0450020014B93F9A6027047B045002096
:1029E0007047000010B52DED028B174BD3F81C4D2E
:1029F0003CB3D4ED360A94ED380AF0EEE00AB0EEBE
:102A0000C00A88F0FFF9D4ED370AB0EE408A94EDA1
:102A1000350AF0EEE00AB0EEC00A88F0F3F9F0EE05
:102A2000400AB0EE480A88F0EDF9DFED087A20EEB2
:102A3000270ABDEEC00A10EE103A18B2BDEC028BA8
:102A400010BD2046FAE700BFB04500200000C84294
:102A500044F010BB10B5044641F050FE054802F0AA
:102A600073FB054A034606212046BDE8104041F0AD
:102A70002DBE00BFB0250020DC1F0A0840F01CBF9F
:102A800008B5084607F0C8FF00280CBF0420002046
:102A900008BD0000162A01D040F04EBC03220A7087
:102AA0000120704710B44B7A8C7ACA7A43EA042327
:102AB00043EA0243863B012B03D95DF8044B45F002
:102AC000BDB95DF8044B704708B540F091FE40F485
:102AD0001C6040F00D0008BD10B5044608F096F9E2
:102AE000204610BD08B5094B93F8082DD2060BD42B
:102AF00003F58053D3F8B00803689B6A9847002811
:102B00000CBF0220042008BD0120FCE7B0450020D6
:102B1000044B187820B9044B93F8090DC0F38010CA
:102B2000704700BFC45F0020B04500201FB50023E0
:102B300001930293039304F095FA01A904F080F83D
:102B400028B101A81BF0C6FE05B05DF804FB11F02A
:102B500031FC90F8F432B02202FB030090ED3B0A06
:102B6000F2E700000C4B93F8A1228AB9A3F5805339
:102B700093F8192D51070BD193F8082DD20609D4DB
:102B800093F8093D13F0020F14BF04200120704791
:102B90000520704703207047B05500202DE9F04F05
:102BA000354F97F80C3D012B8DB0044652D9334E6A
:102BB000DFF8E8A0082516F9018BB7F9CC3208F147
:102BC000FF3B43FA0BF3D90740D5207C3FF07EFA58
:102BD0008146207C40F07EF900F12103994505D221
:102BE000207C0DB0BDE8F04F3EF0ECBCBBF1070F10
:102BF0002CD8DFE80BF03E04323436383A3C204B18
:102C0000186959695A6AD3F804B0D3F818E0D3F8B0
:102C10000CC0D3ED007A1B6ACDF82520CDF8293001
:102C200062222123CDE9003207900891207CCDED6E
:102C3000037A192303AAC221CDF810B0CDF814E00D
:102C4000CDF818C08DF824803FF0AAFA013D15F0A8
:102C5000FF05B0D10DB0BDE8F08F0A4BD0E70A4BAD
:102C6000CEE70A4BCCE70A4BCAE75346C8E7094B05
:102C7000C6E7094BC4E700BFB045002060220A0840
:102C8000D4590020E45A00205C5B0020E45B002063
:102C9000105C0020FC5D0020A8590020205D002071
:102CA000084BD3F8FC22920701D440F039BB03F55E
:102CB000805393EDAE0ADFED047AB8EEC00A20EE41
:102CC000270A7047B04500200AD7233C10B594B0BE
:102CD000044603A807F098FD1A4BD3F8B008036820
:102CE00003A91B6B984750B3247C5EF0E3FF059B60
:102CF000DDED047A0893069B09930023F8EEE77A4A
:102D00009FED117A0B930C930D930E930F931093E9
:102D1000119312934FF6F853ADF84C3000239622DE
:102D200067EE877A8DF84E303323CDE90032079075
:102D300007AA57212046CDED0A7A3FF031FA14B0A8
:102D400010BD00BFB05500200AD7233C014802F057
:102D5000F9B900BFB0250020014B93F80C0D704766
:102D6000B0450020024B93F8090DC0F340007047B6
:102D7000B045002030B52DED028B154B91ED018A49
:102D80000546D3F8B008036885B0DB690C46984760
:102D900028B9BDEEC88A18EE103ADB0712D5D4E97F
:102DA000040119F05BFA68B1684607F02DFD6A4628
:102DB0002146284644F0B6FB20B10649684607F094
:102DC00037FE00B1022005B0BDEC028B30BD00BF64
:102DD000B0550020645800208B8B162B05D0C02BDB
:102DE00001D1FFF7C7BF45F04FBE0020704700007C
:102DF00030B52DED028B8DB000230546039304936F
:102E0000059304F02FF903A903F01AFF58B304F057
:102E100029F900F55A7393E8070006AC84E8070027
:102E2000DDED060A9DED070A2D7CF1EE600AB1EE9C
:102E3000400A88F083F92046B0EE408A1BF04AFD34
:102E4000DFED0B7A089B0B93012228EE278A0C23D7
:102E5000CDE90032A82109AA28468DED098A8DED19
:102E60000A0A3FF09DF90DB0BDEC028B30BD00BFEA
:102E7000E02E6542242938B505460FD003D81B291A
:102E800007D1012412E04029FBD0A1F14203012B1C
:102E9000F7D92846BDE8384044F002BD0C213EF089
:102EA000A3FB044610B12846FFF7A2FF204638BD19
:102EB00008B591ED007AF6EE007AB4EEE77AF1EE1D
:102EC00010FA06DD044801220521FEF7C1FD0020AD
:102ED00008BD0420FCE700BF445000202DE9F0416C
:102EE00088B080461B22002101A810EE107A10EE57
:102EF000906A11EE105A11EE904A8AF005FBA32356
:102F00008DF8043095238DF805300B238DF80630AD
:102F10005EF0D8FE1B22CDF80700CDF80B1008F5A7
:102F20007F6001A9CDF80F70CDF81360CDF8175070
:102F3000CDF81B4039F02EFD08B0BDE8F08100004F
:102F400070B58CB00D46144606462B22002101A810
:102F50008AF0DAFAA3238DF8043095238DF8053032
:102F60000C238DF806305EF0ADFE2B68CDF80F30E7
:102F70002368CDF813306B68CDF817306368CDF84F
:102F80001B30AB68CDF81F30A368CDF82330EB6859
:102F9000CDF80700CDF80B10CDF827302B22E368D1
:102FA000CDF82B3001A906F57F6039F0F3FC0CB0A9
:102FB00070BD000070B500F57F6500F54E56044603
:102FC00006F1780228460E2139F0A8FB06F1A4028A
:102FD00028460F2139F0A2FB04F55452284634321A
:102FE000102139F09BFB04F55652284604F557563C
:102FF0002C32112139F092FB06F1740228466E2121
:1030000039F08CFB06F1A00228466F2139F086FBCF
:1030100004F55D52284630320D2139F07FFB04F56E
:10302000615228460C32BDE870406B2139F076BB06
:103030001FB500F59250002301A9103001930293AF
:10304000039302F081FA05B05DF804FB08B504F0C3
:1030500009F8BDE8084003F0A5BD00007FB50E46A5
:103060004FF6FF710446154602F054F8E0B1102205
:10307000002168468AF048FAA3238DF80030952392
:103080008DF8013004238DF802305EF01BFE102213
:10309000CDF80300CDF8071004F57F6069468DF880
:1030A0000B60039539F0F6FC04B070BDA3207047A7
:1030B00038B5044600F57F6502F046F80C49024633
:1030C000284639F003FE04F50053284693F80D2DE9
:1030D00093F80C1D39F01EFE04F59250103004F0E8
:1030E000D1F904F59070BDE8384010F0CDB900BFBB
:1030F000DC1F0A0837B5069D044600B92C7801B9D3
:10310000697802B9AA7803B9EB78002064F3070064
:1031100061F30F2062F3174063F31F6003B030BD0B
:103120002DE9F04F2DED0C8B9DB0E14C0D93D4EDBE
:10313000379ADFEDE05A90ED006A04F50054F7EE9F
:10314000006AD4F81C3DD3ED367A93ED387AF0EE70
:10315000E77AB0EEC77A77EE877A9246F4EEE67AAF
:10316000F1EE10FAC8BF86EEA78A06460F46DFEDDD
:10317000D27AD8BFB0EE668A28EE277AA6EE257AF4
:1031800080ED007AD4F81C3D93ED357A93ED376AE3
:10319000B0EEC77AB0EEC66A37EE067AB4EEE67ADB
:1031A000F1EE10FACCBFC6EE878AF7EE008A90EDFA
:1031B000017A68EEA77AE7EE257AC0ED017A3AF057
:1031C000E1FB05465EF07EFD814618EE900A8846DA
:1031D000FDF79AF9CDE9080118EE100AFDF794F908
:1031E000CDE906017068FDF78FF9CDE9040130687B
:1031F000FDF78AF9CDE902012846B04DB04BB14A3E
:10320000B149CDE9009839F0E9FF05F5F4513846A8
:1032100095ED00AA1AF04AFF8DED160A9AED000A04
:10322000CDED170A30EE4A0A8DED181A18F0FCFDA4
:103230009DED167AD4EDBB7AB0EEC77AB4EEE77A9C
:10324000A5F25C43F1EE10FA0C9300F11082D4F871
:103250001C3D1B7B002B00F00A82B4F8EA92C9F3F4
:1032600040099DED177AB0EEC77AF4EEC77AF1EE19
:1032700010FA00F3FF81D4F81C3D1B7B002B00F0FB
:10328000F981B4F8EA3203F001039DED187A0B934B
:10329000B0EEC77AF4EEC77AF1EE10FA00F3EC81E3
:1032A000D4F81C3D1B7B002B00F0E681B4F8EA3219
:1032B000C3F38008B0EEC00AF4EEC07AF1EE10FA63
:1032C00000F3DD81D4F81C3D1B7B002B00F0D7817F
:1032D000B4F8EA32C3F3C00B0DAB00930B999FED2A
:1032E0007B8A5B4642464846FFF704FFC3B20BEEBB
:1032F000103AC0F307230AEE903AC0F307430CEEEE
:10330000903A030E0DEE103A9DF834300F90002BDA
:1033100040F0B8819DF83530002B40F0B381F8EED5
:103320004B7A6B4ACDED197AF8EE6A7AB0EE690AFB
:10333000CDED1A7AF8EE6C7A19AB394602F5467083
:10334000CDED1B7A54F038FF8DED140ACDED150A42
:10335000B0EE409AF0EE608A9DF836305D4C002B5E
:1033600040F095811CEE901AD4EDB90A97ED020A4F
:10337000B0EE691A04F5E86055F03CF8B0EE40CACA
:103380009DF83730002B40F085819AED000A30EE31
:103390004A0A18F049FD1DEE101A4F48F0EE690A6E
:1033A00054F00AFD04F64C03DAF800201A6004F524
:1033B0000563F0EE40BA83ED00AA484D95EDB41ACE
:1033C0004720F1EE410AB0EE490A18F041FD95EDB3
:1033D000B41AB0EE40AAF1EE410A4820B0EE680AF5
:1033E00018F036FD95EDB51AB0EE409AF1EE410AAF
:1033F0004920B0EE4C0A18F02BFD95EDB61AF0EE10
:10340000408A4A20B0EE6B0AF1EE410A18F020FD26
:1034100096ED007AD6ED017A9DF834308DED148A60
:103420006AEE076AF0EE40BACDED106A69EE276ADF
:103430008DED158ACDED116AD4EDB46A27EE267AAA
:10344000D4EDB56A8DED127A67EEA67ACDED137ADA
:10345000B3B99DF835309BB9B8EE4BBAF8EE6AAA0D
:10346000B0EE690A1E488DED19BA19AB12AA10A95F
:10347000CDED1AAA54F06CFD8DED140ACDED150AB0
:103480009DF83630002B40F0088196ED000AD4ED0F
:10349000B60A144860EE200A1CEE901A28EE800A44
:1034A000B0EE691A54F0A6FFF0EE40AA1CE000BF8F
:1034B000B0250020A4707D3F00D7233C0C3A0020AB
:1034C00021280A0810550A0829550A08000000009A
:1034D0008C580020B0550020685D0020B0450020C9
:1034E00068590020B45A0020844814A9FEF762FEEF
:1034F0009DF83730002B40F0D38096ED010AD4EDD3
:10350000BB0A7F4860EE200AB0EE691A1DEE101A61
:1035100020EE2B0A54F06EFFF0EE409AD5F81C3DD9
:103520001B7B7BBB19A977488DED198A8DED1A8A13
:1035300054F058FE9FED740A744854F077FF9FEDE5
:10354000720A734854F062FC19A972488DED198A09
:103550008DED1A8A54F046FE9FED6B0A6E4854F0CA
:1035600065FF67489FED680A54F060FF04F5377304
:1035700093E807000C9B87E8070003F25C431B6895
:10358000CAF80030B9F1000F00F08D80D5F81C3D6D
:1035900083ED368A0B9B002B00F09080D5F81C3D04
:1035A00083ED358AB8F1000F00F09380D5F81C3D0B
:1035B00083ED388ABBF1000F00F09580D5F81C3DF3
:1035C00083ED378A9FED558A9FED4F4AD4EDB42A9B
:1035D00094EDB71AD7ED000A62EE882A2AEE082A7F
:1035E00021EE081A60EE880AF0EE443AB0EE443A52
:1035F000F0EE441AB0EE440A5DF078F99FED424ACD
:10360000D4EDB52A94EDB81AD7ED010A62EE882AF6
:1036100029EE082A21EE081A60EE880AF0EE443AF4
:10362000B0EE443AF0EE441AB0EE440A5DF062F9AE
:103630009FED354AD4EDB62A94EDB91AD7ED020ABA
:1036400062EEC82A28EEC82A21EE481A60EEC80A9F
:10365000F0EE443AB0EE443AF0EE441AB0EE440ACA
:103660005DF04CF91DB0BDEC0C8BBDE8F08F4FF058
:103670000109F6E5012308E64FF001081AE64FF0CC
:10368000010B29E6F0EE488AB0EE489A64E69FED19
:103690001ECA75E6DFED1CBA8FE6DFED1BAA23E735
:1036A000DFED199A3AE79DF83430002B7FF472AFC2
:1036B000D5F81C3D149AC3F8D8206BE79DF8353037
:1036C000002B7FF46FAFD5F81C3D159AC3F8D420BA
:1036D00068E79DF83630002B7FF46CAFD5F81C3DC1
:1036E000C3ED38AA66E79DF83730002B7FF46AAF48
:1036F000D5F81C3DC3ED379A64E700BFB025002024
:103700002C5B0020A45B002000000000F05C002087
:10371000685D002068590020B45A00200000C842AB
:103720002DE9F04F2DED068B8FB0B74C0393D4ED00
:1037300037AA04F500548046D4F81C3D1B7B0D4687
:103740001746002B00F02E81B4F8EA62C6F3400B56
:1037500006F0010AC6F3800916F0080600D001261B
:1037600003AB4A465146009358463346FFF7C2FC26
:1037700094EDB41A95ED000A0590F1EE410A9A20F5
:1037800018F066FB94EDB41AF0EE409AF1EE410A9F
:1037900095ED010A9B2018F05BFB94EDB51AB0EE95
:1037A000409AF1EE410A95ED020A984D9C2018F0DE
:1037B0004FFB94EDB61AF0EE408A9D2097ED000A7B
:1037C000F1EE410A18F044FB98ED007AD8ED017A49
:1037D0009DF80C3069EE876A0027CDED066A69EE28
:1037E000276AB0EE408ACDED076AD5EDB46A0A9734
:1037F00027EE267AD5EDB56A8DED087A67EEA67AC2
:103800000B97CDED097AFBB99DF80D30E3B99DF822
:10381000143007EE103A9DF8153007EE903AB8EEE6
:10382000477AF8EE677AB0EE6A0A0CAB08AA06A9E6
:1038300005F56E708DED0C7ACDED0D7A54F088FBA8
:103840008DED0A0ACDED0B0A9DF80E30002B40F0ED
:10385000AE8098ED000AD5EDB60A9DF816106C48BA
:1038600060EE200AB0EE6A1A28EE800A54F0C2FD1B
:10387000B0EE40AA64480AA9FEF79CFC9DF80F3000
:10388000002B40F0978098ED010AD5EDBB0A9DF81A
:103890001710604860EE200AB0EE6A1A20EE080A9F
:1038A00054F0A8FDB0EE408AD4F81C3D1B7B7BB9D8
:1038B00059480C970CA90D9754F094FC9FED570AAA
:1038C000534854F0B3FD9FED550A524854F0AEFDF5
:1038D000BBF1000F71D0D4F81C3DC3F8D870BAF119
:1038E000000F74D0D4F81C3DC3F8D470B9F1000FA8
:1038F00077D0D4F81C3DC3F8E070002E7AD0D4F80D
:103900001C3DC3F8DC709FED468A9FED444AD5ED1F
:10391000B42A95EDB71A62EE882A29EE882A21EE9C
:10392000081AF0EE443AB0EE443AF0EE441AF0EEE3
:10393000440AB0EE440A5CF0D9FF9FED384AD5ED59
:10394000B52A95EDB81A62EE882A29EE082A21EEEA
:10395000081AF0EE443AB0EE443AF0EE441AF0EEB3
:10396000440AB0EE440A5CF0C5FF9FED2C4AD5ED49
:10397000B62A95EDB91A62EEC82A28EEC82A21EEB9
:10398000481AF0EE443AB0EE443AF0EE441AF0EE43
:10399000440AB0EE440A5CF0B1FF0FB0BDEC068BF8
:1039A000BDE8F08F4FF00109CA46CB46D7E69FED40
:1039B0001BAA5FE79FED198A76E79DF80C30002B74
:1039C0008DD1D4F81C3D0A9AC3F8D82087E79DF81A
:1039D0000D30002B8AD1D4F81C3D0B9AC3F8D420AB
:1039E00084E79DF80E30002B87D1D4F81C3D83ED81
:1039F00038AA82E79DF80F30002B84D1D4F81C3D03
:103A000083ED378A7FE700BFB0250020B055002046
:103A1000B45A00202C5B00206859002000000000F0
:103A20000000C84270B50446143045F06DFD0B4EE1
:103A30000B4B63616425601945F02EFF66513035EC
:103A4000B5F5597FF7D104F5597047F01FFA2046B4
:103A5000044935F0FBF9204670BD00BFE85E0A0856
:103A6000FC5E0A08AC570A0837B500F50A51012276
:103A70002031044637F09EFC184A1368D90706D453
:103A8000174904F5035318330B600123136004F541
:103A90000B50134901223430012534F0B5FC114A92
:103AA0000095002304F57F61FD2034F05BFC0E4B94
:103AB0001A68D20705D40D4A1D6004F58B541834DA
:103AC00014600A48012134F0BBFC35F0C5FB084AFC
:103AD000138843F04003138003B030BD6C5F0020B7
:103AE000002200204CE00A08705F00200C22002019
:103AF000806000200069C0F3401070470F299DBF0F
:103B0000302303FB0100503000207047014B93F934
:103B1000BE027047B0450020024B93F8190D00F02B
:103B200001007047B0450020014BD3F8880A704768
:103B3000B0450020054A92F8193D92F8182D03F07F
:103B4000010313430CBF012000207047B045002043
:103B5000002910B517DB104C94F8902ACBB29A428A
:103B600011D3D4F88C3A0122595CA4F5005000F02E
:103B7000ABFD94F8093D38B99A0704D5074A137884
:103B800043F00403137010BD9B07FCD5034A137860
:103B900043F00203F6E700BFB045002014600020A8
:103BA000022A10B50F4C12D13522A4F5005000F0B6
:103BB0008BFD94F8093D9B0705D50B4B1A7818B17E
:103BC00042F002021A7010BD42F00402FAE794F8C3
:103BD0000C2D8A42F7D145F029FEBDE8104045F092
:103BE000AFBD00BFB04500201460002010B500F547
:103BF0000053DFED186AD3F8802AD3F87C3AB2F983
:103C00000820B3F908309FED147A07EE902AF8EEF9
:103C1000E77A0446C7EEA60A00F59250012110305B
:103C200007EE903AF8EEE77A60EE870A87EEA60A8A
:103C300020EE070A03F0A0FA39F0A4FE262139F09D
:103C400039FC04F52B50054ABDE810400621203010
:103C50003DF098BA0000C84235FA8E3C385D0A083B
:103C6000332901D046F0C2BB70470000332910B59C
:103C700019D0382913D0052917D1022A0DD10D48A2
:103C800090F80C3D012B08D8D0F8843AB3F90830ED
:103C90001BB9A0F50050FFF7A9FF012010BD0321BB
:103CA000FFF77EFFF9E70121FAE7BDE8104046F093
:103CB000FBB800BFB045002030B5044689B0684667
:103CC00004F5925506F0A0FD103504A806F09CFD01
:103CD0006946284602F07CFF60B104A9284602F03C
:103CE000C7FF38B1059B019323680022DB6C69464E
:103CF0002046984709B030BD00F5805292F8CC2498
:103D0000D2070AD400F50052D2F81C2D117B09B15C
:103D1000FFF7D2BF03689B6C1847704710B586B099
:103D2000044602A8019106F06FFD04F5925002A925
:103D3000103002F04DFF28B12368019ADB6C02A914
:103D40002046984706B010BDF0B5044685B004F58E
:103D50009256684610360F46154606F055FD6946E0
:103D6000304602F085FF10B9002005B0F0BD39469D
:103D7000304602F009FE0028F6D0002DF5D004F5FB
:103D80008054284694F8CC3443F0020384F8CC34B1
:103D9000EBE7000010B500F50054D4EDB27AF5EE73
:103DA000C07AF1EE10FA8AB04FF0000344D90793BD
:103DB0000893099306AB019300F5925007AB03AA51
:103DC00004A90093103005AB02F076FEDDED080A81
:103DD0009DED070A87F016F8DDED090A87F012F865
:103DE000D4EDB27A9DED047A77EEA76AB4EEE70AD5
:103DF000F1EE10FAF4EEC76AACBF01200020F1EE3C
:103E000010FA0CD802309DED037AF4EEC77AF1EE89
:103E100010FA0CD8003818BF01200AB010BDF4EE1B
:103E2000C77AF1EE10FA9CBF0130C0B2EBE701286F
:103E300094BF00200120F0E70020EEE738B500F540
:103E40000055044695F8193D5A071AD443F0040367
:103E500085F8193D39F096FD0122112139F04AFB10
:103E6000084BD3F8B00803689B68984718B995F9D0
:103E7000C532032B05D120460621BDE8384000F0AD
:103E80001DBD38BDB055002008B500F5005090F8B4
:103E9000193D5A070BD56FF3820380F8193D39F0AD
:103EA00071FDBDE808400022112139F023BB08BD97
:103EB0002DE9F043054685B005F59258684608F1AE
:103EC000100806F0A1FC6946404602F0D1FEC8B1D8
:103ED00005F50053424CD3F81C2D424F127B32B1F2
:103EE000D3EDB27AF5EEC07AF1EE10FA0DD8238850
:103EF00023F4FF7323F00103238028460023FB7380
:103F0000FFF7C2FF05B0BDE8F083284601F0BEF818
:103F1000064618B9284601F07FF806462846FFF7FE
:103F200039FF814640B93EB12378002B41D16378F7
:103F300003F00103FB73E5E76378DB07F7D423782D
:103F40000133DBB2082B237006D12846FFF722FF8E
:103F500010B1404602F01CFE2378092B02D14046E6
:103F600002F00EFE2378092BE1D9238823F4FF7396
:103F700023F0010343F48573238039F003FD02220B
:103F8000102139F0B7FA5DF095FE6368C01A47F268
:103F90003053984209D905F52B50134A022120309D
:103FA0003DF0F0F85DF086FE60602846FFF746FFC2
:103FB000BDE7013B23702388C3F30803B3F5807F7B
:103FC000B5D1637860F30003637039F0DBFC4A46D7
:103FD000102139F08FFA2846FFF756FFA7E700BFF8
:103FE000745F0020F55F0020185F0A0837B50446AB
:103FF00000F5925001A9103004F5005502F0DAFBEB
:10400000D5F8CC3A834206D0C5F8CC0A39F0BAFCD0
:104010003E2139F04FFA04F5805395F9D01A93F800
:10402000602593F96035994213D0FF2A11D085F8A5
:10403000D03A39F0A7FC95F8D02A182139F05AFA6D
:1040400004F52B5095F9D03A034A042120303DF075
:1040500099F803B030BD00BF285F0A082DE9F0438E
:1040600095B006465DF026FE06F5925803AB019327
:1040700008F1100802AB0024009305460EAB0BAA12
:1040800008A94046089409940A940B940C940D9442
:104090000E940F94109402F0FDFCDFED437A9DED39
:1040A0000A7AB4EEE77AF1EE10FA074637DB9DEDB7
:1040B0000D7AB4EEE77AF1EE10FAACBF4FF00109D9
:1040C0004FF0000907AB019311AB009304AA06ABB4
:1040D00005A9404611941294139402F0EDFC06F5E4
:1040E0000054002894F9703A08BF002783B17FB1CB
:1040F000D4F81C3D1B7B5BB1B9F1000F08D09DEDDE
:10410000057AF7EE007AB4EEE77AF1EE10FA09D507
:1041100094F8D43A73B90023C4F8D83A0FE04FF0BA
:104120000009CFE7D4F8D80A20BBC4F8D85AC4F89D
:10413000DC0A04E0D4F8DC0A20B9C4F8DC5A15B073
:10414000BDE8F083281A43F698239842E3D9002566
:1041500084F8D45AC4F8DC5A39F014FC2A461D21DC
:1041600039F0C8F906F52B50104A022120303DF0F5
:1041700009F8D0E72D1AB5F57A7FE0D994F8D43A4A
:10418000002BDCD1012584F8D45A39F0FBFB2A46F8
:104190001D2139F0AFF906F52B50054A02212030D8
:1041A0003CF0F0FFCBE700BF00000034405F0A089E
:1041B0005B5F0A0810B5044639F0E4FB00220521D4
:1041C00039F098F904F52B50034ABDE8104004215A
:1041D00020303CF0D7BF00BF785F0A0800F50050E0
:1041E00090F8093D9B065ABF90F8080DC0F30010E7
:1041F0000120704737B5044600F54E501C305CF086
:104200009FF804F50052C0F3803592F8093DC3F3DE
:104210000011A9421DD065F3041304F52B5482F854
:10422000093D20346DB139F0ADFB02220B2139F08C
:1042300061F9094A0221204603B0BDE830403CF054
:10424000A1BF39F09FFB2A460B2139F053F9034AED
:10425000F0E703B030BD00BF905F0A089B5F0A081B
:1042600070B500F50055044695F9AE32B3B3D5F8F4
:10427000986C9EB35DF01EFD05F6782393ED000A61
:10428000DFED177A9FED171ADFED170A861B20EE78
:10429000270A6B2017F0DCFDBCEEC00A10EE103AC6
:1042A0009E4209D295F8193D9A0717D5204600215C
:1042B000BDE87040FDF75EBC10D995F8193D9B072D
:1042C0000CD420460121FDF755FC04F52A500122AB
:1042D000BDE8704012211430FDF7BABB70BD00BFBD
:1042E00000007A440000804F000000000B46012BC4
:1042F00010B4114604D0052B06D05DF8044B70476E
:104300005DF8044B00F0DABA142100F52A505DF88C
:10431000044B01220844FDF79BBB00002DE9F0414E
:10432000044604F5005839F02DFB0122052139F02F
:10433000E1F898F9B2522046003D18BF0125FFF779
:104340004DFF04F52B56203698B11E4A0421304605
:104350003CF018FF04F52A50012210211430FDF71B
:1043600077FB0025294620460322BDE8F041FFF7F0
:10437000BDBF04F54057D7F8B00803689B6A98475B
:1043800068B197F8A13253B197F9A032012B06DC3E
:104390000D4A042130463CF0F5FE0125E2E7D7F84E
:1043A000B00803689B6A984718B1D8F8743A1B079D
:1043B00005D4064A042130463CF0E4FED2E7044A24
:1043C000E7E700BFB05F0A08CB5F0A08F95F0A0899
:1043D00008600A0870B50446154639F0D3FA012280
:1043E000062139F087F82046FFF7F8FE04F52B5632
:1043F000203698B104F52A50012207211430FDF728
:1044000027FB154A042130463CF0BCFE0025294616
:1044100020460422BDE87040FFF768BF04F5405312
:10442000EDB2D3F8B00803689B6A984768B104F509
:104430000053D3F8743A1B0707D535B1074A042156
:1044400030463CF09FFE0125E1E7054A0421304655
:104450003CF098FEDBE700BF2C600A08D35F0A0837
:1044600049600A08F8B504465DF018FC284BB4F81A
:10447000BE201988274E914205460ED01A80264B41
:1044800018603378A3B10024347039F07BFA2246E7
:104490001321BDE8F84039F02DB833781F4FC3B968
:1044A0003B782BB11C4B1E4A1B68C31A934200D8A1
:1044B000F8BD0123337004F50053D3F81C0D037BC2
:1044C0000BB1FEF7FDF939F05DFA0122132139F045
:1044D00011F83B78002BEBD03378002BE8D00E4A54
:1044E00010491368EB1A8B42E2D904F500541560A9
:1044F000D4F81C2D137B002BDAD0002313730A4A47
:10450000D4F81C0D1371BDE8F840FEF7A9B800BF40
:104510007E5F00207C5F0020805F00207D5F0020A8
:1045200080841E0040420F00F55F002070B500F54A
:10453000005300F54E551C3586B093F8D41A044646
:1045400028465BF0ABFE02A806F05EF904F5925037
:1045500002A9103002F03CFB04F54053049AC3F862
:10456000BC22059AC3F8C02228465BF0E9FE820609
:104570001AD528465BF0EEFE04F54A55FDEEC07AEA
:10458000343504F5805417EE901A0222284617EEAF
:10459000906A06F03FF994F8CC34DB0706D4012288
:1045A0003146284606F036F906B070BD012128468E
:1045B00006F0F4F90028F2D0F6E700000120704779
:1045C000002070470020704700207047002070478F
:1045D000002070470020704700207047002070477F
:1045E0009FED010A704700BF000000007047000007
:1045F0000F4A02600F4A426002F1540181600E4985
:10460000C1600E49016102F67C21416102F5286119
:10461000816102F2DC71C16102F5FC61016202F2AA
:10462000E47102F5FD628262054A4162C26270472E
:10463000D4600A08504800204C590020003800205F
:10464000C8260020042917D8DFE801F003070B0F64
:10465000130000F563502430704700F56250343089
:10466000704700F564501430704700F56550043011
:10467000704700F56650FAE70020704700F540509B
:10468000D0F8B00803685B681847000038B500F53B
:1046900040550446D5F8B00803685B699847094B54
:1046A00004F50052187492F80C2DD5F8B008DA70A1
:1046B00003685B6A9847014604F59050BDE83840AE
:1046C00031F098BBF55F00202DE9F84F00F5005A56
:1046D00006469AF80C3D8B420F46914605D18AF862
:1046E0000D2D01252846BDE8F88FFFF7ABFF0446E6
:1046F00020B9304637F0E4F82546F3E7DAF81C3DF8
:104700001B7B06F52B5883F0010B08F12008E3B959
:10471000236859461B6820469847054678B306F536
:1047200040534A46C3F8B048394606F57F608AF8D8
:104730000C7D8AF80D9D38F0EDFA4046002144F0DA
:104740007BF93046FFF7A2FFCCE703689B689847E8
:10475000E0B11C4800F084FC0546B8B92368204647
:104760001B6A9847184A0346042140463CF00AFD5C
:1047700039F008F93A460A2138F0BCFEB2E723685E
:1047800020461B6A9847114A0346EDE70D4800F0A2
:1047900085FC0028BCD106F54053D3F8B008036867
:1047A000DB6898470028B3D023682046DB68984729
:1047B00005460028ACD1236820461B6A9847044A66
:1047C0000346D1E7B02500205C600A08AE600A0805
:1047D00085600A080148FFF777BF00BFB0250020B9
:1047E00070B5234B93F8193DDB0705460C4616467A
:1047F00005D5002363602360A360336070BD45F07E
:1048000015F8037F002BF4D0EB699FED1A7A1B6833
:10481000B3F9083007EE903AF8EEE77AC7EE876A08
:10482000C4ED016A2B6A1B68B3F9083007EE903AB1
:10483000F8EEE77AC7EE876AC4ED006A6B6A1B6818
:10484000B3F908305B4207EE903AF8EEE77AC7EE2C
:10485000876AC4ED026AAB6A1B68B3F9083007EED9
:10486000903AF8EEE77AC7EE876AC6ED006AC5E7C8
:10487000B045002000007A440020704701207047B6
:1048800000207047002070470048704718610A08F0
:104890000048704718610A0843691A680023C2F883
:1048A000D43042691268C2F8D83042691268C2F83E
:1048B000DC3042691268C2F8E03070470A4608B539
:1048C0000021FFF701FF034A137843F00803137038
:1048D00008BD00BF14600020012070470020704711
:1048E0000120704700207047004870476C610A083B
:1048F0000048704774610A0830B5084B03F54B5205
:104900001C32044600F1300507CA85E8070003F5AC
:10491000A2531C3301201B68E36330BDB025002087
:1049200030B52DED028B044687B0574D002301AA08
:1049300003A995ED378A039304930593FFF750FF7E
:1049400063689DED037AD3ED0F7A68EE277A27EE40
:10495000277A8DED037A9DED047A67EE277ACDED07
:10496000047AD3ED107A28EE277ADDED057A67EE2A
:10497000877ACDED057AD3ED117A93F9483028EE98
:10498000278ADDED017A27EE888A8DED018A1BB931
:1049900003A92846FDF7F6FB3C4A94ED0C7AD2EDCC
:1049A000B77A636894ED0F0AD3ED0F6A77EE677AF2
:1049B000F0EEE77AF4EEE67AF1EE10FA44BFDDEDC0
:1049C000037A77EE877A94ED0D7A48BFC4ED0C7ABE
:1049D000D2EDB87AD3ED0F6A77EE677AF0EEE77A28
:1049E000F4EEE67AF1EE10FA44BFDDED047A77EEEC
:1049F000877A94ED0E7A48BFC4ED0D7AD2EDB97A7C
:104A0000D3ED106A236977EE677AF0EEE77AF4EE79
:104A1000E67AF1EE10FA42BFDDED057A77EE877A9D
:104A2000C4ED0E7AD3ED837A30EE670A17F0FCF905
:104A30006368D3ED117AB0EEC00AB4EEE70AF1EE86
:104A400010FA09D594ED0F0ADDED017A30EE270A50
:104A500017F0EAF984ED0F0A00230D488DF80830AD
:104A60008DF809308DF80A308DF80B30029BD0F8A4
:104A7000200D04F13C0204F13001FEF751FB07B0B8
:104A8000BDEC028B30BD00BFB0250020B05500202A
:104A9000B04500200020704701207047012070477A
:104AA0000020704700487047C8610A0800487047F6
:104AB000D0610A081FB5044600236A4601A9019384
:104AC00002930393FFF78CFE6369029A1B68C3F895
:104AD000D4206369019A1B68C3F8D8206369009ADF
:104AE0001B68C3F8DC206369039A1B68C3F8E020E5
:104AF00004B010BD012070470020704701207047AE
:104B00000020704700487047882D0A080048704709
:104B1000882D0A08012070477FB500230393049372
:104B200005930193094800238DF808308DF809306A
:104B30008DF80A308DF80B30029BD0F8200D01AAB9
:104B400003A9FEF7EDFA07B05DF804FBB0450020BD
:104B500001207047002070470120704700207047F7
:104B60000048704770620A08004870477C620A0873
:104B700010B5044686B0002301AA03A90393049349
:104B80000593FFF72DFE63689DED037AD3ED0C6A64
:104B9000DDED047A93F9483027EE267A67EEA67A9F
:104BA0008DED037ACDED047A1BB9144803A9FDF706
:104BB000E9FA6368DDED057A93ED0D7A104867EE4A
:104BC000877A93ED0E7ACDED057ADDED017AD0F896
:104BD000200D002367EE877A8DF808308DF80930B4
:104BE0008DF80A308DF80B30029BCDED017A01AAC9
:104BF00003A9FEF795FD06B010BD00BFB02500204B
:104C0000B045002038B5044646F094F946F066FAFF
:104C100004F50054054646F0F7F945F083FED4F854
:104C20001C0DFDF71DFD2846BDE8384046F0F4B9DF
:104C300070B500F50055044695F9A43A43B1D5F88E
:104C4000842A344EB2F90820002A02DD0023338082
:104C500070BDD5F8882AB2F90820B2F5617F31DD40
:104C6000B6F90030642BDCBF01333380B6F9003075
:104C7000142B0DD1D5F81C3D197B0029E8D100F586
:104C80002A5001221430FCF749FE08B93080DFE7D2
:104C9000B6F90030642BDBD1D5F81C3D1B7B002B13
:104CA000D6D095F80C3D012BD2D104F52B501A4AE1
:104CB0000621203004F540543CF064FAFA23A4F8AD
:104CC000A438C5E712F5617FC0DA022BBED100F52A
:104CD0004053D3F8B0080368DB68984718B995F8D3
:104CE000083DDB06B2D5B6F90030142BB0DC013339
:104CF0001BB2142B3380ABD1D5F81C3D1B7B002B92
:104D0000A6D004F52A500122BDE8704000211430DD
:104D1000FCF79EBE845F0020D0620A0810B500F543
:104D200000541421D4F87C0A44F0CAFDD4F8800A57
:104D3000142144F0C5FDD4F8840A1E2144F0C0FDBE
:104D4000D4F8880A142144F0BBFD44F06FFD0368D9
:104D500005211B689847BDE81040002144F0B0BD14
:104D600038B5054644F062FD44F038FD05F50054C1
:104D7000C4F87C0A44F05AFD44F03AFDC4F8800AB5
:104D800044F054FD44F03EFDC4F8840A44F04EFD66
:104D900044F042FD4FF47A71C4F8880AD4F87C0AD2
:104DA00044F08AFDD4F8800A4FF47A7144F084FD0F
:104DB000D4F8880A4FF47A7144F07EFDD4F8840A5E
:104DC0004FF47A7144F078FD2846FFF7A7FF94F876
:104DD000093D43F0080384F8093D38BD08B546F0A5
:104DE0007DF945F021FFBDE8084045F0D3BE000045
:104DF00000F50050D0F81C0DFDF762BD38B500F588
:104E00000054054694F9B232BBB1B4F8B4328B42C7
:104E10001DD994F8193DDA070FD444F007FD037F3C
:104E20001BB9D4F81C3D1B7B3BB194F8183D0133F2
:104E30005BB2022B02DC84F8183D38BD032384F8F2
:104E4000183D01212846BDE83840FCF779BE94F8AA
:104E5000183D013B5BB2002BEDDC94F8193D0021BD
:104E6000DB0784F8181DE8D5EDE7000038B50D46DE
:104E700004465CF01FFF002D0B4B09DD04F50054C8
:104E8000186094F8093D6FF3C30384F8093D38BDF9
:104E90001B68C01AB0F5C87FF9D904F5005494F81E
:104EA000093D43F00803F0E7885F0020F7B50446AA
:104EB0005CF000FF064644F0B9FC44F05FFB04F5EB
:104EC0000055B0B395F8083D43F0200385F8083D40
:104ED000D5F8843A2046D988FFF790FFD5F8843A70
:104EE00004F54057B3F908102046FFF7BFFFD7F885
:104EF000A8389FED267AF31A07EE903AD5F8843A4F
:104F0000F8EE677AB3F9083067EE877A04F54A500D
:104F1000CDED007A07EE903AF8EEE77A6A4601A9FD
:104F20002830CDED017A3BF057FAC7F8A86803B0F6
:104F3000F0BD95F8193DDB07F9D404F54053D3F8DB
:104F4000A808361A44F0A4FB002814BF4FF47A7363
:104F50004FF4FA73B342EAD895F9B232002BE6D097
:104F600044F064FC037F23B9D5F81C3D1B7B002B68
:104F7000DDD038F007FD0222114638F0BBFA0121DE
:104F8000204603B0BDE8F040FCF7DABD6F12833A6B
:104F900038B5044600F58C65284604F01FFA94F8ED
:104FA00071049FED087A242202FB0055D5ED0B7A9F
:104FB00067EE877A04F54053FDEEE77AC3EDA97AF0
:104FC00038BD00BF0000C842FEF772B80148FFF7C5
:104FD00049BA00BFB025002038B500F5925510350C
:104FE0000446284600F014FD04F58053022283F89D
:104FF0006424B4F9A43004F6C8001BB9B4F8A23094
:10500000A4F8A430B4F8A41016F0B8FA2846BDE805
:10501000384000F0F7BD000013B5044600F592508B
:10502000103000F0F9FE98B104F54E5004F500542C
:105030001C305BF085F9D4F81C2D0190127BC3B2B3
:10504000C0F3001032B918B99DF80500C0F3400054
:1050500002B010BD0028FBD083F08000C009F7E744
:1050600038B500F50053054693F8193D5B070AD49F
:10507000FFF7D2FF044620B905F59250103000F03A
:10508000CBFE204638BD0024FBE7000008B500F544
:105090009250103000F0C0FE002008BD13B5044649
:1050A00000F59250103000F0B7FE58B104F54E50A4
:1050B0001C305BF045F94207C3B203D5C3F340107F
:1050C0009B0600D4002002B010BD000038B500F5EA
:1050D0000055044695F8083D590719D5D5F81C3DEB
:1050E0001B7B2BB920460021BDE83840FCF712BDE0
:1050F00000F54053D3F8B0080368DB68984738B12F
:1051000095F8093D1A0703D595F8193DDB07E9D550
:1051100038BD000037B500F57F65044604F500543E
:105120002846019137F056FD94F8083D019960F347
:10513000C303284684F8083D03B0BDE8304038F08A
:1051400047BA00000720704700487047E0620A082D
:1051500037B5154BB3F9A42005461AB9B3F8A22008
:10516000A3F8A420B3F8A4100191EC2005F046FEAA
:10517000044610B10199FDF713FA05F50050C0F887
:105180001C4D24B990F90413084805F0FDFA0849AC
:10519000204634F069F8012033F0E4FC03B0BDE8A8
:1051A000304034F059B800BFB0250020E8620A084A
:1051B0006C1F0A08F7B5044600F5905030F0E6FD84
:1051C0002046FFF763FA04F53450303004F0CCFD8C
:1051D00004F58C6704F5895046F048F9384604F028
:1051E00033FC04F52B50203040F0AEF96C4E2046D5
:1051F000FFF7B6FD2046FFF7ABFFB6F9A4301BB9A9
:10520000B6F8A230A6F8A430082005F0F7FD18B1D2
:105210004FF07E530360436004F50055C5F8200D40
:1052200044F004FB9922292145F0BCFA44F0FEFA2F
:1052300044F0A4FA2046FFF7D1FD95F8093D04F5A6
:105240008E5043F0400385F8093D0C3048F0DEFDF8
:10525000544B55491B68986A03684FF47A72DB6AAD
:1052600098470423C4F8A43104F590700DF05AFD5A
:1052700006F03CFB4FF40053036306F037FB07F0E6
:10528000FBFB8023C4F874340121384604F0B6F9DE
:10529000464B0193009602AB13E9060004F57F60CC
:1052A00037F050FB2046FFF797FE4FF40023C4F879
:1052B000E03BD5F81C0DFDF77DF904F52A500121DE
:1052C0001430FCF731F910B12046FFF791FDB4F925
:1052D000A43004F54B5030301BB9B4F8A230A4F818
:1052E000A430B4F8A420D5F81C3D00EE102AD3ED6C
:1052F000390AB8EE400AF2EE0E1AB6EE001A3BF08A
:105300001DFDB4F9A43004F54C5034301BB9B4F889
:10531000A230A4F8A430B4F8A420D5F81C3D00EEC7
:10532000102AD3ED390AB8EE400AF2EE0E1AB7EEA3
:10533000001A3BF017FBB4F9A43004F54D502830A7
:105340001BB9B4F8A230A4F8A430B4F8A420D5F85E
:105350001C3D00EE102AD3ED390AB8EE400AF2EEF9
:105360000E1AB1EE041A3BF0FDFA95F8BF121A229C
:105370002046FFF7A9F960B9212201212046FFF755
:10538000A3F995F8093D43F0020385F8093D03B000
:10539000F0BD074A137843F008031370F1E700BF2C
:1053A000B0250020685F0020CD4F0108C94F0108DB
:1053B0001460002070470000002070477047000014
:1053C0000020704700207047002070470020704781
:1053D0009FED010A704700BF000000009FED010A29
:1053E000704700BF000000007047000000207047B9
:1053F0007047000010B50446143000F019F804F1AD
:105400002C0000F015F804F174005CF05FFC04F16E
:10541000F4005CF05BFC4FF0FF33C4F850312046E1
:1054200010BD0000014B1868704700BF8C5F002062
:1054300070470000F0B52DED048B91B004466D4629
:10544000284605F0E1F994F8BC33002B72D004F53E
:105450007A730FCB85E80F0094F8F833D4EDEC8A1B
:1054600094EDED8A94EDEE9A002B63D094F8D0334E
:10547000002B5FD02D22002104A8D4F8C073D4F8EB
:10548000C463D4F8C853D4F8CC4388F03DF8A323C0
:105490008DF8103095238DF8113046238DF8123099
:1054A0005CF010FC9FED250A9FED257ACDF81710D2
:1054B00068EE807ACDF8130067EE877AFDEEE77A22
:1054C00017EE903A68EE007A29EE000A67EE877AC6
:1054D000ADF81B30FDEEE77A20EE070A17EE903AA2
:1054E000ADF81D3016F074FCDDED017A9FED157AF4
:1054F000CDF82D70BCEEC00AF8EEE77A10EE103A47
:1055000067EE877AADF81F3017EE903ACDF821306C
:10551000029BCDF82530039BCDF82930CDF83160C2
:10552000CDF83550CDF8394038F02CFA2D2204A9A9
:1055300037F030FA11B0BDEC048BF0BDE02E6542BF
:105540000000C8420AD7233C30B52DED028B8BB04A
:10555000044624220D4601A8002187F0D5FFA3238D
:105560008DF8043095238DF8053048239FED1F8A70
:105570008DF806305CF0A6FBD4ED817A2B68CDF86F
:105580000F3067EE887A95ED020ACDF80B1017EE12
:10559000903AD4ED827ACDF8133067EE887A6B6852
:1055A000CDF8173017EE903ACDF80700CDF81B3044
:1055B00016F0E4FB10EE103A94ED830ACDF81F309C
:1055C00020EE080A16F0DAFB10EE103ACDF8233080
:1055D00094F80C338DF8273038F0D4F9242201A93F
:1055E00037F0D8F90BB0BDEC028B30BDE02E654230
:1055F00030B587B014460D4618220021684687F062
:1056000083FFA3238DF8003095238DF801304923C3
:105610008DF802305CF056FBA3680393E3680493B3
:105620006368CDF807100593CDF803008DF80B5093
:1056300038F0A8F91822694637F0ACF907B030BD48
:1056400010B58EB0044602A805F0DEF802A9204687
:1056500001F0BEFA002845D001F004FD694601F0D2
:105660003DF91F22002106A887F04EFFA3238DF8E5
:10567000183095238DF819304A238DF81A305CF0D4
:1056800021FBDDED037A9FED1B7A049BCDF82330DF
:10569000F8EEE77A059BCDF8273067EE877ACDF8EC
:1056A0001B0017EE903ADDED007ACDF82B30F1EECD
:1056B000677A17EE903ACDF81F10204601A9CDF871
:1056C0002F3000F013FC78B1DDED017AF1EE677A4E
:1056D00017EE903ACDF8333038F054F91F2206A96E
:1056E00037F058F90EB010BD38F04CF9DFED027A02
:1056F000EEE700BF0AD7233C5241C07F002303607E
:1057000043608360C360036143618361C36103627B
:105710007047000090F8F432B02202FB030390F8C7
:10572000382393F8D13012B1012B28BF012318463A
:10573000704700002DE9F04F04468BB04FF0000A8F
:105740000D461AF0F9F984F814A204F506704FF02A
:105750007E575BF063F94FF47A73A4F8623284F8F1
:105760006852C4F84872C4F84C72C4F8507204F518
:105770001B70002505F048F804F52B790323C4F8C5
:10578000803204F53476C4F89452C4F89852C4F8C0
:105790009C52C4F8A052C4F8A452C4F8A852484677
:1057A000FFF7ACFF04F5487B3046FFF7A7FFC4F8CE
:1057B0001453C4F81853C4F81C535846FFF79EFFFF
:1057C000C4F84453C4F84853C4F84C53C4F8505375
:1057D000C4F85453C4F85853C4F85C53C4F8605325
:1057E000C4F86453C4F86853C4F86C53C4F87053D5
:1057F000C4F88C53C4F89053C4F89453C4F8A85315
:10580000C4F8A453C4F8A053C4F8B053C4F8B453B4
:10581000C4F8B853C4F8CC53C4F8C853C4F8C4533C
:10582000C4F89C73C4F8C07304F5757004F0ECFF01
:1058300004F57A7004F0E8FF04F58063C4F8FC53C3
:105840001D6004F5816304F583601D605D609D60EB
:1058500004F0DAFF04F22C4304F264481D605D603A
:105860009D60684BC4F83C3404F50D73C4F84034B3
:1058700004F50E73C4F8443404F50F73C4F84834C7
:1058800004F51073C4F84C3404F24523C4F85034C2
:1058900004F51173C4F8543404F58B6340461D605D
:1058A0005D609D60FFF72AFF04F59160FFF726FF1A
:1058B00004F5976304F23C421D605D609D6004F254
:1058C000C44304F2A4501D605D609D6004F59A63BA
:1058D0001D605D609D6004F2DC431D605D609D6045
:1058E00004F2EC431D605D609D6004F2FC431D60AA
:1058F0005D609D6004F5A463C2F8D470C2F8D870EE
:105900001D605D609D6004F22C531D605D609D60B4
:1059100004F5A9631F605D6004F26C531D605D6057
:105920009D6004F5AF631D605D609D6004F5B2632A
:105930001D605D609D6004F067FF04F2B453242293
:105940001D605D6004F2BC5351461D605D6004F251
:10595000C45340461D605D6087F0D6FD04F2E450FC
:10596000C8F82070C8F81070C8F80070FFF7C6FEBD
:1059700004F5C16304F5C7601D605D609D6004F2BD
:1059800014631D605D609D6004F5C4631D605D600F
:105990009D6004F22C631D605D609D6004F034FF27
:1059A000194B1A491C60204633F050FA5146242204
:1059B000584687F0A9FDC4F84073C4F83073C4F8A2
:1059C000207304F5257207CA04F5287383E80700DD
:1059D000484694EDAA1AD4EDA90A94EDA80A16F047
:1059E0002FFE3546494668466E4616F04BFD0FCEF3
:1059F0000FC50FCE0FC533682B6020460BB0BDE836
:105A0000F08F00BF5C650A08905F002024640A08DC
:105A100010B5044688B001F0F1FB94F93232012B45
:105A200002D1274804F0CEFE022B0AD1032384F8CA
:105A3000323204A9012304F111008DF8103033F043
:105A4000CDFF94F8323284F8903204F23C4001F0F9
:105A500049FB94F93132642B30D1652304A904F257
:105A600031208DF8103033F0F7FF04A9204632F0D2
:105A7000FDF918B304238DF818300023CDE9013364
:105A800003930F230593694604A832F06FFB059B2F
:105A900028B108AA02EB8302009942F8581C01338E
:105AA000112B0593EFD959F06BF99DED031ADDED3C
:105AB000020A9DED010A652159F020F908B010BDD8
:105AC00008630A0870B500F5257600F528758CB0D6
:105AD00004463146284618F089FAE0B996E80700EE
:105AE00085E8070004F52B7194EDAA1AD4EDA90AF4
:105AF00094EDA80A0191084616F0A2FD02AD0199A5
:105B000002A816F0BFFC0FCD04F534740FC40FCDFE
:105B10000FC42B6823600CB070BD000013B540F2B9
:105B2000411200F50671044601A812F055FD04F279
:105B30003C4001F001FD20461AF046FA01A812F09F
:105B40006DFD02B010BD0000F8B50B68C0F804325E
:105B50004B68C0F808328B68C0F80C3201F10C06B3
:105B600007460C4600F548750FCE0FC50FCE0FC582
:105B700033682B6004F1300207CA07F5457383E8E8
:105B8000070004F13C0207CA07F5517383E80700D8
:105B900004F1480207CA07F5547383E80700543438
:105BA00094E8070007F5577383E80700384601F0CB
:105BB00039FC3846BDE8F84001F01CBC13B504467A
:105BC00000F23C40019003F0BBF804F5BB61019882
:105BD000009102F009FC0099204602B0BDE8104097
:105BE000FFF7B2BF4A78064BC2F340121A754A78E3
:105BF000C2F380125A750A78C2F300129A75704780
:105C0000F55F002013B540F2F522044600F5067159
:105C100001A812F0E1FC002104F23C4001F000FF79
:105C200094F8603223B120461AF0EAFB84F860024F
:105C300001A812F0F3FC02B010BD000038B590F8D6
:105C40000C3305460C462BB1032B0BD095F868326C
:105C5000DB070CD405F5C7630FCB84E80F0095F87C
:105C6000480603E01AF030FA0028EFD038BD0020D3
:105C7000FCE7000000F23C4090ED350A7047000060
:105C800000F23C4090ED360A7047000010B490F8E6
:105C90000C230C462AB1032A0AD000205DF8044BDD
:105CA000704700F5B26007C884E807000120F5E7F7
:105CB0005DF8044B1AF0C6B990F88403431E5842AD
:105CC0005841704738B590F80C330D468BB900F247
:105CD0003C4001F0A3FC044610B90024204638BD26
:105CE00001F0F0FBD5ED007A27EE800A85ED000A81
:105CF000F4E7D0EDE07AC1ED007A90F87C43002C17
:105D0000EBD090EDDE7ADFED086AB4EEE67AF1EEE4
:105D100010FAF7EE006AB8BFB0EE667A67EE877ADF
:105D2000C1ED007ADAE700BF0000003490F80C33D0
:105D3000032B01D11AF006B90020704790F80C230C
:105D4000032A01D11AF084BA00F23C4002F0CAB82A
:105D500030B590F80C3385B004460D468BB1032B5B
:105D600018D004F5257018F07BF9284601A98DEDAF
:105D7000010ACDED020A8DED031A17F003FF012091
:105D800006E000F23C4001F0F3FB0028E9D10020DE
:105D900005B030BD90F86032002BF8D01AF032FA1E
:105DA000DFE700007FB590F80C2332B1032A4FF0F3
:105DB000000309D0039304930CE000F23C4007B0C9
:105DC0005DF804EB01F0B0BC03A9039304930593C1
:105DD0001AF0AEF89DED030ADDED040A07B05DF898
:105DE00004FB000007B590F80C3333B100F57F7069
:105DF00003B05DF804EB18F05DB800F23C4001F030
:105E000093FC68468DED000ACDED010A18F052F8BA
:105E100003B05DF804FB000090F80C03003818BFD5
:105E20000120704708B590F80C23032A05D0BDE87F
:105E3000084000F23C4001F05FBC1AF079F8012004
:105E400008BD000010B590F80C230C461AB1032AC7
:105E500007D0002010BDBDE8104000F23C4001F02A
:105E6000EFBB1AF07BF8012084ED000AF2E7000096
:105E700090F80C33032B01D11AF084B9002070473D
:105E800030B590F80C3385B005460C4623B1032B92
:105E900009D0002005B030BD00F23C4005B0BDE89F
:105EA000304002F0D1BA002302A9029303931AF002
:105EB00027F80028EDD001A928461AF02DF800286F
:105EC000E7D0029B2360039B6360019BA360E1E733
:105ED00090F80C231AB1032A05D00020704700F275
:105EE0003C4002F0E5BA1AF00BB8000090F80C2321
:105EF0001AB1032A05D00020704700F23C4002F09E
:105F0000C9BA1AF009B8000090F932323BB990F8DA
:105F1000683213F0010F14BF0320002070470320E4
:105F200070470000F7B50446FFF7EEFF054600286E
:105F300062D0032839D194F860326BB394F8683298
:105F4000D8072BD501A920461AF084FBBDF80430F0
:105F5000002B18BF002594F8146206F0FD06012EF0
:105F60004AD10023032D019307D101A920461AF03D
:105F70007DFB20461AF084F9064604F23C4002F00C
:105F800015FB08B994F809039DF80430D90703D527
:105F90005A0701D59F0632D400252DE0204619F07E
:105FA0001FFF002808BF0025D5E70025D3E713F021
:105FB000020F2EE094F9443223B99DF80430DB0936
:105FC0002FD0E9E7002EF8D00EF0F4F9FFF7A2FB8E
:105FD000022807D99DF805309806DDD59DF80430D4
:105FE000D906D9D5FB6A93F89C30002BE5D118E08F
:105FF000DA0601D41B0718D5284603B0F0BD0028E7
:10600000FAD094F80923B4F94C36002ACFD013F013
:10601000010FF1D1154B1F68FB6A93F89C30002BE0
:10602000C8D19DF804309C07E2D405F05FFC05F070
:106030005BFB0028B0D10EF0BDF9FFF76BFB022827
:10604000AAD90EF0B7F990F8F432B02202FB03009F
:1060500090ED3B7AF0EE007AB4EEE77AF1EE10FACA
:106060009AD59DF80530DB09C6D195E7685F002019
:106070002DE9F04790F8603292B00446002B00F012
:10608000948020461AF032FC2046FFF74BFF03288D
:106090007BD104F5487800274146204600970197B8
:1060A00002971AF085F8694620461AF077F8009BA7
:1060B000C4F80432019BC4F80832029BC4F80C32C5
:1060C000204601F0AFF9204601F094F915F0E8F907
:1060D0000546204619F006FF0028A8BFC6B203AA4D
:1060E0004FF0FF312046BCBF95F8129395F813632B
:1060F0000397A8BFB1460497059719F03DFF03A881
:1061000017F0AEFF4FF00C0A0AFB095084EDD10ADC
:10611000C4EDD20A84EDD31A04F5517100F5117063
:1061200017F0AEFF04F557770AFB065584EDC50A54
:10613000C4EDC60A84EDC71A3A464FF0FF31204637
:1061400005F5C47519F02CFF95E8070006AE86E842
:1061500007003946304617F0F9FF04F52B72414627
:1061600009A816F01FF9314609A816F09DF809A9EB
:10617000204684EDD40AC4EDD50A84EDD61A1AF06F
:1061800075FA09A92046FFF72DFD94F84E36002B2D
:106190003AD109A804F038FB09A9204619F0A0FF5C
:1061A00090B3012384F84E362EE0D0F864321BB948
:1061B0005BF080FDC4F86402154B1B68D86A036865
:1061C0005B68984788B15BF075FDD4F86432C01AFB
:1061D000B4F86232984204D920461AF011F984F8D2
:1061E000600294F860327BB14BE75BF063FDD4F85A
:1061F0006432C01A41F287339842E4D837F0C2FBC8
:1062000037F002FA0028DED112B0BDE8F08700BFF7
:10621000685F002090F80C3323B1032B4FF000008F
:1062200007D0704790F93222032A04D10A70012066
:1062300070470870FBE718467047000073B50D46BD
:106240000DF107010446FFF7E5FF064628B19DF86A
:1062500007302BB1032B09D00026304602B070BDA9
:1062600004F5C7630FCB85E80F00F6E72946204603
:1062700019F02AFF94F86062EFE700007FB50E4640
:106280000DF103010446FFF7C5FF054618B90025C7
:10629000284604B070BD9DF8033083B1032B16D09F
:1062A00004F5257017F0DCFE01A930468DED010ADA
:1062B000CDED020A8DED031A17F064FCE8E73146D4
:1062C00004F23C4001F054F90028E9D1DFE794F8EA
:1062D0006032002BDBD03146204619F093FFDFE718
:1062E00037B50D460DF107010446FFF793FF28B1BE
:1062F0009DF8073023B1032B0FD0002003B030BD31
:1063000004F5BB631B682B6004F2DC5304F5BC642A
:106310001B686B602368AB60F0E72046294619F0E4
:106320003DFF94F86002E9E710B50446FFF7ECFD85
:1063300018B1032807D0002010BD04F23C40BDE88E
:10634000104001F03FB994F86032002BF3D02046A2
:1063500019F046FD0028EED094F8143203F0FD0346
:10636000012BE9D194F80C03C31E58425841E3E7CE
:1063700010B50446FFF7C8FD80B1032810D194F88A
:10638000600250B15BF096FCD4F86432C01A44F657
:106390002063984294BF0020012010BD0120FCE73B
:1063A0000020FAE708B50246FFF7AEFD032804D146
:1063B00010461AF05BF9012008BD0020FCE7000040
:1063C00030B585B004460191FFF72CF801990546D8
:1063D00010B9002005B030BD0191FEF7F3FF01991F
:1063E0000028F6D02846FEF7F1FF0028F1D0B4F8D7
:1063F0004C365907EED494F80933002BEAD00B4AF7
:106400001268D26A92F89C506DB103A92046FFF73A
:10641000C9FF30B19DF80E309A07DBD5C3F3800079
:10642000D8E72846D6E71846D4E700BF685F0020C3
:1064300010B50446FFF768FD032804D12046BDE8E7
:10644000104019F017BE002010BD00002DE9F041EA
:1064500090F80C338CB00027032B06460C461546EB
:1064600000970197029719D119F03CFD6A468046C2
:106470004FF0FF31304619F093FDB8F1FF3FA760B0
:10648000676027600DD115F00BF82B4690F81313B9
:10649000224614F093F80CB0BDE8F0814FF0FF38BD
:1064A000EBE714F0FDFF2B4622465FFA88F114F06B
:1064B00085F895ED000A684617F00EFE03A9204600
:1064C0008DED051A8DED030ACDED040A17F03EFEA1
:1064D00006F52B7206F5487103A815F063FF2146F7
:1064E00003A815F0E1FE84ED021A84ED000AC4ED64
:1064F000010A95ED007ADFED037AA7EE271A84ED05
:10650000021AC8E70AE81C411FB5DFED0B7A20EE3E
:10651000270A0C461946094BCDE90042BDEEC00AD8
:1065200018688DED020A064B9DF81820C06A12F01B
:1065300031FA04B010BD00BFE02E6542685F002054
:106540001C630A082DE9F0472DED028B92B000255F
:1065500004460F464FF07E5A00F5487106A8904653
:10656000CDF818A009950895079516F055FF05F088
:10657000BDF905F0B9F881462046FFF7C5FC0328B0
:1065800003D094F80C33032B4FD19FED558ADFEDE8
:10659000558A00262379F2B2934247D90AAA71B2EA
:1065A0002046CDF828A00D950C950B9519F00AFE04
:1065B0000AA906A817F058FBB4EEC80AF1EE10FAC3
:1065C0000DDD494ACDF800803B4648492046FFF79B
:1065D0009BFF002012B0BDEC028BBDE8F0870AA93A
:1065E00006A803950495059517F028FB03A90EA8A6
:1065F0008DED0E0ACDED0F0A8DED101ACDED111AAD
:1066000017F090F8B9F1000F0DD09DED050AB0EE2E
:10661000C00AB4EEE80AF1EE10FA04DD344ACDF80F
:1066200000803B46D1E70136B4E7002394F8686266
:1066300016F0010001D0012BCCD104F2E4510AA8DC
:10664000CDF828A00D950C950B9516F0E5FE0AA93E
:1066500006A817F009FBDFED227AB4EEE70AF1EEA7
:1066600010FA05DD204ACDF800803B462149ADE710
:106670002046FFF749FC03282DD1204619F0F4FDF0
:1066800094F86832DB0728D438BB0AA906A803951A
:106690000495059517F0D2FA03A90EA88DED0E0A00
:1066A000CDED0F0A8DED101ACDED111A17F03AF855
:1066B000B9F1000F11D09DED050ADFED0A7AB0EEB9
:1066C000C00AB4EEE70AF1EE10FA06DD084ACDF88A
:1066D00000803B46CAE70020D2E701207AE700BFEE
:1066E000C2B8323EC2B8B23E48630A0853630A08D1
:1066F0005F1A0A0858630A082DE9F743144605464D
:1067000088460193FFF710FE019A074638B92448DE
:10671000244B00682146C06A12F03CF9019A0192AC
:1067200021462846FFF70EFF064630B32846FFF7FE
:10673000EBFB95F80C33019A83420DD005F0D6F8A7
:1067400004F0D2FF019A38B1174B15480068214672
:10675000C06A12F01FF910E02846FFF7D5FB18B108
:1067600003280FD0114BF0E713464146224605F2AD
:106770003C4000F03BFF00B107B90026304603B0B3
:10678000BDE8F08395F86092B9F1000F01D1084B94
:10679000DBE7134641462246284619F031FBEAE77B
:1067A000685F00205C630A0868630A0898630A0847
:1067B00087630A0890F80C33032B01D119F06CBFE2
:1067C0000020704737B5054600F5067140F60332E4
:1067D00001A811F001FF2846FFF796FB044640B1DF
:1067E00003280AD0002401A811F018FF204603B0A6
:1067F00030BD284619F002FCF5E7284619F0FEFBEB
:106800000446F0E708B50246FFF77EFB10B1032807
:1068100006D008BDBDE8084002F23C4000F09CBE36
:10682000BDE80840104619F02DBF00000B4610B41B
:1068300011462BB1032B09D000205DF8044B7047A3
:106840005DF8044B00F23C4000F09CBE5DF8044B48
:1068500019F046BC13B50446FFF756FB0A4601463D
:1068600020460192FFF7E2FF70B9084B019A1B68BE
:10687000DB6A93F89C0038B194F80C13204602B000
:10688000BDE81040FFF7D2BF02B010BD685F002026
:1068900037B504460D4640F2B25200F5067101A824
:1068A00011F09AFE2946204619F038FC94F80C3372
:1068B000032B054610D148B104F583612046FFF74C
:1068C000C9FF84F82804204600F0DCFD01A811F07F
:1068D000A5FE284603B030BD0025F7E770B590F857
:1068E0007C32DB0786B004460D460CD402F0DCFF98
:1068F000437C242202FB0300D0ED0B7AF1EE677A91
:10690000C5ED007A3BE002A803F07EFF01A9204616
:10691000FFF7ECFAE8B90DF04DFD94F94432022B83
:106920000646E3D1FEF7F6FE0228DFD996F8F40218
:106930009FED147AB02303FB0066D4F87032D6F8CA
:10694000E0209B1A07EE903AF8EEE77A67EE877A36
:10695000D6E702A92046FFF77DFF0028DBD0D4F858
:106960007022039BDFED076A9DED017A9B1A07EE0B
:10697000903AF8EEE77AA7EEE67A85ED007A06B06F
:1069800070BD00BF0AD7233CF0B50C4687B000F5B8
:106990000671064640F6863201A811F01DFEA36876
:1069A00053B9E36843B9636833B9002701A811F00C
:1069B00035FE384607B0F0BD204604F02DF800281B
:1069C000F3D094E80F0002AD85E80F0000212846BF
:1069D00003F0E4FF07460028E7D096F87C32DB0797
:1069E00004D436F0CFFF192136F064FD95E80F008E
:1069F00006F51B7C8CE80F0096F87C3243F001030F
:106A000086F87C32304600F03DFD41F0F7F9462132
:106A100042F012F841F0F2F9452142F00DF8054B31
:106A2000A2681B68DB6A1A61E2685A6162689A614F
:106A3000BCE700BF685F002038B5144B1B68DD6AF7
:106A40002B6804465B6828469847F0B12B690BB960
:106A50006A69D2B1C4F874326B69C4F87832A96932
:106A6000002204F51B7003F0D5FE94F87C3223F06D
:106A7000030343F0030384F87C3241F0BFF9BDE81F
:106A80003840034A06213AF07DBB38BD685F0020DC
:106A9000AC630A0813B504460193FFF735FA0328DF
:106AA000019B05D1204602B0BDE8104019F0B4BBEF
:106AB000002002B010BD000010B588B00446059358
:106AC000FFF722FA0328059B4FF000000AD1069039
:106AD000079006A802900B9801900A980090204613
:106AE00019F0A8FB08B010BD38B50446FEF79AFCB3
:106AF0000546D0B194F80C33032B03D095F84E41E2
:106B0000204638BD204619F0A9FAFF280446F5D0E2
:106B100001462846FEF75AFC0028EFD021462846B9
:106B2000FEF750FC0028E9D0EAE70446E8E7000059
:106B300008B590F80C33032B05D014F0B1FC90F994
:106B40001203C0B208BD19F0CDF9431CF9D1F4E726
:106B500008B590F80C3383B1032B03D1BDE808408E
:106B600019F0B8B935F0FCF840F6ED424FF4801159
:106B700035F0AEF84FF0FF3008BD1846FCE70000D6
:106B800090F80C33032B01D119F0FCBF70470000C3
:106B900090F80C33032B01D119F080B87047000036
:106BA00019F006B910B504461CF078F82046FEF737
:106BB00041FC2046BDE81040FEF742BD90F80C3382
:106BC0000BB1032B01D11AF059B800207047000017
:106BD00030B500F5757304460D460FCB85E80F0000
:106BE00094F8E40330BD00007FB5054668460E46C4
:106BF00003F00AFE95F87C32DB0703D4002420461C
:106C000004B070BD69462846FFF7E2FF044600283D
:106C1000F4D0694605F51B7004F00EF886ED000A05
:106C2000C6ED010AEBE70000D0F880330B6090F866
:106C30007C037047D0F888330B6090F88503704769
:106C400010B500F5637203460C4607CA84E80700D6
:106C500093F8980310BD000030B500F56773044643
:106C60000D460FCB85E80F0094F8AC0330BD000053
:106C700030B500F5836304460D460FCB85E80F0061
:106C800094F8280430BD000010B500F22C420346F1
:106C90000C4607CA84E8070093F8380410BD0000CA
:106CA0002DE9F0432DED028B8BB005460E461746BD
:106CB000FFF71AFF014680462846FFF781FB04468E
:106CC000002848D0FEF7AEFB4146FEF781FB86ED7B
:106CD000000A95F93032002B3ADD0DF06BFBFEF720
:106CE00019FD012834D90DF065FB90F8F432D5ED8B
:106CF000DE7ADFED5D8A96ED000AB02202FB03002A
:106D000095F93032D0ED3B0A07EE103AF4EEE87A0E
:106D1000B8EEC77AF1EE10FAB7EE008AB8BFF0EE1F
:106D2000487A37EE201A20EE270A70EEC70A40F2A2
:106D3000B63015F08DF8D5EDDE7AF4EEE87AF1EEA6
:106D400010FAB8BFF0EE487A80EE277A86ED007A26
:106D500001233B7003E095F8083333B938702046BF
:106D60000BB0BDEC028BBDE8F08395F80C334FF00F
:106D70000009CDF80490CDF80890CDF80C9043B1FF
:106D8000032B10D0CDF81090CDF81490CDF81890BA
:106D90007CB902233B703246414605F23C4001F08B
:106DA000C9FB0446DBE701A9284619F04BF9044664
:106DB000E8E795F80C33002BEBD004A92846FFF741
:106DC00063FF04460028E4D001A904A817F06EF977
:106DD00007A8CDED080A8DED091A8DED070A17F009
:106DE00079FD04A8B0EE408A17F074FD95F93032B1
:106DF000002B30DD07EE903AF8EEE77A4FF47F7023
:106E000070EE670A37EE801AF5EEC00AF1EE10FA5E
:106E100048BFDFED160AF4EE410AF1EE10FAB0EECB
:106E2000480AC8BFB0EE601A15F012F8B0EE408AFA
:106E3000D5EDDE7A9FED0C7AF4EEC77AF1EE10FA1A
:106E4000B7EE007AB8BFF0EE477A88EE277A0323D0
:106E500086ED007A7DE7B5EEC08AF1EE10FA48BF04
:106E60009FED028AE4E700BF00000034000000004C
:106E700010B50446FFF75CFE84F80D032046FFF7CB
:106E800057FE84F80E032046FFF752FE84F80F03E6
:106E90002046FFF75DFE04F55A7184F81003204682
:106EA000FEF7F4FE84F8740300F00CFB04F5617245
:106EB00084EDDE0A04F560712046FFF7F1FE04F56B
:106EC000627184F87C032046FEF7FCFE04F56371D2
:106ED00084F885032046FEF729FF04F5677184F8DE
:106EE00098032046FEF734FF04F56C7184F8AC0378
:106EF0002046FFF7F5F904F5707184F8BC032046CD
:106F0000FFF7BCF904F5757184F8D0032046FEF74D
:106F100095FE04F57A7184F8E4032046FFF78EF9B4
:106F200084F8F8032046FEF73DFF04F5806384ED06
:106F3000FF0A2046C3ED000AFEF754FF04F20443A3
:106F400083ED000A04F2144204F581612046FFF744
:106F50007DFA04F583612046FFF77CFC04F22C41A6
:106F600084F828042046FEF75DFF84F8380410BD3D
:106F700037B50D46044600F041F91DB914F090FAFA
:106F800013F04CFA4FF4BE7204F5067101A811F02B
:106F900023FB94F869322BB92046FFF74DFD0123FE
:106FA00084F86932224B1D68A86A03689B69984778
:106FB0002046FEF787FD2046FEF700FE204600F043
:106FC00093FA2046FFF754F8286B30B10368D4EDEC
:106FD000D20ADB6894EDD10A9847D4F8100208B1C0
:106FE0005BF0D6FD204600F07DF82046FEF79AFFC4
:106FF00094F8903284F80C0383420ED084F8900207
:1070000098B10C4D0C4B032808BF1D4640F0F6FE0E
:107010000A4A2B4606213AF0B5F82046FFF728FF2A
:1070200001A811F0FBFA03B030BD054DEEE700BF3B
:10703000685F0020E7320A0853630A08C4630A083D
:1070400058630A08D0EDDE7A9FED057AF4EEC77A30
:10705000F1EE10FAB7EE000AA8BFB0EE670A70476B
:1070600000000034014B1868704700BF905F00209B
:107070004FF0FF307047000001207047704700005C
:1070800000207047002070477047000070470000E4
:107090000020704700207047002070470020704794
:1070A0000020704700207047002070470120704783
:1070B0000368D3F8943018470020704700207047C9
:1070C0000020704700207047002070470020704764
:1070D0000020704700207047002070470020704754
:1070E000704700007047000008B514F0D9F990F817
:1070F000130308BD08B514F0D3F990F8120308BDC6
:1071000030B52DED028B9FED1A1ADFED1A0A91EDC5
:10711000000A87B005462D200C468DED011ACDEDF5
:10712000000A14F095FE9DED011ADDED000AF0EE67
:10713000408A2E2094ED010A14F08AFE9DED011A7A
:10714000DDED000AB0EE408A2F2094ED020A14F023
:107150007FFE03A905F52570CDED038A8DED048A28
:107160008DED050A32F05CFD07B0BDEC028B30BD41
:10717000C2B8323EC2B832BE70B52DED048B00F5F8
:10718000257403460E4694E8070084B0D3EDA57A33
:107190009FED181A93EDA69A01AD85E8070030EE31
:1071A000270AF0EE608A3A20DFED130A14F050FE51
:1071B0003B20B0EE408A9FED0F1ADFED0F0A38EE4C
:1071C000890A14F045FE8DED018A8DED020A95E8DD
:1071D000070084E8070046B10021204604B0BDEC5A
:1071E000048BBDE8704030F05DBE04B0BDEC048B94
:1071F00070BD00BFC2B8323EC2B832BE10B5044640
:107200005AF058FDD4F8F4321BB1C21AB2F57A7FA5
:1072100012D30A4A1268D26A92F89C2002B15BB972
:10722000C4F8F40294F8314214F03AF980F80D43AE
:1072300004F05CFB80F8254010BD00BF685F0020B3
:107240002DE9F0432DED028B91ED007AD1ED037A1B
:1072500087B08DED047AB0EEC77AB5EEC07AF1EE64
:1072600010FADDE91087DDF84C90CDED057A0C467B
:1072700015461E4606DCF0EEE77AF5EEC07AF1EE32
:1072800010FA02DD04A816F093FE6B20B7EE001A88
:10729000FFEE000A9DED050A14F0DAFD6C2089ED81
:1072A000000AB7EE001AFFEE000A9DED040A14F082
:1072B000CFFD04A888ED000A16F0D6FDB7EE008ACF
:1072C000002852D00023C9F8003088ED008AD4EDA0
:1072D000067A67EEA77AF4EEC87AF1EE10FA4ADB86
:1072E0000023336085ED008ADFED3F0A96ED000A4A
:1072F0007C20B7EE001A14F0ABFD86ED000A95ED88
:10730000000A7D20B7EE001AFFEE000A14F0A0FD7F
:1073100085ED000AD4ED067A129BDFED346AF1EEBA
:10732000677AC3ED007A96ED007AF0EEC77AF4EE54
:10733000E67AF1EE10FA2BD503AB02AA01A920469A
:1073400015F0DEF99DED018AB0EE480A83F0D4FC19
:1073500085ED000AB0EE480A83F024FE87ED000AAE
:1073600007B0BDEC028BBDE8F08304A816F068FD01
:107370000028A7D1ABE738EE670A14F0C5FC86ED0C
:10738000000A94ED087AC7EE007AC5ED007AABE703
:1073900094ED076AC6EE077AC7ED007A96ED007A9B
:1073A000B0EEC77AB4EEE67AF1EE10FAC4D495EDF9
:1073B000007ADFED0F6AB0EEC76AB4EE666AF1EEEE
:1073C00010FAB9DCB4EE477AF1EE10FAB4D6B0EEAA
:1073D000E77AB4EE667AF1EE10FAADDCF4EE677A95
:1073E000F1EE10FABCD7A7E700000000000000345F
:1073F000FFFF7F7F1FB500F51773039300F516732A
:10740000029300F51573019300F51473009300F5D2
:10741000127200F5137300F54871FFF711FF05B004
:107420005DF804FB9FED156A90ED817ADFED146A3B
:10743000D0ED837A27EE067A67EE867A27EE267AF3
:1074400067EEA67ABDEEC77AFDEEE77A80ED7E7A2A
:1074500090ED827A27EE067A17EE903A27EE267A9A
:10746000002BB8BF03F50C43BDEEC77AB8BFA033FD
:1074700080ED7F7AC0F80032704700BFE02E654291
:107480000000C8421FB50E4B1B680446B3B16846E6
:1074900003F0BAF969462046FFF7EAFB20B16A46D5
:1074A00000212046FEF7A4F894F87C32DB0705D5CE
:1074B00004F51B7201212046FEF79AF804B010BDB6
:1074C0004062002008B502F0EFF9BDE8084001F085
:1074D0007DBD000010B580F8F81204465AF0EAFBB2
:1074E000C4F8FC0210BD000010B590F8F832044654
:1074F00053B15AF0DFFBD4F8FC32C01AB0F57A7FF2
:1075000084BF002384F8F83294F8003353B15AF062
:10751000D1FBD4F80433C01AB0F57A7F84BF0023BE
:1075200084F8003310BD000000F5AA700B4607C8B0
:1075300083E80700012070470023C0F89C30C0F8A2
:107540009830C0F89430C0F8A830C0F8A430C0F823
:10755000A030C0F8AC30704770470000024B0B60A1
:107560004FF07C53136070470000484270470000A2
:1075700008B50B4600F12801184615F04DFF012013
:1075800008BD000010B500F5B4700C460FC884E8C3
:107590000F00204603F028F930B1FFF763FD00F536
:1075A0001B700FC884E80F00204603F01DF980F01F
:1075B0000100C0B210BD000010B5044603F026FC67
:1075C000204610BD10B5D0F8603104465BB15AF0CA
:1075D00071FBD4F86031C01A41F28833984294BFED
:1075E0000020012010BD0120FCE7000013B500932E
:1075F00003680192D3F890309847DDE900210446F2
:1076000028B90448044B0068C06A11F0C3F9204649
:1076100002B010BD685F00205C630A0813B5044621
:107620000191FDF7FFFE2368019A1B6D014608B129
:1076300090F84E11204602B0BDE8104018470000F7
:1076400030B585B0002301930293039303680D4680
:10765000DB6D01A99847044620B1039B2B602046AF
:1076600005B030BD02F020F9417C01F0EBFD04468D
:107670000028F4D002F018F901F04AFDB1EE400AFA
:1076800085ED000AEBE7000090ED007ADFED0F7A60
:10769000B0EEC77AB4EEE77AF1EE10FA14D590EDB9
:1076A000017AB0EEC77AB4EEE77AF1EE10FA0BD5B4
:1076B00090ED027AB0EEC77AB4EEE77AF1EE10FA06
:1076C0004CBF0120002070470020704700000034AC
:1076D00010B5FDF7A7FE044658B190F84E11FDF71E
:1076E00071FE30B194F84E112046BDE81040FDF710
:1076F0006DBE002010BD000038B50D460CF05AFEDE
:107700000446FEF707F8022881BF94F8F402B0237C
:1077100003FB004000F5827089BF07C8002085E8A0
:107720000700012038BD00002DE9F0432DED028B4C
:107730008FB003680025DB6C0395049505950695CD
:10774000029502A904469847064638B1FFF7BAFEEB
:10775000DDED027A27EE800A8DED020A0CF02AFE9A
:10776000FDF7D8FF0746002E50D0DDED027AD4EDAC
:10777000646A94ED657A23680B9527EE877A67EE45
:10778000A67A8DED097ACDED0A7A0C950D959B6C54
:107790000BA9204609AD98470BA9284616F0BEFA5A
:1077A000012F8DED030ACDED040A40F2B3800CF0F9
:1077B00001FE90F8F432DFED5B7AB02505FB0300A3
:1077C00090ED3C8A28EE278AB0EE480A83F094FABE
:1077D000F0EE408AB0EE480A83F0E4FBCDED0B8A70
:1077E0008DED0C0A0CF0E6FD90F8F43205FB030079
:1077F00090ED3B0A0BA816F0B1FA09AD8DED050A24
:10780000CDED060A05A896BB03C885E00128CED8B1
:107810009DED020AB5EEC00AF1EE10FA7FDD07AE6B
:10782000D4F89421D4F8903107923046089316F09A
:10783000BFFA23680B950C950D959B6C0BA9204600
:107840009847DDED077A9DED0B7A77EE877A9DED0F
:107850000C7ACDED077ADDED087A77EE877A09AB01
:10786000CDED087A96E8030083E8030049E0236938
:1078700093ED000AB7EE008A38EE408A16F06EFAF1
:1078800004F5BC798DED090A4846B0EE480ACDED05
:107890000A0A16F063FA0BA92846CDED0C0A8DED05
:1078A0000B0A16F03BFA04F5C47603AFC4ED5F0A89
:1078B000314684ED5E0A384616F040FA04F5C07889
:1078C0008DED090A4046B0EE480ACDED0A0A16F0E1
:1078D00045FA0BA928468DED0B0ACDED0C0A16F0E2
:1078E0001DFA97E8030084ED600AC4ED610A86E89A
:1078F00003004946404616F011FA8DED090ACDED18
:107900000A0A9DED090ADDED0A0A0FB0BDEC028BF3
:10791000BDE8F083DDE9030185E80300F1E709959F
:107920000A95EEE735FA8E3C10B590F842130446FE
:1079300003F006FC7C23C0B203FB0044D4F8A00093
:1079400010BD0000044B026F1B68DB6A5A60426F77
:107950009A60826FDA607047685F0020F0B58FB080
:10796000044613F09DFD002302930393049390F8C3
:10797000121301AB02AA054612F0C6FD04F19407EA
:10798000D8B39DED010AB5EEC00AF1EE10FA34DD70
:1079900002A816F0B1FB04F1B00684ED2C0AC4ED88
:1079A0002D0A84ED2E1A3946304616F0B5FB04F147
:1079B0007C01304616F064FB04F1880105A88DEDCA
:1079C000050ACDED060A8DED071A16F059FB08A839
:1079D0008DED080A9DED010ACDED090A8DED0A1A1B
:1079E00016F07AFB0BA904F128008DED0B0ACDED02
:1079F0000C0A8DED0D1A14F02FFF95F812030C23CD
:107A000003FB0050394600F5117016F039FB84ED88
:107A10002C0AC4ED2D0A84ED2E1A0FB0F0BD000023
:107A20002DE9F047824B00251F682DED028BC0F831
:107A30009C50C0F89850C0F89450C0F88450C0F8DA
:107A40008050C567C0F89050C0F88C50C0F888507E
:107A5000C0F8B850C0F8B450C0F8B0500446F86A46
:107A600003688AB05B680E46984704F1280900282D
:107A700054D05AF01FF942F20F7398424ED8FB6A65
:107A80009FED6C8A93ED010A84ED1C0AD3ED020A86
:107A9000C4ED1D0A93ED031A484684ED1E1A14F036
:107AA000CFFD40F0ABF9D4ED1E7A67EE887A05463B
:107AB00017EE900AF8F728FDD4ED1D7A67EE887A64
:107AC000CDE9040117EE900AF8F71EFDD4ED1C7AFB
:107AD00067EE887ACDE9020117EE900AF8F714FDF7
:107AE000554ACDE900010621284639F04BFB94EDBB
:107AF0001E8AB0EE480A83F0FFF884ED650AB0EE06
:107B0000480A83F04FFA84ED640A5AF0D3F8C4F8B7
:107B100064010AB0BDEC028BBDE8F087A6B194ED1C
:107B20001C0AB4EE400AF1EE10FA0DD6D4ED1D0A8F
:107B3000F4EE600AF1EE10FA06D694ED1E1AB4EED9
:107B4000411AF1EE10FA52D713F0AAFC90F8133351
:107B50004FF00C0A0AFB030303F5C473074693E8CE
:107B6000070007AE86E807004FF01508B2EE028A5C
:107B7000F2EE068A304616F0ADFEB4EEC80AF1EE1B
:107B800010FA38D508F1FF3818F0FF083CD130461C
:107B900016F0A0FEF1EE047AB4EEE70AF1EE10FA68
:107BA00043DD9DED090ADDED087A9DED078A20EEA3
:107BB000000AA7EEA70A83F00BFCF0EE400AB0EE35
:107BC000480A83F0BBFADDED090A84ED1D0A9DED3C
:107BD000080AF1EE600AB1EE400A83F0AFFA84EDD4
:107BE0001C0A9FED161AD4ED1D0A94ED1C0A484696
:107BF00014F026FD7BE7304616F06CFEB4EEE80A82
:107C0000F1EE10FABEDCC2E7384612F03FFB384610
:107C100012F004FC97F813330AFB037303F5C473E3
:107C200093E8070086E80700A4E725676567D8E7BB
:107C3000685F0020E02E6542E4640A08000000004E
:107C40000021FFF7EDBE000037B504460846154693
:107C5000019116F03FFEB7EE007AC7EE007AB4F855
:107C6000D03001980133A4F8D03094ED337A37EE58
:107C7000277A84ED337AB0EE007AF4EEC77AF1EE2B
:107C800010FA06D5B6EE007AF4EEC77AF1EE10FAE5
:107C90000DDC9FED0E7AF4EEC77AF1EE10FA13D5F3
:107CA0009FED0B7AF4EEC77AF1EE10FA0CDDB0EE30
:107CB000670A16F011FA012085ED000AC5ED010AE8
:107CC00085ED021A03B030BD0020FBE700247449A3
:107CD000BD37863570B52DED028B00F1280600F119
:107CE00034058AB029460446304616F071FAB6EEDD
:107CF000008A20EE088A2846B0EE480A16F0ECF911
:107D000007A93046CDED080A8DED091A8DED070A59
:107D100016F0CCF930468DED010AB0EE480ACDEDF3
:107D2000020A8DED031A16F0D7F907A928468DED42
:107D3000070ACDED080A8DED091A16F0B7F904A966
:107D400001A88DED040ACDED050A8DED061A16F099
:107D500053FA324601A920468DED070ACDED080AF7
:107D60008DED091AFFF770FF58B959F0A3FF0121F3
:107D7000C4F860012046FFF753FE0AB0BDEC028B49
:107D800070BD2A4604A92046FFF75EFF0028ECD00C
:107D900004F1400207A92046FFF756FF0028E4D06F
:107DA000EBE7000030B52DED028B0D4683B091F866
:107DB00042130446284603F0C3F9C1B27C2000FBFD
:107DC0000151903104F1280014F0CAFA68468DED93
:107DD000000ACDED010A16F06DF8DFED1C7AB4EE65
:107DE000E70AF1EE10FA05D59FED190A03B0BDECD4
:107DF000028B30BD684616F0DBF8684616F034F8A2
:107E00000028F1D1284694ED428A03F0FDFAF0EE05
:107E1000400AB0EE480A13F043FF80B9284603F049
:107E2000F3FA84ED420AB0EE408A82F065FF84EDF9
:107E3000430AB0EE480A83F0B5F884ED440A04F52D
:107E40008671684615F0DEFFD0E700BF0000003401
:107E5000000000009FED0C7AB4EEC70AF1EE10FAB4
:107E60000BD4DFED0A7AB4EEE70AF1EE10FA07DC84
:107E7000C0EE077AB0EE670A7047F7EE007AF9E7CE
:107E8000F2EE047AF6E700BFF3665F3F58A00B41BD
:107E900008B51C3016F00EF8F1EE007AB4EEE70AE1
:107EA000F1EE10FA9DBFF1EE027A37EEC00ADFED77
:107EB000047A9FED040A98BF20EE270A08BD00BF90
:107EC000CDCC4C3ECDCCCC3D08B5836993F90000B8
:107ED00038B10CF06FFAFDF71DFC012894BF0020AB
:107EE000012008BDF8B52DED028B054603F0FEFC20
:107EF00003F0FAFB0446B8B3FFF7B4F890F809337F
:107F000093B32846FFF7E0FF064668B30CF052FA39
:107F100090F8F432B02707FB030090ED3B7AF0EEC7
:107F2000087AB4EEE77AF1EE10FA1DD495ED1E8AC8
:107F30000CF040FA90F8F432DFED1E7A07FB0300F4
:107F400090ED3C0A98EE270A13F02EFFDFED1A7A27
:107F5000B0EEC00AB4EEE70AF1EE10FA08DC59F010
:107F6000A9FE3446C5F85001BDEC028B2046F8BD91
:107F700005F5AA7016F0AEFCB0EE408A0CF01AFAC5
:107F800090F8F4329FED0D7A07FB0303D3ED3B7AB3
:107F900067EE877AB4EEE78AF1EE10FADFD559F092
:107FA00089FED5F85041001BB0F5FA6F8CBF002454
:107FB0000124D9E7E02E654200003442CDCC4C3F8D
:107FC00010B50A4B1B68DB6A93F89C3004465BB91A
:107FD00059F070FED4F86431C01A44F61F63984219
:107FE0008CBF0020012010BD0020FCE7685F00204E
:107FF000F8B52DED068B04460CF0DCF9054603F0D0
:1080000075FC064606F0ACF9002840F0AB8020462F
:10801000FFF768FF002800F0A8803046FFF784FCD7
:10802000D4F8DC30984200F01A813046FFF77CFC2F
:10803000D4F8DC30DFED8F7AC31A08EE903AF8EE10
:10804000688A304668EEA78AFFF76EFC94F8BC3069
:10805000C4F8DC00F3B9304603F058FBD0B104F1AA
:10806000280796F842233946304603F0D1F9D4ED7B
:108070001D0AB0EE401A384694ED1C0A14F0E0FADE
:108080000023C4F89030C4F88C30C4F88830012341
:1080900084F8BC3020463146FFF784FE95F8F402A0
:1080A00005EB0015B0EE408AD5F8A030C4F8E030FA
:1080B00004F1B000D4ED129A16F00CFC6368DFED09
:1080C0006E7A93ED007AB4EEE77AF1EE10FA68EE8C
:1080D000299AB0EE40AA01D5C3ED007A2046B0EE51
:1080E0004A0AFFF7B7FE636820EE299A93ED000A6B
:1080F00029EE009AFFF7CCFE29EE009A204684ED87
:10810000249AFFF75DFF38B1D4ED247AB2EE007AFD
:1081100067EE877AC4ED247AF0EE007AF4EEE78A0F
:10812000F1EE10FA10D5DFED557AB4EEE7AAF1EED4
:1081300010FA09D5DFED527A69EEA79AD4ED2A7AC2
:10814000E9EEA87AC4ED2A7A9FED4E0A94ED367ACC
:10815000DFED4D7AB0EEC88A28EE008AA7EE278AB6
:1081600084ED368ABDEC068BF8BDFEF77BFF90F8F8
:108170000933002B73D02046FFF7A6FE00286ED0EF
:1081800095F8F42205EB0213D3F8A010D4F8E030F0
:108190008B4264D0B02606FB025292ED3B7AF0EEA1
:1081A000087AB4EEE77AF1EE10FA58DBCB1AC4F88D
:1081B000E01008EE903A95F8F4329FED341A94ED01
:1081C0001E0ADFED337A06FB0353D3ED3C9A69EECA
:1081D000819AF8EE688A39EEC00A68EEA78A13F031
:1081E00023FEB0EE409A82F0DDFE94F8BC30B0EE93
:1081F000408AF3B1F3EE047AF4EEE78AF1EE10FA76
:1082000017DC95F8F40206FB005595ED3B7AF2EE8B
:10821000027AB4EEE77AF1EE10FAFFF649AFDFED3D
:108220001D7AB0EEC99AB4EEE79AF1EE10FAFFF6B5
:108230003FAF9FED198AD4ED1D0A94ED1C0AB0EEF4
:10824000691A04F1280014F0FBF9012384ED248A53
:1082500084ED238A84ED228A84F8BC3028E7BDECC3
:10826000068B04F188009FED0D0ABDE8F84015F07B
:1082700087BF00BFBD378635CDCC4C3DC2B8B23EBE
:108280000AD7233CCDCC4C3ECDCC4C3F35FA8E3C6E
:108290006F12833A1904863F00000000EC51783FCA
:1082A00030B50C2303FB010101F1C003144693E830
:1082B00007008BB004AD85E8070094E8070083E869
:1082C00007002846FFF7E0F907AB58B194E807002C
:1082D00083E807009DED070ADDED080A9DED091A08
:1082E0000BB030BD95E80700F2E70000F0B52DEDCA
:1082F000028BD0F818318B60D0F81C31CB6085B080
:1083000004460D4601F0D0FA06460CF053F8A36976
:1083100093F90030022B07464BD1FDF7FBF90228F9
:1083200047D997F8F432B02202FB0373D3F8E01078
:108330000022284602F06EFAD4ED4A0A94ED490A6A
:10834000284602F04FFD94F82C3163B359F0B2FC8B
:108350009FED228A97F8F4128DED018A01AA064654
:1083600038460BF0ABF8D4F820019FED1D0A361A01
:1083700007EE906AF8EE677A4FF4876027EE800A7E
:10838000B6EE001AF0EE480A13F062FDDDED017A58
:1083900030EE270A04F1F0008DED010A15F0DEFC45
:1083A000284602F01FFD94F82C0105B0BDEC028BAD
:1083B000F0BD707C242303FB006696ED0B8AFEF76C
:1083C00051FED0ED9C7A9FED077AF8EEE77AE8EE61
:1083D000077AFDEEE77A17EE901AA9E70000000091
:1083E0006F12833A0000C842F8B5036F0B60436F09
:1083F0004B60836F8B6000F14C050E46074601F120
:108400000C040FCD0FC40FCD0FC42B68236007F1F0
:10841000B00207CA06F1300383E8070007F19402AF
:1084200007CA06F13C0383E8070007F11C0207CAEC
:1084300006F1480383E8070006F160013846FFF7BC
:1084400055FF86F87000F8BD30B589B0044668461F
:108450000D4602F0D9F969462046FFF793F818B99E
:108460000024204609B030BD04A802F0CDF9204612
:1084700004A9FFF73BFF04460028F1D004A9684691
:1084800002F008FC85ED000AC5ED010A85ED021A2F
:10849000E7E700001FB500230C4601A901930293F2
:1084A0000393FFF7D1FF08B1039B236004B010BD15
:1084B00030B585B001AD00230C46294601930293E7
:1084C0000393FFF7C1FF034618B195E8030084E862
:1084D0000300184605B030BDF8B506460F461546F0
:1084E000FCF7A0FF044690B13946FCF76BFF70B172
:1084F00020463946FCF76AFF044640B1FCF792FF7C
:108500003946FCF765FF85ED000A2046F8BDFEF709
:10851000A9FD90F8083343B13046FFF7D5FC044677
:1085200018B1D6F84C312B60EFE7D6F84C312B6000
:108530000024EAE770B52DED048B1646FFF7CCFF5B
:10854000054670B3FEF78EFD90F930424CB30BF048
:1085500031FFFDF7DFF8012823D9E4B207EE904A96
:10856000B8EE678A0BF026FF90F8F43296ED009A89
:10857000B02202FB0300D0ED3B8AFEF7A3FF38EEEA
:10858000281A78EEC80A40F2614029EE000A13F07A
:108590005FFCB0EE408AFEF795FFC8EE007AC6EDAC
:1085A000007ABDEC048B284670BD000008B503F0CE
:1085B0009DF9BDE8084003F097B8000010B50446E7
:1085C00015F036FE50B904F10C0015F031FE28B953
:1085D00004F11800BDE8104015F02ABE012010BDBE
:1085E00038B500F1280504462846FFF7E7FF28B113
:1085F00020460121BDE83840FFF712BAD4ED107AC9
:10860000B7EE007AF4EEC77AF1EE10FA06D5BFEEB7
:10861000007AF4EEC77AF1EE10FA12DC2046FFF78A
:1086200059FB2846FFF7CAFF0028E1D1D4ED107AA4
:10863000B2EE047AF0EEE77AF4EEC77AF1EE10FAD1
:10864000D6DC38BD10B5044616F044F92046BDE826
:10865000104015F0A9BD00002DE9F04F2DED048B61
:108660009FEDC98A95B00446F0EE408A8DED028AEE
:108670008DED038A8DED048AFFF7BAFC12F010FF2E
:108680000023054695F87921012AA8BF01229342CB
:108690003FD20021284611F065FD01230028F1D0CA
:1086A00008AB0BAA002128468DED0B8A8DED0C8AB4
:1086B0008DED0D8A11F082FF9DED080AB5EEC00A1E
:1086C000F1EE10FA23DD0BA815F016FD11A904F147
:1086D00028008DED110ACDED120A8DED131A13F05D
:1086E000E3FD0EA88DED0E0AB0EE680ACDED0F0A7F
:1086F0008DED101A15F0F0FC11A904F1E4008DEDD8
:10870000110ACDED120A8DED131A15F005FD0123A6
:10871000B8E795F813130C2303FB015104F1280B60
:1087200001F5C471584613F0BFFD84ED070A94EDBE
:108730003F0AC4ED080A70EE288A84ED091AC4EDD8
:108740003F8A0BF037FE0646FEF78CFC90F80933A3
:1087500001932046FFF7B8FB80B13046FCF7DAFF03
:1087600002280BD996F8F4226169B02303FB026357
:1087700091F9001093F8020188425FDA94ED3F7A94
:10878000DFED827AB4EEE77AF1EE10FA5ED4D4ED42
:10879000538AFEF79DFF38B1FCF744FE90F84E1166
:1087A000FCF716FEF0EE408A236C626BA16A13930D
:1087B000B0EE680A11A81292119115F08DFC04F523
:1087C000AA7102A88DED020ACDED030A8DED041AFF
:1087D00015F0A2FC59F06EFA0023074684F8143114
:1087E0002046FFF771FB002867D096F8F422B021ED
:1087F00001FB0262D2F8E430C4F8183196F8F43282
:1088000001FB0363D3F8E830C4F81C3159F052FA85
:108810000123C4F8200184ED498A84ED4A8A84F852
:108820002C31D4F80031002B5AD102AB93E8070069
:10883000C4F80071F03484E8070007E006EB021288
:10884000D2F8A070D4F80021BA4204D115B0BDEC22
:10885000048BBDE8F08F03F5827393E8070094F86A
:1088600014310DF1080C8CE807001BB904F1F0037A
:1088700083E807000123604684F8143104F5AA71E7
:1088800015F014FC11A904F14C008DED110ACDED89
:10889000120A8DED131A13F035FDB5EEC00AF1EE94
:1088A00010FA8DED110AD8BF9FED370ACDED120AEF
:1088B0008DED131A84ED530A92E794ED3F7AD4EDCF
:1088C000497ADDED026AE6EE877ADDED036AC4EDF2
:1088D000497AD4ED4A7AE7EE267AC4ED4A7AA0E7DF
:1088E000D4ED3F7A254B8DED058AF5EEC07AF1EE99
:1088F00010FA8DED068A0793A8D9214B9FED217AB6
:108900001B68DB6A67EE877A93F89CA0B7EE007A63
:10891000C7EE279ABAF1000F4AD094F8143113B970
:10892000019B002B42D0E36804F1F001D3ED008AF3
:1089300002A815F0BBFB69EEA88A8DED110A11A8FB
:10894000B0EE680ACDED120A8DED131A15F0C4FBD6
:108950000EA905A88DED0E0ACDED0F0A8DED101AAA
:1089600015F0DAFB05A8FFF76DFE05A815F07AFCF7
:10897000F0B159F09FF9C4F8600167E7000080BFCB
:10898000685F00200AE81C4100000000CDCC4C3E8E
:10899000CDCC4C3FCDCC4C3D920A06BF920A063F4F
:1089A000C2B8B23E728A0E3C5B821839DDF804A070
:1089B0005FED0B8A0023CDE90833CDE90A33CDE919
:1089C0000C334FF0FF32009204F1E40895F879215E
:1089D000012A1046A8BF0120834255D20123002A54
:1089E000FAD095F835130029F6D0B0EE690A404662
:1089F00015F0C6FB0DF12C09BAF1000F3FD042462D
:108A000000212046FFF74CFC8DED0B0ACDED0C0A42
:108A10008DED0D1A4846FEF737FE70BB4846FFF74E
:108A200011FE484615F01EFC38BB05A9484615F056
:108A3000E3FB05A94846CDED090A8DED0A1A8DED37
:108A4000080A15F0C5FB08A8B0EE409A15F042FFE1
:108A5000009B33B9F4EEC08AF1EE10FAD8BFB0EE45
:108A6000680AB5EEC09AF1EE10FAF7EE008A4FF000
:108A7000000358BFF0EE408A00930123A6E798E870
:108A8000070089E80700C5E7009B002B7FF471AF62
:108A9000002384F804312046FFF724FA38B1204639
:108AA000FFF712FA002840F025818DED0A8A95F82B
:108AB000123395F878219A4240F233812B4493F88F
:108AC0003433002B00F02D8195F8133395F879217C
:108AD0009A4240F226812B4493F83533002B00F064
:108AE000208108A9584613F00DFC8DED080ACDED44
:108AF000090A8DED0A1A08A815F09AFB002840F023
:108B0000178108A815F0AEFB002840F011815FED39
:108B1000617A94ED357A68EEA78A5FED637AE7EEC5
:108B2000278A04F1B000C4ED358A15F0D3FEA3689E
:108B30005FED687A93ED007AB4EEE77AF1EE10FA21
:108B4000F0EE408A00F1F8802046B0EE680AFFF7A8
:108B500081F908A815F0C0FAA3688DED110ACDEDD2
:108B6000120A8DED131A93ED000A11A815F0B4FA4C
:108B7000204684ED1F0AC4ED200A84ED211AFFF778
:108B80001FFA28B1B2EE000A04F17C0015F0F8FAE1
:108B9000019BB3B33046FCF7BDFD012831D996F8EF
:108BA000F402B02303FB006696ED3B7AF0EE087A00
:108BB000B4EEE77AF1EE10FA23D595F813030C23FF
:108BC00003FB005595ED627AF1EE0C7AB4EEE77A8C
:108BD000F1EE10FA15DBD4ED1D7A1FED917AF4EE6B
:108BE000C77AF1EE10FA0CDD1FED947AF4EEC77A35
:108BF000F1EE10FA05D5B6EE000A04F17C0015F08E
:108C0000BFFA5FED997AF4EEE78AF1EE10FA22D519
:108C10001FED9C0A08A815F05FFA0EA88DED0E0A4C
:108C200094ED3F0ACDED0F0A8DED101A15F054FAB0
:108C300011A904F1A0008DED110ACDED120A8DED00
:108C4000131A15F069FAD4ED2B7A94ED3F7A77EE8A
:108C5000877AC4ED2B7A94ED2B7AF1EE047AB4EE98
:108C6000E77AF1EE10FA3BDB12F01AFC5FEDB27A14
:108C700094ED2B1A94ED280A21EE271A40F2C53004
:108C8000F1EE410A8DED011ACDED000A13F0E0F886
:108C90009DED011ADDED000A84ED280A40F2C63090
:108CA00094ED290A13F0D4F89DED011ADDED000AC8
:108CB00084ED290A40F2C73094ED2A0A13F0C8F86F
:108CC00004F1A00184ED2A0A04F1940015F024FABD
:108CD00084ED2A8A84ED298A84ED288A84ED2B8A02
:108CE0000023C4F8E430C4F8E830C4F8EC3084ED74
:108CF0003F8A9AE5E368F7EE000A93ED000A12F066
:108D0000CFFF00283FF4D1AE94ED1C0AB0EEC00AAC
:108D100082F048F9DDED0A7A27EE800A8DED0A0A25
:108D2000C5E68DED0A8A8DED098A8DED088AE2E6A9
:108D30002046FFF755FC1CE6C3ED007A04E700BFB0
:108D40002DE9F04D2DED048B9EB0044612F0A8FBEA
:108D5000D0EDC87A90ED618AF4EE487AF1EE10FA1F
:108D600048BFB0EE678ADFED5C7AB4EEE78AF1EED9
:108D700010FA0EDD0023C4F8E430C4F8E830C4F87B
:108D8000EC300023C4F8FC301EB0BDEC048BBDE811
:108D9000F08D2046FEF7E2FD2046FEF79BFFB0EE89
:108DA000480A2046FFF758FC2046FFF719FCFEF75B
:108DB00059F914AD00F5347204F1280114A813F028
:108DC000F1FA0FCD04F14C060FC60FCD0FC62B687C
:108DD000336004F1740204F1780304F1700104F1CA
:108DE0004C0013F08DFC94ED1E8AB0EE480A81F021
:108DF00083FF84ED650AB0EE480A82F0D3F820467E
:108E000084ED640AFEF79EFDFEF72CF904F5B471BB
:108E1000FDF72EFF58F04EFFD4F89831C31A632B9C
:108E2000B2D9C4F8980134F0ADFD9FED2C9A0546F7
:108E300058F048FFD4ED1C7A67EE897A074617EEA2
:108E4000900A0E46F7F760FBD4ED1D7A67EE897A3B
:108E5000824617EE900A8B46F7F756FB94ED1E0AF2
:108E600020EE090A41EC180B12F088FFD4F85C01DF
:108E700010EE108AF7F748FBCDE91201D4F858013B
:108E8000F7F742FBCDE91001D4F85401F7F73CFBAA
:108E9000CDE90E01D4F8D800F7F736FBCDE90C0187
:108EA000D4F8D400F7F730FBCDE90A014046F7F7D4
:108EB0002BFB0B4B01930B4B0093CDE908018DED80
:108EC000068BCDE904ABCDE90276074B074A08498A
:108ED000284634F099F957E7CDCC4C3EE02E654258
:108EE00043450A0849650A0810650A081A650A0810
:108EF00058630A0808B52DED048BB0EE609AF0EEC9
:108F0000408A00F011F9B0EE408A89EE280A82F01A
:108F10007FF9DFED0B7A20EE270A82F011F9DFED01
:108F2000097A38EE278ADFED087A28EE278AF7EEED
:108F3000007A37EEC00A28EE000ABDEC048B08BDAB
:108F400041D3423E33938843A1D81943FFF7D2BFA0
:108F500008B52DED048B9FED189AF0EEE07AF4EE53
:108F6000C97AF1EE10FAF0EE408AB0EE608A1ED4B3
:108F700000F0DAF8DFED117A9FED117A70EE277AC2
:108F80009FED100AE8EEC77A9FED0F7A27EE800A70
:108F9000C8EE007A87EE270AB4EEC90AF1EE10FA9D
:108FA00005DBBDEC048BBDE8084082F011BABDECD6
:108FB000048BB7EE000A08BD0000003433938843E9
:108FC000F4FDD43B48A18F43CDCC9C3F427CD0EDF7
:108FD000257A242101FB020292ED0B0AD2ED090A47
:108FE00030EE270AFFF7B4BF38B52DED088BDFED63
:108FF00021AA9FED21AA9FED21BA0546B0EE409A25
:10900000F0EE609AB0EE408A1524013CA4B25CB345
:10901000F0EE490A2846B0EE480AFFF76BFFF0EE83
:10902000490A70EE698A284638EE2A0AFFF762FF7D
:10903000B0EEE87A70EE697AB4EECA7AF1EE10FA20
:1090400077EEE87A10D468EEAA8A40F2631088EED0
:10905000A70AB0EE4B1A38EE400AF0EE4A0A12F0B8
:10906000F7FEB0EE408AD0E7B0EE480ABDEC088BC0
:1090700038BD00BFCDCCCC3D0AD7233C0024744979
:10908000002343608360C360036143618361C36104
:10909000002380F82030704790F82020531CDBB26A
:1090A000062B80F8203000EB820288BF002382ED7F
:1090B000010A88BF80F82030704700004FF0FF336E
:1090C00010B543610E4BC0F8A8300023044680F869
:1090D000C830A830FFF7D4FF0A4BC4F8A83004F515
:1090E000867057F09BFC084B08491C6020462FF007
:1090F000ADFED4F89030C4F89430204610BD00BFC7
:1091000064670A0874670A08945F00200C680A08FC
:1091100008B5A83036F006FDDFED027A20EE270A0A
:1091200008BD00BF00007A4490ED3C0ADFED057AEF
:10913000B0EEC07AB4EEE77AF1EE10FA48BF90EDE7
:109140003D0A70470000003473B5D0F8A4300446DF
:109150000E4663B158F0AEFDD4F8A430C01A42F206
:109160000F73984203D894ED280A02B070BD114BDA
:109170001D687DB195F84E112846FCF727F948B1D6
:1091800095F84E1101AA2846FCF716F910B19DED8D
:10919000010AEAE7242101FB064494ED0A0ADFED07
:1091A000067AB4EEE70AF1EE10FA58BFB0EE670A9D
:1091B000DBE700BF8C5F002000000C4208B561B106
:1091C0000378022B02D9064858F042FD5A1C02705F
:1091D00000EB83004160012008BD0846FCE700BFAA
:1091E0002C660A082DE9F84305460E4691460024F0
:1091F00000F13C082B78A34211DD00234A4631469A
:1092000001200FF05DF8242363430746002158F83E
:1092100003000FF065F8874204D00134EAE700202C
:10922000BDE8F8830120FBE7054B1B682BB14169C2
:109230004A1C02D0184634F0CBB90020704700BF5A
:109240004062002002290BD8242303FB010191F87E
:10925000390030B191F83A0018B191F83B007047ED
:10926000002070472DE9F047044658F023FDD4F85C
:10927000F86042F21073861B9E4288BFC4F8F80063
:1092800000274FF0240942F2107A237CFDB2AB4252
:109290001CD929462046FFF7D5FF70B109FB0548C8
:1092A00098ED0D0AD8ED097AD4ED250A30EE270A9B
:1092B0002046FFF799FE88ED0C0A564504D909FBB4
:1092C000054030302FF09AFF0137DEE7617C204601
:1092D000FFF73AFF84ED3D0ABDE8F08770B504461C
:1092E00086B058F0E7FCD4F89830C31AB3F57A7F0B
:1092F00005464FD3344B94ED257A1B68DFED336A76
:10930000DB6AD4ED247A93F89C60B0EEC76AB4EEC1
:10931000E66AF1EE10FA32D5B0EEE76AB4EEE66A2C
:10932000F1EE10FA2BD502A801F06EFA96BBFDF70C
:1093300099FE02A9FDF79CFC60B3DDED037A9FED79
:10934000247AF8EEE77A67EE877AC4ED257AC4F8D6
:109350009850FDF787FEFDF735FA2046FFF782FFAC
:109360003EF04CFD0546D4F89400F7F7CDF8194AC5
:10937000CDE900010621284637F004FF0AE037EE68
:10938000676AF7EE005AB0EEC66AB4EEE56AF1EE2F
:1093900010FA01DC06B070BDB0EEE76AB4EEE66A22
:1093A000F1EE10FAF6D4002ECFD02046903080EDAA
:1093B000007A2FF023FF3EF021FD074A012106B07D
:1093C000BDE8704037F0DEBE685F0020000000346A
:1093D0000AD7233C6D660A0848660A08F0B52DEDE9
:1093E000048B85B004464FF4537200F5867103A8D0
:1093F0000FF0F2F8D4ED227AD4ED236A9FED796A6A
:10940000637C37EEE67A2422B0EEC77AB4EEC67AF1
:10941000F1EE10FAC1BF9FED747A67EE877A9FED87
:10942000737AE6EE877A02FB03430025C4ED237AC4
:1094300093F839602378E9B28B4206D904EB8103B3
:10944000013558685AF0C2FDF4E7DFED698A9FEDF7
:10945000698A9FED699A0027237CFDB2AB4264D9EB
:10946000242303FB054393F83920002A5BD0D3ED76
:109470000C7AF4EEE87AF1EE10FA0BDBF4EE677A90
:10948000F1EE10FA06D6F0EEE77AF4EE487AF1EE55
:1094900010FA04DD242303FB05435A6A1A632423CC
:1094A00003FB0543D3ED090AD3ED0D7A93F8382079
:1094B00070EEA70AA2B993ED0C0A2046FFF746FD0D
:1094C000D4ED257A30EE670AB4EE400AF1EE10FAD8
:1094D00016D7242303FB0545002385F83A3022E004
:1094E000012A09BFD3ED0C7A93ED0B0A77EEE00A5F
:1094F000D4ED3B7A04BF80EE897A87EE270AE3E752
:10950000F0EEC07AF4EE487A2423F1EE10FA03FB71
:109510000545E1DC012385F83A30D4ED237A37EEB6
:10952000800A85ED0B0A013796E7627C20461146DA
:10953000FFF788FE48B1242101FB024292ED0B0A9D
:10954000D16904F1A80036F0CDFA94F99C10277C7B
:10955000002907DBB94205DACAB211462046FFF7F7
:1095600071FE68B900226274D5B2AF4209D92946AA
:109570002046FFF767FE01320028F5D0657400E051
:1095800062742046FFF7AAFE2046FFF74DFE10B199
:1095900020465BF023FD637C242505FB034393F801
:1095A0003930B34216D034F0EDF94FF6FF7134F094
:1095B0000FF878B1607C05FB004494F83930002B3B
:1095C00014BF00220422019234F0DCF9019A122126
:1095D00033F090FF03A80FF021F805B0BDEC048B29
:1095E000F0BD00BF0AD7233C0AD7A33C48E17A3F2D
:1095F00000000034FFFF7F7F002019462DE9F04F67
:109600000446007C0F4687B004F13A030022012192
:10961000D5B2A84203F1240305D903F8231C03F8AB
:10962000241C0132F4E76F4B1E68F06A03685B6824
:10963000984740B13EF0E2FB6B4A062107B0BDE817
:10964000F04F37F09FBD3EF0D9FB684A062137F056
:1096500099FD002303A904F18800039330F092F9E7
:109660000A2558F027FB80462046FFF7B7FE58F042
:1096700021FBA0EB0800B0F5FA7F02D95C4801F0AD
:10968000A1F8B06A03680A215B689847617C2046AC
:10969000FFF7D8FD0028E7D0B06A036864215B6853
:1096A000013D984715F0FF05DBD1524B05951B880E
:1096B0008DF80650CDE90355ADF80430052558F076
:1096C000F9FA80462046FFF789FE58F0F3FAA0EB3E
:1096D0000800B0F5FA7FD1D8617C2046FFF7B2FDD3
:1096E0000028EFD094F810B00DF10C08A14601AAA3
:1096F0004FF0000A5FFA8AF18B4516D92046FFF732
:10970000A1FD50B1D8ED007A99ED097A137877EE82
:10971000877A0133C8ED007A13700AF1010A08F163
:10972000040809F124090132E4E7B06A03686421FE
:109730005B68013D984715F0FF05C0D1A9464FF081
:109740002408237C5FFA89F6B34226D906AB33445A
:1097500013F8143C33B908FB064686F83B3009F190
:109760000109EEE7002FFAD007EE903A06AA02EBC5
:109770008602F8EEE77A12ED030AD4ED250A2046B8
:1097800080EE270AFFF730FC08FB064002A93030C4
:109790008DED020A30F0F6F8E1E7617CDFF85C90CD
:1097A0002046FFF7D1FC002684ED3D0A4FF0240847
:1097B000237CF7B2BB420FD908FB074393F83B3039
:1097C00043B13EF01BFB7B1C4A46062137F0DAFC16
:1097D0000135EDB20136EBE70DB907484FE707B0A9
:1097E000BDE8F08F685F002088660A08B3660A0843
:1097F000C9660A0844170A0805670A08E3660A08E2
:1098000008B5037C022B02D9034858F021FA5A1CF0
:109810000274184608BD00BF24670A0838B5057CE5
:1098200002460024E1B28D4206D91046FFF70AFD38
:1098300001340028F6D138BD281E18BF0120FAE7F0
:1098400070B50D4609780729044606D8027E437E86
:1098500022B901228A401343437670BD002BFCD00D
:1098600000262278F3B29A42F7D904EB8303294603
:1098700058680368DB6898470136F2E737B50D464C
:109880000192FFF7CBFF0199044630B90448054B1C
:1098900000682A46C06A0FF07DF8204603B030BD4C
:1098A000685F00200B7B0B08014B1868704700BFF6
:1098B000945F002010B50446006810B103685B682F
:1098C0009847204610BD000013B500220B680A60BF
:1098D00001A901935AF0CAFE044601A8FFF7EAFF66
:1098E000204602B010BD000013B500220B680A60CC
:1098F000022201A901935CF0A5F8044601A8FFF734
:10990000D9FF204602B010BD13B500220B680A60D3
:10991000012201A901935CF095F8044601A8FFF724
:10992000C9FF204602B010BD13B500220B680A60C3
:1099300001A901935CF086F8044601A8FFF7BAFF7D
:10994000204602B010BD000010B50446006810B1FA
:1099500003685B689847204610BD00002DE9F04F72
:109960008FB0D0F800310893344B354D1B68059308
:109970000446586803689B68984794F99D300690A0
:10998000002BA2BF012606FA03F3069305F1D80ABD
:109990002B68089A1A420BD000274FF0010BB946EA
:1099A000069A0BFA07F3134206D10137202FF7D19D
:1099B0000C355545ECD12DE0F9B26B682A7A099146
:1099C00020460793FFF70EFC0999804628B3CDE99E
:1099D0000A990B9B0D930DA9079BCDE90B99204686
:1099E000984701462046FFF7E9FB0DA8FFF762FF05
:1099F0000CA8FFF75FFF0BA8FFF7A6FFB8F1000F59
:109A000002D00AA8FFF7A0FF2378032B02D0237C03
:109A1000032BCAD10FB0BDE8F08F059B5868042214
:109A20000368CDE90182074A00921B680A461E4678
:109A300001462B7A0BA8B047CBE700BF685F002038
:109A4000FC680A08801A060070B5D0ED247A9FEDF4
:109A5000657AF0EEE77AF4EEC77A0123F1EE10FAB8
:109A60008AB00446037609D49030002309A90590F2
:109A700009932FF087FF05982FF0C0FB0026E663BF
:109A80002666C4F88460762231462046FFF7AAFB9A
:109A9000054600283FD0CDE90666079A09920023C3
:109AA00009A92046CDE907335CF01EFB014620469C
:109AB000FFF784FB09A8FFF7FDFE08A8FFF7FAFEF1
:109AC00007A8FFF741FF15B106A8FFF73DFF237870
:109AD000032B59D0237C032B56D094F99D100029D9
:109AE00028DA2046FFF73AFFD4F80031DA045DD4D3
:109AF0000025637EEB40DB07EAB25DD40135082D1B
:109B0000F7D1237823B1237C13B16368002B3BD1B9
:109B1000354800F057FE354B1B68596804220B6826
:109B2000CDE90102324A00921E680246762307A858
:109B3000B047B2E77722C9B22046FFF753FB05468C
:109B400020B30023CDE90633079B0993002209A91E
:109B50002046CDE907225BF075FF01462046FFF75E
:109B60002DFB09A8FFF7A6FE08A8FFF7A3FE07A88C
:109B7000FFF7EAFE15B106A8FFF7E6FE2378032BF0
:109B800002D0237C032BACD10AB070BD174B1B68ED
:109B9000596804220B68CDE90102154A00921E683B
:109BA00094F89D20772307A8B047CDE7637E002B6C
:109BB0009ED1012363769BE73820059201F01EF9C0
:109BC000064618B1059A21465BF0DAFF3146204679
:109BD000FFF7F4FA2378032BD6D0237C032B8DD107
:109BE000D2E700BF0000003438670A08685F002031
:109BF000801A060090F86035934207D902F5A772E3
:109C000050F8220010B103689B6A18470020704783
:109C10002DE9F34105466E4686E80C00134B45F8E6
:109C2000043B04460F4600F5C87828462C3500F062
:109C3000CFFCA845F9D196E8030004F26453C4F8B8
:109C40005C7583E80300089BC4F86C35084920461E
:109C50002FF0FCF8074B1A6812B1074857F0F8FFCD
:109C600020461C6002B0BDE8F08100BF046C0A0809
:109C7000CC6A0A08985F0020106A0A082DE9F041B2
:109C8000A2B00C4607A92EF0F1F8002855D000210B
:109C90000D220CA80591ADF818100B9183F034FC3F
:109CA0002B4B611C1F68C9B20BAD0129F86A0A95DC
:109CB00046D1284B062205A90EF06CFE264B0193D7
:109CC00005AB0093002411222946244BF86A8DF835
:109CD00019400EF05FFE04AA0DF10F0128468DF821
:109CE0003C4004942FF026FD38B31D49DFF86C800A
:109CF000482210A883F0BEFB062610AC2268531E33
:109D0000049AC2F3513202EB831223798DF8243086
:109D1000A368019305AB009308924346112229469C
:109D2000F86A0EF037FE0021B7EE000A07A82EF001
:109D300069FA013E04F10C04E0D122B0BDE8F081E3
:109D40000091084B062205A90EF024FEB6E700BFDD
:109D5000685F002051570A08416A0A083B6A0A08EE
:109D600048170A08346A0A082DE9F04F90F8606530
:109D700085B00446002E59D17F2380F870350DF14F
:109D80000F0104232A308DF80F302FF037FE04F531
:109D9000C87504F5A768271D5FFA86FA1822FF2107
:109DA000284683F0B1FB85F85FA097F92690B9F1BA
:109DB0000A0F5CD03DDCB9F1040F0FDCB9F1020FE2
:109DC0000FDD442001F01AF8834620B13B462A46B5
:109DD00021465CF03BFAC8F800B002E0B9F1090F87
:109DE00039D0D8F8000050B1696EC5F8609031B133
:109DF0002C4B43F826102FF037FA2FF02DFA58F895
:109E0000040B0AF101095FFA89F940B103689B6804
:109E1000984784F8609551462046FFF72FFF01369A
:109E2000092E05F1680507F12C07B5D105B0BDE88D
:109E3000F08FB9F1150F28D0B9F1190FD1D1482001
:109E400000F0DCFF83460028C5D03B462A46214669
:109E50005DF0D0FBBFE7382000F0D0FF834600283C
:109E6000B9D03B462A4621465CF056FEB3E7302087
:109E700000F0C4FF83460028ADD0CDF800A03B46DB
:109E80002A4621465DF038FBA5E7782000F0B6FFB2
:109E9000834600289FD03B462A4621465CF0A4FE1C
:109EA00099E700BF9C5F002090F860358B4283BF2C
:109EB000682303FB010090F8DD01002070470000DB
:109EC00090F860358B4283BF682303FB010090ED5F
:109ED0006A0A9FED010A70470000000090F86035A3
:109EE0008B4206D901F5A77150F8210008B15CF04A
:109EF0004DBB9FED010A70470000000010B490F8C0
:109F000060458C420A4614D901F5A77450F82440E4
:109F10007CB1E468246A640603D55DF8044BFFF75E
:109F2000DDBF682101FB020393ED6A0A5DF8044B73
:109F300070479FED010AF9E70000000090F86035D6
:109F40008B420BD901F5A77150F8210038B1C368D5
:109F50001B6A1A4214BF012000207047002070477E
:109F600070B590F86035934204460E46154601D808
:109F7000002070BD02F5A77350F823000028F7D029
:109F800003689B6998470028F2D0682202FB0544C9
:109F9000D4F8AC313360ECE770B590F8603593429B
:109FA00004460E46154601D8002070BD02F5A77381
:109FB00050F823000028F7D003689B6998470028D1
:109FC000F2D0682202FB0544D4ED6C7AF4EE677A95
:109FD000F1EE10FAE8D6C6ED007AE6E770B590F833
:109FE0006035934204460E46154601D8002070BDE8
:109FF00002F5A77350F823000028F7D003685B69C7
:10A0000098470028F2D0682202FB0544D4F8B43106
:10A010003360ECE790F8603593420ED902F5A773F0
:10A0200050F823305BB1682303FB020292F8EC0185
:10A0300030B1D2F8E8310B60704700207047184605
:10A040007047000008299DBF2C2303FB01004068D6
:10A05000002070472DE9F04F4B4B2DED028B1B6814
:10A06000DB6A93F89C3089B00446002B00F08680B0
:10A07000DFF82CB19FED458A4FF0000994F8603568
:10A080005FFA89F5AB4279D905F5A77354F8230037
:10A0900000285DD003685B6B9847682303FB05438A
:10A0A000074693F8DC31834252D2032861D8DFE8B7
:10A0B00000F04F025259364E4FF000083DF09EFE20
:10A0C00094F86025AA4284BF682202FB05424FF043
:10A0D000680105F1010301FB05458CBFD2F8A821F9
:10A0E00018EE102A8246D5F8B001CDE90632F6F70F
:10A0F0000BFA079ACDE904011046F6F705FA069B1C
:10A100000096CDE902015A460421504637F03AF84C
:10A110000123204A84F8713585F8DC71D372D4F8B4
:10A120006C354BB3002255B25957481C03D04145FA
:10A1300002F10102F7D194F97035AB4208DBD4F893
:10A140006835D4F8640542463146984784F870551E
:10A1500009F1010992E72C2303FB05430E4E93F905
:10A160002D80ABE72C2303FB05430C4E93F92E8087
:10A17000A4E70026B046A1E71D46DCE709B0BDEC28
:10A18000028BBDE8F08F00BF685F00200000000078
:10A19000556A0A08F55F00200A890B084C6A0A080C
:10A1A000646A0A0890F860358B4207D901F5A771F7
:10A1B00050F8210010B10368DB6918470020704790
:10A1C00008299CBF682303FB010000F5C870704795
:10A1D00090F86035934207D902F5A77250F8220033
:10A1E00010B103685B6A18470020704790F860352B
:10A1F0008B420DD901F5A77350F8233043B1682382
:10A2000003FB0101012081ED730A81F8C801704749
:10A2100000207047F8B5002402460E4625462C273C
:10A2200092F86035E1B28B4210D901F5A77352F86C
:10A2300023304BB107FB01239B689E4204D110469B
:10A24000FFF7D4FF2843C5B20134E9E72846F8BD3B
:10A250002DE9F04F002493B005460E4617462146DF
:10A260002F2206A8059405F5A76983F04DF905F19D
:10A270002A0A4FF02C0B05F5F8730BFB04F259F882
:10A28000040B1AF90210E5B230B951B90134092CA6
:10A29000F3D14FF0010813E0682262439A589142CB
:10A2A00012D01548154B006801930135EDB20095A9
:10A2B000134BC06A324639460EF06CFB4FF0000873
:10A2C000404613B0BDE8F08F05A9332203935CF03C
:10A2D0003FFA039B804605A90028D7D10648019183
:10A2E0000135EDB200680095054BC06A324639462B
:10A2F0000EF050FBE4E700BF685F00209A6A0A088E
:10A300008C6A0A082DE9F04FDFF88090DFF880A012
:10A31000DFF880B08DB00646002796F86035FCB2B5
:10A32000A3422ED9682505FB046595F8E43133B3C3
:10A3300095F8E51119BB4FF001082022444404A808
:10A3400089F8198083F0E0F807EE904A4AF210434A
:10A35000F8EEE77A03AA4C21ADF8283050462423C2
:10A36000CDED037A38F024FE3DF048FD9BF8003037
:10A37000054A0094042136F005FF85F8E581013790
:10A38000CBE70DB0BDE8F08FA46A0A08F55F0020A6
:10A39000CD620020F02200202DE9F04F2F4B1E68E7
:10A3A00085B0044646B1D0F85C15304633F010F95C
:10A3B00010B1304632F05CF857F07CFC4FF00008EA
:10A3C00001904FF02C0A4FF0680B94F860355FFA5B
:10A3D00088F5AB4239D904EB8507D7F8380588B33F
:10A3E0000AFB05430BFB054993F92A20D9F8F01124
:10A3F0008A4227D132B30268D2689047D7F838052D
:10A400000268126B904799F8DD2112B1019BC9F8DF
:10A41000E031BEB1D4F85C15304633F0D9F888B1DC
:10A4200057F050FCCDE9021002460B46D7F838052C
:10A4300029465CF0D3FEDDE90232D7F8380529461B
:10A440005CF04AFF08F10108BFE72046FFF702FE73
:10A45000204605B0BDE8F04FFFF754BF4062002032
:10A460002DE9F0474FF000082DED028B0446894698
:10A47000B0EE408A474601264FF0680A94F86035EE
:10A480005FFA88F5AB421AD929FA05F3DB070AD53A
:10A4900005F5A77354F8230078B10368B0EE480AB5
:10A4A0009B6B984706400AFB054508F1010895F8A3
:10A4B000DC319F4238BF1F46E0E70646F3E727B985
:10A4C0007F23A4F87035034BDF72BDEC028B30465E
:10A4D000BDE8F087F55F002090F860358B4207D922
:10A4E00001F5A77150F8210010B10368DB6B184724
:10A4F000002070470B46114690F860259A4207D914
:10A5000003F5A77350F8230010B103681B6C1847BC
:10A510007047000070B504460E46002594F860357B
:10A52000E9B28B4205D932462046FFF7E3FF0135F9
:10A53000F4E770BD2DE9F84390F860550246002419
:10A5400000F12A062C2700F5F8784FF06809E1B2EF
:10A550008D420FD907FB04F309FB04F0F35658F8BA
:10A560000000834209D11BB11046FFF79DFC10B1DA
:10A570000134ECE70120BDE8F8830020FBE7000090
:10A5800010B590F860258A42044617D9682202FB6C
:10A59000010393F8DC31022B03D004D9032B18BF3D
:10A5A0000023184610BDFFF797FF48B92046FFF774
:10A5B000C1FF00280CBF06230123F2E70023F0E7C8
:10A5C0000623EEE7014B1868704700BF985F002034
:10A5D00010B5034904462EF039FC204610BD00BFDB
:10A5E000846C0A0810B50446203047F041FF044B44
:10A5F00004491C6020462EF029FC204610BD00BFF7
:10A60000C05F0020206E0A082DE9F3410022B7EE5A
:10A61000000A022105462DF029FF28465DF03AF890
:10A6200047F0A0FF234B1E680446F06A03685B6A8C
:10A6300098470B46022102460091204647F02EFF24
:10A64000B5F94A70002F13DDD6F82C80D8F8003009
:10A6500040465B68BCB2984728B198F84D3013B1BA
:10A66000C92FA8BFC824B06A036821465B68984711
:10A6700095F949002022002111F028FCC4B24AF0CB
:10A680006BFE4AF0CFFD70B9B06A036801345B68B5
:10A69000E4B205219847072CF1D9074802B0BDE87C
:10A6A000F04156F0BDBB072CF7D885F8494002B001
:10A6B000BDE8F081685F0020846D0A0810B504468B
:10A6C0005CF0B6FF2046BDE810405CF0E1BF000042
:10A6D0002DE98048284BDFF8A490DFF8A4A0DFF82C
:10A6E000A4B01446012293B005460E461A704FF0EE
:10A6F000000857F0DFFAD9F800300393A0EB080206
:10A7000041F287339A4207461FD9CDE90056039894
:10A710005346342205A9C06A0EF03CF9214605A82B
:10A72000049456F06DFBCDE9005603985B46342245
:10A7300005A9C06A0EF02EF904943DF05FFB049B5E
:10A7400005AA022136F004FDB8463DF057FB3CF067
:10A75000F1FD3DF053FB3EF0B5FC0A2105A80DF0DC
:10A7600021FF039B986A036805215B68984705A849
:10A770000DF024FFBDE700BFC45F0020685F00202C
:10A7800065E20A08619F0B080FB400B595B016AAE0
:10A79000002152F8043B039205A83C220193049146
:10A7A00082F0B2FE054A019B402104A856F0D0FA7F
:10A7B000039A034804A9FFF78BFF00BF9C6D0A08AA
:10A7C000B26D0A080FB407B504AA034852F8041B77
:10A7D0000192FFF77DFF00BFC46D0A08014B1868A6
:10A7E000704700BFC05F002008B50449102282F006
:10A7F00031FEB0FA80F0400908BD00BFC85F0020FC
:10A800001022002182F080BE10B50446FFF7F8FF49
:10A81000204610BD0378416023F00D03022A037027
:10A8200008D0032A0AD0012A03D1DBB243F0010386
:10A8300003707047037843F00803F9E7037823F0C7
:10A84000050343F00503F3E773B504460E461546CA
:10A850000193FFF7D5FF2046C4E90265069A0199E6
:10A86000FFF7D8FF02B070BD0078420704D4030799
:10A8700004D400F0010070470320704702207047A5
:10A88000F0B587B004461546FFF7EEFF88420F4645
:10A89000064605D163682B600126304607B0F0BD3F
:10A8A00000230328019301D0032913D130F07CFD4C
:10A8B00008B90026F1E7012301AA214630F0B0FBD8
:10A8C0000028F6D0DDED017A9FED337A67EE877AC6
:10A8D000CDED017A032E32D8DFE806F00209162406
:10A8E0006468032FE5D8DFE807F02C2E3C49FCF71D
:10A8F000B9FB90F87C32DB07DBD56468FCF7B2FB70
:10A90000D0F870321C44ECE702A8FFF779FFFCF79F
:10A91000A9FB02A9FCF7ACF906460028BDD0646883
:10A92000039BEFE7D4ED017A9DED017AF8EEE77A2B
:10A9300077EE877AFDEEE77A17EE904AD1E70024AA
:10A94000CFE72C60A8E7FCF78DFB90F87C6216F04F
:10A950000106AED0FCF786FBD0F87032E41A2C600A
:10A960009BE702A8FFF74CFFFCF77CFB02A9FCF772
:10A970007FF90646002890D0039BEFE707EE904A48
:10A980009DED017AF8EEE77A77EEC77AFDEEE77A89
:10A99000C5ED007A80E700BF0000C84273B501AA88
:10A9A00005460E46FFF76CFF044620B1019932467A
:10A9B0002846FFF72FFF204602B070BD13B514469E
:10A9C00001AAFFF75DFF48B1DDED017A9FED047A42
:10A9D000F8EEE77A67EE877AC4ED007A02B010BD30
:10A9E0000AD7233C07EE900A9FED090AF8EEE77AB2
:10A9F00008B527EE800A80F07FF9DFED067AB4EE25
:10AA0000E70AF1EE10FAD8BFB0EE670A08BD00BF42
:10AA100050E0EF300AD7233C10B50446806811F0AF
:10AA2000D9FB20B1E068BDE8104011F0E7BB10BDD4
:10AA300073B5856804460E461DBBC36823B98B6891
:10AA40008360CB68C3600125636873B92378DB0733
:10AA50000BD52046FFF708FF01AA01463046FFF755
:10AA60000FFF10B1019B636005462046FFF7D4FF3E
:10AA700020B9B368A360F368E3600125284602B0FB
:10AA800070BD0025E0E700000D4B83424FF000034E
:10AA90008B4106DA00F1255000F5311000F5E05049
:10AAA0007047084B98424FF0FF3371EB0303BEBF72
:10AAB00000F1564000F5130000F52440704700BF38
:10AAC00000D2496B002EB69490EA010F01D4401ACF
:10AAD0007047C317401A63EBE1710D4B83424FF08F
:10AAE00000038B4106DA00F1255000F5311000F526
:10AAF000E0507047074B98424FF0FF3371EB030370
:10AB0000BEBF00F1564000F5130000F52440704729
:10AB100000D2496B002EB69470B52DED028B84B037
:10AB2000044668460D46FFF76BFEFCF79BFA694644
:10AB3000FCF79EF8064608B3A368029ADFED128A76
:10AB400003999B1A07EE903AF8EEE77A67EEA87A37
:10AB5000C5ED007AE068FFF7B7FF08EE100AA068BD
:10AB6000024402EBD272B8EEC88A5010FFF73AFFE7
:10AB700028EE288A28EE000A85ED010A304604B046
:10AB8000BDEC028B70BD00BFF67C8E3F37B5002355
:10AB90000C4601AA022105460193FFF771FE10B988
:10ABA000002003B030BD21462846FFF7B5FF00283E
:10ABB000F6D0DDED017AF8EEE77AC4ED027AF0E73F
:10ABC00038B52DED028B0C460246C168E068FFF7F0
:10ABD0007BFF9568A46808EE100A601900EBD0703E
:10ABE0004010641BFFF7FEFE07EE904AF8EEE77A8E
:10ABF000F8EEC80A87EE807ABDEEC70A10EE103A6A
:10AC00005B4200EE103AB8EEC00A80F097FADFED32
:10AC1000087A30EE270ABDEC028BB5EEC00AF1EEE1
:10AC200010FA44BFDFED037A30EE270A38BD00BFCB
:10AC3000DB0FC93FDB0FC94030B52DED028B0B4652
:10AC400085B08C68D0E90251D868FFF73DFF08EE67
:10AC5000100A601900EBD0704010FFF7C3FE641BB0
:10AC600007EE904AF0EE400AB8EEC88A9FED060A59
:10AC7000F8EEE77A28EE008A27EE800A68EE200ACE
:10AC800005B0BDEC028B30BD8262363C82B002B0B2
:10AC9000FFF7D2BFF0B52DED028B0D4689B08C6861
:10ACA0000646D0E90271E868FFF70EFF08EE100AC9
:10ACB000E01900EBD0704010FFF794FE73686A68EB
:10ACC0009FED0E1A9B1A07EE903AE41BB8EEE77A56
:10ACD000F0EE400A07EE904A9FED090AB8EEC88AE6
:10ACE000F8EEE77A28EE008A27EE011A27EE800AAE
:10ACF00068EE200A09B0BDEC028BF0BD0AD7233CF8
:10AD00008262363C10B52DED028B84688A680B4652
:10AD1000111B08EE901AC168D868FFF7D5FE2244CF
:10AD200002EBD27208EE100A5010FFF75BFEB8EE8D
:10AD3000C88AF8EEE88A28EE000A20EE000AA8EE9B
:10AD4000A80A80F045FBBDEC028BDFED027A20EE15
:10AD5000270A10BD8262363C094B984206DDC0F1DD
:10AD6000D64000F5930000F5A4407047054B98428B
:10AD7000BEBFC0F1144000F5360000F538507047F2
:10AD800000E9A43500175BCAF8B52DED028BDFEDA5
:10AD9000148A076820EE280A0646FDEEC07A0D46A2
:10ADA00017EE904A04EBD47007EB6000B0EE608AB7
:10ADB000FFF718FE28EE288A3819C8EE007AFFF748
:10ADC000CBFF306017EE900AF6F7C8F82B68C01872
:10ADD00041EBE371FFF758FEBDEC028B2860F8BD34
:10ADE00002AAB34200F10C010830FFF7CDBF00000A
:10ADF0000148FFF705BD00BFC85F00200121884260
:10AE000038BF08467EF03AB8FFF7F8BF08B17EF0C9
:10AE100039B87047FFF7FABF00214FF0FF3310B584
:10AE200000220363044601600171C0F805104172FD
:10AE300080F8251000F13C0300F50B70D9709A6082
:10AE4000DA601A615A619A61DA611A625A629A6228
:10AE5000DA631A645A649A64DA641A655A659A6500
:10AE6000DA65DA661A675A677C339842E6D121467A
:10AE700004F5167007F016FC044B1A6822B9044951
:10AE80001C6020462DF0E2FF204610BDD85F002058
:10AE900088700A0873B5D0F83C3201919942044693
:10AEA00013D0D0F84032994218D0D0F844328B42B7
:10AEB00016D102200AE0D4F8343253B3D4F8383231
:10AEC0004BB34FF0030002B070BD002094F8223065
:10AED0008342F8D8431C84F82230F4E70120F5E7D8
:10AEE000D0F83062002EE6D194F841233546B60002
:10AEF0009AB1A319C3F83012A319019AC3F83C22DE
:10AF000094F82230AB429CBF6B1C84F82230284658
:10AF1000D9E70126E8E70226E6E704F50C7001A967
:10AF200030442EF03DFEE7E738B504460D462EF0DE
:10AF3000ADFD291D201D2EF0A9FD05F1080104F12C
:10AF400008002EF07DFE05F1140104F114002EF02E
:10AF500077FE05F1200104F120002EF071FE05F1CD
:10AF60002C0104F12C002EF025FD05F1300104F137
:10AF700030002EF02DFE05F13C0104F13C002EF0D6
:10AF80005FFEAB6BA3636B6B636338BD2DE9F0436E
:10AF9000A1B00023002500F13C0706468DF80750BC
:10AFA00003930493059306930793089309930A93D5
:10AFB0000B93109311931293139314931593169369
:10AFC000179318931C931D931E9300F50F78B946A1
:10AFD00058F8043BF3B1F26E934223D0D6F8E82040
:10AFE000934221D0D6F86421934213D10221EBB2CF
:10AFF00099420FD0C1EB411109EB8104214601A810
:10B00000FFF792FF39462046FFF78EFF01A9384629
:10B01000FFF78AFF0135032D07F17C07D8D121B056
:10B02000BDE8F0830021E2E70121E0E72DE9F047E8
:10B0300006460F461546804604464FF0000A39463C
:10B040003046FFF727FF626FBA425FFA8AF90ED1E6
:10B05000C3B2022B0BD87C2202FB0A66012086F8C1
:10B060003E0086F83F3085F80090BDE8F0870AF191
:10B07000010ABAF1030F04F17C04E0D1002439463F
:10B080003046FFF707FFD8F86C205FFA84F912B951
:10B09000C3B2022B22D90134032C08F17C08EED173
:10B0A00000244FF07C0906F13E0A39463046FFF78E
:10B0B000F1FE034609FB04F05FFA84F81AF8002059
:10B0C00012B9DBB2022B12D90134032CEDD196F860
:10B0D0002300042814D9194856F0BAFD7C2000FB3F
:10B0E0000464012084F83E0084F83F30BBE7064446
:10B0F000012086F83E0086F83F3085F80080B4E7EE
:10B1000006F54371002251F8043BBB42D4B208D18A
:10B11000A04202D8631C86F8233003342C70002030
:10B12000A3E73BB9421C06EB800086F82320C0F859
:10B130000C73F2E70132052AE5D1F0E7C06E0A0888
:10B14000C9B200EB8101D1F83C3253B1026F934296
:10B150000AD0D0F8EC20934208D0D0F8682193426E
:10B1600006D04FF003007047002070470120704761
:10B170000220704759B190F82030032B07D05A1C99
:10B1800080F8202000EB83004161012070470020FF
:10B19000704700002DE9F8430F469146044600F53C
:10B1A000BA7894F83E5035B97C344445F9D100253D
:10B1B0002846BDE8F88300234A46394601200DF0B1
:10B1C0007FF800210646E06E0DF08AF88642EBD14A
:10B1D000EEE700002DE9F043DFF87C8085B00446FF
:10B1E00000F50F7600257C27B14656F80C3CD9F8BF
:10B1F00000209342E9B206F1040619D1C3B12046FA
:10B20000FFF79EFFC0B207FB004090F83E307BB9CD
:10B2100003A9A9F10C0003932EF0C2FC3CF0EEFD53
:10B2200056F8043C009342462B46012135F0AAFF14
:10B230000135032DD8D104F16C0504F5F0742968AB
:10B2400021B9AB6813B128462CF02CFE7C35A54201
:10B25000F5D105B0BDE8F083DC6E0A0838B50446C8
:10B260001546FFF76DFFC0B2022808D87C2303FB08
:10B27000004029465030BDE838402EF0D1BC38BDE2
:10B2800038B504461546FFF75BFFC0B2022808D860
:10B290007C2303FB004029465C30BDE838402EF09B
:10B2A000BFBC38BD37B50D4604468DED010AFFF72A
:10B2B00047FF022D07D8C0B27C2303FB004001A941
:10B2C00068302EF05FFB03B030BD000038B5054696
:10B2D000FFF736FFC4B2022C13D8C4EB4414A40009
:10B2E0003C3504F10800284400212CF0DBFD04F17A
:10B2F000340104F1300029442844BDE838402EF0E0
:10B300004FBC38BD70B505460E461446FFF718FF12
:10B31000C3B2022B0DD87C2000FB035394E8070036
:10B32000443383E8070031462846BDE87040FFF704
:10B33000CDBF70BD37B504461546FFF701FFC0B25B
:10B34000022809D87C2303FB00400DF1070140309F
:10B350008DF807502EF09AFB03B030BD1FB590F961
:10B360002C30044623B390F921300BB36846FFF725
:10B370004BFAFBF777FE6946FBF72AFCC0B1DDED1F
:10B38000037A9FED0C0AF8EEE70ADDED027AF8EE9B
:10B39000E77A0123C0EE800A84F83D3387EE800A05
:10B3A00007F0C2FBDFED047A20EE270A84ED0A0ADB
:10B3B00004B010BD8096184B35FA8E3C024690F9C9
:10B3C000210058B192F8400340B1114491F92C0288
:10B3D00020B192F92400033818BF01207047000003
:10B3E00038B590F8223005465BB100242346E1B21F
:10B3F0002846FFF7E3FF08B10133DBB20134032C29
:10B40000F5D1184638BD000090ED0A0A70470000DB
:10B4100038B50C46D1ED066A11460546FFF790FE99
:10B42000C3B27C2000FB0353D4ED087AD3ED260A87
:10B4300094ED076AD3ED255A93ED245A26EE600A5F
:10B4400067EEA00AA5EEA70AF0EE607AE5EE867A2E
:10B45000B7EE007AA6EEE67A67EEE60AB1EE400AAB
:10B46000E5EE070A7FF06AFE9FED071ADFED070A97
:10B4700040F61C0010F0ECFCD5ED0A7ABDE838402F
:10B4800030EE270A10F0D0BCDB0F4940DB0F49C07B
:10B490002DE9F04190F822308B4204460D4602D24D
:10B4A0000020BDE8F081FFF74BFEC0B204F13C067E
:10B4B000C0EB401006EB8000083013F00BFADFED14
:10B4C000157AB0EEC00AB4EEE70AF1EE10FAE7D44E
:10B4D00029462046FFF734FEC5B27C2000FB054715
:10B4E0003B6F002BDCD0032DDAD000FB0560303041
:10B4F000D7F86C802DF080FDD7E91B32934201D143
:10B50000984505D07C2000FB0544C4F86C80C7E753
:10B510000120C6E7000000342DE9F74F04460E462F
:10B52000174600F50F7A4FF0000B5AF8049B5FFAAC
:10B530008BF8B9F1000F26D041462046FFF73EFFB9
:10B5400008B341462046FFF7FBFD7C23C0B203FB56
:10B55000004090F83E505DB908F101031B4ADBB290
:10B560003946304655F0F4FB284603B0BDE8F08F6D
:10B570005AF8102C914506D0154A3946304655F0F8
:10B58000E7FB0025F0E70BF1010BBBF1030FCCD17A
:10B590004FF0000894F822305FFA88F18B420DD901
:10B5A00020460191FFF774FF054620B90199204616
:10B5B000FFF704FF20B908F10108EBE70125D3E705
:10B5C000044A3946304655F0C3FBCDE7046F0A08FC
:10B5D000196F0A083E6F0A082DE9F0412DED048B22
:10B5E00090F842139FED348ADFED348A9FED349A50
:10B5F00082B00646FFF7A4FD06F13C07C5B27C20E9
:10B6000000FB057554354FF0000896F822205FFACC
:10B6100088F39A424ED919463046FFF7CFFE10B94B
:10B6200008F10108F1E719463046FFF789FDC4B279
:10B630007C2000FB0474D4ED157AF0EEE77AF4EE8A
:10B64000C87AF1EE10FA04F154040ED5D4ED017A63
:10B65000F0EEE77AF4EEC87AF1EE10FA05D50020A4
:10B6600002B0BDEC048BBDE8F0812946204613F002
:10B6700049F9B4EEE80AF1EE10FAF0DC294620466A
:10B6800012F02CFCB4EEC90AF1EE10FAE7DC214608
:10B69000284612F053FB68468DED000ACDED010AF5
:10B6A00012F008FCDFED077AB4EEE70AF1EE10FACB
:10B6B000B6DDD4E70120D3E700000034DB0FC93F3B
:10B6C000920A863F00004843022910B5044608D874
:10B6D000FFF736FD7C23C0B203FB004494F83D0025
:10B6E00010BD0020FCE7000013B590F84213019153
:10B6F0000446FFF7E9FF30B10199204602B0BDE8EA
:10B700001040FFF75BBE02B010BD0000F7B590F926
:10B7100021500446002D73D090F84053002D6FD077
:10B7200090F84213FFF7D0FF94F83D33064613B963
:10B730002046FFF713FE002594F82020EBB29A4232
:10B7400007D904EB83030135586903689B68984760
:10B75000F2E756F0AFFA0027224604F5BA7140F23C
:10B76000F315D2F89C30C31AAB428CBF00230123DF
:10B7700082F83D307C32914247EA0307F1D194F9D7
:10B780002430032B07D194F83C33002B3BD0D4F862
:10B790003803002849D167B1236B013309D032F057
:10B7A000F1F8216B31F014FF18B132F0EBF830F002
:10B7B00073FF94F92C32002B3AD194F92D32CBBB84
:10B7C00094F92E3213B1022384F8423394F84213D1
:10B7D0002046FFF779FF8642054611D032F0D2F8B5
:10B7E0004FF6FF7131F0F4FE50B1002D14BF00226E
:10B7F0000422019232F0C6F8019A032131F07AFE58
:10B80000284603B0F0BD012384F83C330420FFF741
:10B81000F5FA054610B1214606F0DAFF94F9243016
:10B82000C4F83853032BB2D0B5E706F0DFFFB2E718
:10B830000023C9E70123C7E738B590F92130044652
:10B84000D3B190F84053BDB1FFF77AFCC0B20228E3
:10B8500012D87C2303FB0044D4ED1A7A9FED087ABA
:10B86000F4EEC77AF1EE10FA06D4B7EE087AF4EEE9
:10B87000C77AF1EE10FA00DD0025284638BD00BF7A
:10B88000ABAA2A3F70B5D0F8085315F4003504462A
:10B890000E460DD190F840335BB90A78072A07D8D5
:10B8A000012303FA02F290F83F33134380F83F3349
:10B8B00070BD94F82020EBB29A42F9D904EB8303CF
:10B8C000314658690368DB6898470135F1E70000A5
:10B8D00038B505466C242B591BB1002128192CF0D2
:10B8E000E1FA7C34B4F5F07FF5D138BD014B18682E
:10B8F000704700BFD85F00202DE9F04FB24BD3F85E
:10B9000000800446D8F8040003688DB09B6898470F
:10B91000002507464FF0010909FA05F33B4240F0C4
:10B9200092820135202DF7D1D8F804000368DB6836
:10B930009847002507464FF0010909FA05F33B42F5
:10B9400040F0C3820135202DF7D1D8F804000368F8
:10B950009B689847002507464FF0010909FA05F34F
:10B960003B4240F0F1820135202DF7D1D8F8040098
:10B9700003689B689847002507464FF0010909FABC
:10B9800005F33B4240F01C830135202DF7D1D8F858
:10B990000400DFF840B203689B68984700250490D4
:10B9A000049A0123AB40134240F046830135202D19
:10B9B000F6D1D8F80400DFF81CB20368DB689847BA
:10B9C00000250490049A0123AB40134240F0058403
:10B9D0000135202DF6D1D8F804000368DB689847BC
:10B9E000002507464FF0010909FA05F33B4240F0F4
:10B9F000BF840135202DF7D1D8F804000368DB6837
:10BA00009847002507464FF0010909FA05F33B4224
:10BA100040F0ED840135202DF7D1D8F804000368FB
:10BA20009B689847002507464FF0010909FA05F37E
:10BA30003B4240F01B850135202DF7D1D8F804009A
:10BA400003689B689847002507464FF0010909FAEB
:10BA500005F33B4240F04A850135202DF7D1D8F857
:10BA6000040003689B689847002507464FF00109CA
:10BA700009FA05F33B4240F079850135202DF7D1D5
:10BA8000D8F804000368DB689847002507464FF0A4
:10BA9000010909FA05F33B4240F0A4850135202D48
:10BAA000F7D14A4B089308AF0425D8F8040003687F
:10BAB0009B689847002683460123B34013EA0B0F87
:10BAC00040F0CB850136202EF6D1D8F8040003686B
:10BAD000DB689847002683460123B34013EA0B0F27
:10BAE00040F001860136202EF6D1013D15F0FF050C
:10BAF00007F10107D9D1D8F8040003689B6898477B
:10BB00004FF00109074609FA05F33B4240F02F8642
:10BB10000135202DF7D1D8F804000368DB68984779
:10BB2000002507464FF0010909FA05F33B4240F0B2
:10BB30005A860135202DF7D1D8F8040003689B6898
:10BB40009847002507464FF0010909FA05F33B42E3
:10BB500040F085860135202DF7D1D8F80400036820
:10BB6000DB689847002507464FF0010909FA05F3FD
:10BB70003B4240F0B0860135202DF7D1144B07939E
:10BB8000D8F8040003689B68984700258346012382
:10BB9000AB4013EA0B0F41D000275FFA85F9D4F8C8
:10BBA000083313F4803A31D107AB4946DB5D049387
:10BBB0001A462046FFF7EEFA049B0646002800F0DE
:10BBC000C686CDE908AA07E0685F00200C0D0E0FBD
:10BBD00020212223801A0600099B0B9300220121B9
:10BBE0000BA8CDE9092204F06FFF01462046FFF7BC
:10BBF000C1FA0BA8FDF75EFE0AA8FDF75BFE09A8D7
:10BC0000FDF7A2FE16B108A8FDF79EFE94F82330BA
:10BC1000052B00F048810137042FC0D10135202DBC
:10BC2000B5D1D8F804000368DB689847002583463F
:10BC30000123AB4013EA0B0F38D000275FFA85F9D8
:10BC4000D4F8083313F4803A28D107AB4946DB5DBA
:10BC500004931A462046FFF79DFA049B06460028E7
:10BC600000F08486CDE908AA0022099B0B931146B7
:10BC70000BA8CDE9092204F027FF01462046FFF773
:10BC800079FA0BA8FDF716FE0AA8FDF713FE09A81E
:10BC9000FDF75AFE16B108A8FDF756FE94F82330BA
:10BCA000052B00F000810137042FC9D10135202D6B
:10BCB000BED1D8F8040003689B68984700268246E6
:10BCC0000123B34013EA0A0F31D010255FFA86F939
:10BCD000D4F8083313F0080B20D12A4649462046F1
:10BCE000FFF758FA0746002800F04F86CDE909BB58
:10BCF0000A9B002201210BA8CDE90A2301F048FC90
:10BD000001462046FFF736FA0BA8FDF71DFE0AA8EC
:10BD1000FDF71AFE17B109A8FDF716FE94F82330B7
:10BD2000052B00F0C0800135EDB2142DD0D10136C5
:10BD3000202EC5D1D8F8040003689B6898470026D8
:10BD400082460123B34013EA0A0F34D014255FFA68
:10BD500086F9D4F8083313F4001B24D12A46494647
:10BD60002046FFF717FA0746002800F02186CDE9A4
:10BD700008BB099B0B93002201210BA8CDE90922E6
:10BD800002F018F801462046FFF7F4F90BA8FDF77A
:10BD900091FD0AA8FDF78EFD09A8FDF7D5FD17B1A5
:10BDA00008A8FDF7D1FD94F82330052B7BD0013591
:10BDB000EDB2182DCDD10136202EC2D1D8F8040015
:10BDC0000368DB689847002682460123B34013EAE4
:10BDD0000A0F34D014255FFA86F9D4F8083313F427
:10BDE000001B24D12A4649462046FFF7D3F90746CF
:10BDF000002800F0ED85CDE908BB0022099B0B93DC
:10BE000011460BA8CDE9092201F0D4FF01462046D6
:10BE1000FFF7B0F90BA8FDF74DFD0AA8FDF74AFDA5
:10BE200009A8FDF791FD17B108A8FDF78DFD94F85D
:10BE30002330052B37D00135EDB2182DCDD1013689
:10BE4000202EC2D12FE0D4F8083313F0010A25D1F7
:10BE50005FFA85FB1E2259462046FFF79BF90646EE
:10BE600020B3CDE908AA099A0B92002308220121E8
:10BE70000BA8CDE9093303F0C7FA01462046FFF7C6
:10BE800079F90BA8FDF716FD0AA8FDF713FD09A81F
:10BE9000FDF75AFD16B108A8FDF756FD94F82330BA
:10BEA000052B7FF43EAD0DB0BDE8F08FD8F804103F
:10BEB00004220B68CDE90102B84A0092D3F800A031
:10BEC0005A461E2309A8D047CDE7D4F8083313F00B
:10BED000010A24D15FFA85FB1E2259462046FFF74E
:10BEE00059F9064608B3CDE908AA099B0B93062227
:10BEF00000210BA8CDE9091103F086FA014620467E
:10BF0000FFF738F90BA8FDF7D5FC0AA8FDF7D2FC1E
:10BF100009A8FDF719FD16B108A8FDF715FD94F85D
:10BF20002330052B7FF40EADBDE7D8F804100422B2
:10BF30000B68CDE90102994A0092D3F800A05A4655
:10BF40001E2309A8D047D0E7D4F8083313F4805A49
:10BF500021D15FFA85FB0D2259462046FFF71AF9D9
:10BF60000646F0B1CDE909AA0A9B0022CDE90A23D1
:10BF7000012108220BA804F0B5FA01462046FFF77C
:10BF8000F9F80BA8FDF7E0FC0AA8FDF7DDFC16B1F7
:10BF900009A8FDF7D9FC94F82330052B7FF4E3AC16
:10BFA00081E7D8F8041004220B68CDE901027B4A2E
:10BFB0000092D3F800A05A460D230AA8D047D3E731
:10BFC000D4F8083313F4801A21D15FFA85FB2C22B0
:10BFD00059462046FFF7DEF80646F0B1CDE909AA3A
:10BFE0000A9B0022CDE90A23012108220BA804F0B4
:10BFF000A7FB01462046FFF7BDF80BA8FDF7A4FC00
:10C000000AA8FDF7A1FC16B109A8FDF79DFC94F85C
:10C010002330052B7FF4B8AC45E7D8F80410042290
:10C020000B68CDE901025D4A0092D3F800A05A46A0
:10C030002C230AA8D047D3E7D4F8083313F4807729
:10C040003FD15FFA85F90C2249462046FFF7A2F856
:10C050000646002800F08480CDE90677079B0A9306
:10C060004FF0000A692249462046CDF81CA0FFF790
:10C0700091F80746002800F08180CDE908AA099BC5
:10C080000B9300221A2309920BA901220AA801F09E
:10C0900007F801462046FFF76DF80BA8FDF754FCA2
:10C0A00009A8FDF751FC17B108A8FDF74DFC0AA837
:10C0B000FDF74AFC07A8FDF747FC16B106A8FDF7F7
:10C0C00043FC94F82330052B3FF4EDAED4F808334D
:10C0D00013F480777FF46AAC5FFA85F90C22494645
:10C0E0002046FFF757F80646002859D0CDE90677D5
:10C0F000079B0A934FF0000A682249462046CDF874
:10C100001CA0FFF747F80746002857D0CDE908AA3A
:10C11000099B0B9300221A2309920BA901220AA85A
:10C1200000F0BEFF01462046FFF724F80BA8FDF7FC
:10C130000BFC09A8FDF708FC17B108A8FDF704FCE3
:10C140000AA8FDF701FC07A8FDF7FEFB16B106A83B
:10C15000FDF7FAFB94F82330052B7FF427ACA2E619
:10C16000D8F8041004220B68CDF800B0CDE9010224
:10C170004A461F6807A80C23B8476FE7D8F8041091
:10C1800004220B68CDF800B0CDE901024A46D3F88D
:10C1900000A009A86923D04771E700BF801A0600F4
:10C1A000D8F8041004220B68CDF800B0CDE90102E4
:10C1B0004A461F6807A80C23B84799E7D8F8041027
:10C1C00004220B68CDF800B0CDE901024A46D3F84D
:10C1D00000A009A86823D0479AE7D4F8083313F4DD
:10C1E00080773DD15FFA85F90C2249462046FEF75B
:10C1F000D1FF0646002800F08180CDE90677079B35
:10C200000A934FF0000A692249462046CDF81CA047
:10C21000FEF7C0FF074600287ED0CDE908AA099B9B
:10C220000B9300221A230BA90AA8099200F038FFE9
:10C2300001462046FEF79EFF0BA8FDF785FB09A8E7
:10C24000FDF782FB17B108A8FDF77EFB0AA8FDF7F2
:10C250007BFB07A8FDF778FB16B106A8FDF774FB7A
:10C2600094F82330052B3FF41EAED4F8083313F4B2
:10C2700080777FF4ADAB5FFA85F90C224946204602
:10C28000FEF788FF0646002855D0CDE90677079BC4
:10C290000A934FF0000A682249462046CDF81CA0B8
:10C2A000FEF778FF0746002853D0CDE908AA099B7E
:10C2B0000B9300221A230BA90AA8099200F0F0FEA2
:10C2C00001462046FEF756FF0BA8FDF73DFB09A8E7
:10C2D000FDF73AFB17B108A8FDF736FB0AA8FDF7F2
:10C2E00033FB07A8FDF730FB16B106A8FDF72CFBC2
:10C2F00094F82330052B7FF46BABD4E5D8F8041009
:10C3000004220B68CDF800B0CDE901024A461F684F
:10C3100007A80C23B84772E7D8F8041004220B686A
:10C32000CDF800B0CDE901024A46D3F800A009A833
:10C330006923D04773E7D8F8041004220B68CDF8BE
:10C3400000B0CDE901024A461F6807A80C23B84790
:10C350009DE7D8F8041004220B68CDF800B0CDE9B1
:10C3600001024A46D3F800A009A86823D0479EE7F7
:10C37000D4F8083313F0200A24D15FFA85FB1C227D
:10C3800059462046FEF706FF064608B3CDE908AA3F
:10C390000022099B0B9311460BA8CDE9092203F05B
:10C3A00031FC01462046FEF7E5FE0BA8FDF782FAB8
:10C3B0000AA8FDF77FFA09A8FDF7C6FA16B108A882
:10C3C000FDF7C2FA94F82330052B7FF412AB6AE52F
:10C3D000D8F8041004220B68CDE90102B84A009293
:10C3E000D3F800A05A461C2309A8D047D0E7D4F8B8
:10C3F000083313F0200A24D15FFA85FB1E22594628
:10C400002046FEF7C7FE064608B3CDE908AA00227B
:10C41000099B0B9311460BA8CDE9092203F0F2FB0F
:10C4200001462046FEF7A6FE0BA8FDF743FA0AA830
:10C43000FDF740FA09A8FDF787FA16B108A8FDF73D
:10C4400083FA94F82330052B7FF4E4AA2BE5D8F87F
:10C45000041004220B68CDE90102994A0092D3F836
:10C4600000A05A461E2309A8D047D0E7D4F80833C5
:10C4700013F0200A25D15FFA85FB1C22594620467D
:10C48000FEF788FE064610B3CDE908AA099A0B927A
:10C490000023022201210BA8CDE9093303F0B2FBEE
:10C4A00001462046FEF766FE0BA8FDF703FA0AA830
:10C4B000FDF700FA09A8FDF747FA16B108A8FDF73D
:10C4C00043FA94F82330052B7FF4B5AAEBE4D8F8AF
:10C4D000041004220B68CDE90102794A0092D3F8D6
:10C4E00000A05A461C2309A8D047CFE7D4F8083348
:10C4F00013F0200A25D15FFA85FB1E2259462046FB
:10C50000FEF748FE064610B3CDE908AA099A0B9239
:10C510000023022201210BA8CDE9093303F072FBAD
:10C5200001462046FEF726FE0BA8FDF7C3F90AA830
:10C53000FDF7C0F909A8FDF707FA16B108A8FDF73D
:10C5400003FA94F82330052B7FF486AAABE4D8F8DD
:10C55000041004220B68CDE90102594A0092D3F875
:10C5600000A05A461E2309A8D047CFE7D4F80833C5
:10C5700013F0400A21D15FFA85FB0C225946204670
:10C58000FEF708FE0646F0B1CDE909AA0A9B002293
:10C59000CDE90A23012106220BA800F047FD014640
:10C5A0002046FEF7E7FD0BA8FDF7CEF90AA8FDF738
:10C5B000CBF916B109A8FDF7C7F994F82330052B7C
:10C5C0007FF45BAA6FE4D8F8041004220B68CDE96D
:10C5D00001023B4A0092D3F800A05A460C230AA855
:10C5E000D047D3E7D4F8083313F0400A20D15FFADC
:10C5F00085FB0C2259462046FEF7CCFD0646E8B1E5
:10C60000CDE909AA00220A9B11460BA8CDE90A230D
:10C6100000F00CFD01462046FEF7ACFD0BA8FDF72F
:10C6200093F90AA8FDF790F916B109A8FDF78CF95E
:10C6300094F82330052B7FF431AA34E4D8F80410A1
:10C6400004220B68CDE901021D4A0092D3F800A034
:10C650005A460C230AA8D047D4E7D4F8083313F07D
:10C66000800A26D13B78F1B21A462046CDE9041360
:10C67000FEF790FDDDE90413814618B3CDE909AA60
:10C680000A9B0022CDE90A2301210C220BA803F00A
:10C6900087F901462046FEF76DFD0BA8FDF754F91A
:10C6A0000AA8FDF751F9B9F1000F02D009A8FDF76A
:10C6B0004BF994F82330052B7FF404AAFFF7F3BB62
:10C6C000801A0600D8F80400B84AD0F800E00092BA
:10C6D0004FF0040CCDE9019C0A46DEF800A00146AB
:10C6E0000AA8D047CCE7D4F8083313F0800A26D143
:10C6F0003B78F1B21A462046CDE90413FEF74AFD15
:10C70000DDE90413814608B3CDE909AA0A9B00229A
:10C71000CDE90A2300210C220BA803F041F90146C0
:10C720002046FEF727FD0BA8FDF70EF90AA8FDF736
:10C730000BF9B9F1000F02D009A8FDF705F994F83B
:10C740002330052B7FF4CEA9FFF7ADBBD8F804004A
:10C75000964AD0F800E000924FF0040CCDE9019C1D
:10C760000A46DEF800A001460AA8D047CEE7D4F872
:10C77000083313F4004A20D15FFA85FB0C22594696
:10C780002046FEF707FD0646F0B1CDE909AA0A9B4F
:10C79000002201210BA8CDE90A2302F077FF014610
:10C7A0002046FEF7E7FC0BA8FDF7CEF80AA8FDF738
:10C7B000CBF816B109A8FDF7C7F894F82330052B7C
:10C7C0007FF4A6A9FFF76FBBD8F8041004220B680A
:10C7D000CDE90102754A0092D3F800A05A460C2315
:10C7E0000AA8D047D3E7D4F8083313F4004A20D17D
:10C7F0005FFA85FB0C2259462046FEF7CBFC064625
:10C80000F0B1CDE909AA00220A9B11460BA8CDE997
:10C810000A2302F03BFF01462046FEF7ABFC0BA8C3
:10C82000FDF792F80AA8FDF78FF816B109A8FDF7F1
:10C830008BF894F82330052B7FF47BA9FFF733BBEB
:10C84000D8F8041004220B68CDE90102574A00927F
:10C85000D3F800A05A460C230AA8D047D3E7D4F84F
:10C86000083313F4007A20D15FFA85FB3022594651
:10C870002046FEF78FFC0646F0B1CDE909AA0A9BD7
:10C88000002201210BA8CDE90A2303F087FC014611
:10C890002046FEF76FFC0BA8FDF756F80AA8FDF737
:10C8A00053F816B109A8FDF74FF894F82330052B7B
:10C8B0007FF450A9FFF7F7BAD8F8041004220B68E8
:10C8C000CDE90102394A0092D3F800A05A4630233C
:10C8D0000AA8D047D3E7D4F8083313F4007A20D15C
:10C8E0005FFA85FB302259462046FEF753FC064688
:10C8F000F0B1CDE909AA00220A9B11460BA8CDE9A7
:10C900000A2303F04BFC01462046FEF733FC0BA83C
:10C91000FDF71AF80AA8FDF717F816B109A8FDF7F0
:10C9200013F894F82330052B7FF425A9FFF7BBBA41
:10C93000D8F8041004220B68CDE901021B4A0092CA
:10C94000D3F800A05A4630230AA8D047D3E7D8F836
:10C95000041004200A68CDE9016014480090D2F860
:10C9600000A009A84A46D047FFF736B9D8F8041006
:10C9700004200A68CDE901600C480090D2F800A0BC
:10C9800009A84A46D047FFF76FB9D8F80410042227
:10C990000B68CDE90102054A0092D3F800B04A467F
:10C9A0002B460AA8D847FFF7A3B900BF801A060094
:10C9B000D8F8041004220B68CDE901020C4A009259
:10C9C000D3F800B04A462B4609A8D847FFF7D1B99B
:10C9D000D8F8041004220B68CDE90102044A009241
:10C9E000D3F800B04A462B4609A8D847FFF705BA46
:10C9F000801A060073B50446FEF77EFF94F82330D4
:10CA0000052B32D0002594F83F33EB40DA07E9B22A
:10CA100016D40135082DF6D194F82330052B24D0F7
:10CA200094F8203013B194F82230F3B9104B114927
:10CA30001B68986903681B6802B0BDE8704018471E
:10CA4000D4F808339B030CD42C200191FEF7D6F9BF
:10CA5000064610B1019903F019FC31462046FEF755
:10CA600089FB94F82330052BD3D102B070BD00BFF1
:10CA7000685F0020586F0A082DE9F04F90F92130C7
:10CA800089B00446002B00F00481012300F50C75E9
:10CA900080F84133024600F50F712B462E46D06ECA
:10CAA000002859D0002384F8413394F94030642B96
:10CAB0005BD094F9BC30642B00F08D8094F9383150
:10CAC000642B00F08A80D4F830722FBB01A9204675
:10CAD0002BF0CCF900B30C230593012306978DF8B6
:10CAE0001830714B07936946BDF80430049704A8C9
:10CAF000ADF810308DF800702BF038FB9DF9001068
:10CB000051B1022908DC38B1C9B27C2303FB0141D1
:10CB10006C3128462DF05CF894F841B3BBF1000F5E
:10CB20005DD0E36E6367D4F8E830C4F8F030D4F831
:10CB30006431C4F86C3194F8233003F1C30204EB80
:10CB400082020021042B7CD852F8040B10610133BF
:10CB500042F8041CDBB2F5E753F8040B0028A1D11E
:10CB60008B4202F17C029AD19FE7002066238DF868
:10CB700010307C2303FB004004A940302CF06CFFF4
:10CB800004A920462BF072F900289CD004238DF8CC
:10CB900018300023CDE9013303933123059369460F
:10CBA00004A82BF0E3FA059B28B108AA02EB830244
:10CBB000009942F8E01C0133332B0593EFD952F072
:10CBC000DFF89DED031ADDED020A9DED010A6621F5
:10CBD00052F094F877E70120C8E70220C6E7012762
:10CBE000A94655F8043B23B1AB600137042FF7D1B8
:10CBF00097E7AA46B8465FFA88F3022BF5D8DAF829
:10CC0000002055F8043C9A4205D104A95046CDF8BD
:10CC100010B02CF0DDFF5AF8043B08F101020BB90B
:10CC20009046E8E704A906EB88000193CDF810B020
:10CC30002CF0CEFF019BAB6001A948462CF0C8FF49
:10CC4000D3E794F8413313B92046FEF79FF994F8DF
:10CC500022300BB3154B1B68986A036864215B682C
:10CC600098472046FEF752FD94F83E3003B9E3663C
:10CC700094F8BA300BB9C4F8E83094F836310BB9EF
:10CC8000C4F86431FAF7EEF9FAF7B8FA0123A4F818
:10CC9000403309B0BDE8F08F2046FFF7ABFE94F8B3
:10CCA0002230002BE0D0D5E7A40C0B08685F0020F1
:10CCB0007047000001207047012070474368986862
:10CCC0007047000010B5054B03600446806A10B140
:10CCD00003685B689847204610BD00BF1C740A08B3
:10CCE000406803685B6A184733B46C46406884E860
:10CCF0000C0003689D6A94E80C00AC4602B030BC9E
:10CD00006047000010B50446FFF7DCFF2046FEF741
:10CD10007DF8204610BD000040680BF003BA00000B
:10CD2000406801230BF0FEB940680BF0D7B9000052
:10CD300040680A220BF07CB940680BF091B9000002
:10CD400040680BF013BA000090F82E2022B190F842
:10CD50002D10002201F06EB97047000073B5044633
:10CD600005250026A06A8DF8076003680DF107020B
:10CD7000DB680121984778B19DF807300C2B09D06A
:10CD8000102B05D0092B07D184F8303002B070BDCC
:10CD90001523F9E71423F7E7013DE3D12846F5E72A
:10CDA00010B4806A03681C690822A44601235DF858
:10CDB000044B31216047000010B4806A03681C698D
:10CDC0000122A44600235DF8044B32216047000095
:10CDD000F0B50446806A036885B05B6998470546EC
:10CDE000002800F08480A06A03685B6998470368A4
:10CDF0009B689847A06A03689B69984760B93D4B58
:10CE00003D491B68986903681B6898472B6828464A
:10CE1000DB689847002667E02046FFF7CDFF002833
:10CE2000F4D02046FFF79AFF0028EFD0A06A0368ED
:10CE30000121DB6A98472046FFF7B2FF30B92D4B3E
:10CE40002E491B68986903681B68DEE7A06A0368BF
:10CE5000DB69984730B9274B29491B6898690368F3
:10CE60001B68D2E7A06A94F83010012784F82E706E
:10CE700003685B6A9847A06A03689B6A984704F155
:10CE80002D020146204601F023F906460028BDD0B8
:10CE9000A06A94F82D10036801919B6A9847019944
:10CEA0000246204601F018F994F82C302BB194F882
:10CEB0002D103A46204601F023F994F82F2094F8DB
:10CEC0002D10204601F03EF92B682846DB68984774
:10CED000A06A029403681D6A0A4B039304AB13E92A
:10CEE0000C0042F21071A847304605B0F0BD06466E
:10CEF000FAE700BF685F002088730A08AE730A086B
:10CF0000CD730A08FDCF010870B5002586B0CDE9C4
:10CF1000005500230446806A8DF80850059303935A
:10CF2000049303686A469E6810210923B047A0B1A4
:10CF30009DF8003013F0010615D194F8313001331B
:10CF4000DBB2052B84F8313007D12046FFF734FFE0
:10CF50002046FFF725FF84F83160A06A03681B6B49
:10CF6000984706B070BD9DF8083084F831501B0713
:10CF7000F3D4BDF901309FED1F6A06EE903ABDF97A
:10CF8000033007EE103ABDF90530F8EEE66A07EE19
:10CF9000903ACDED036AF0EEE66AB8EEC77AF8EEA5
:10CFA000E77AF4EEC66AF1EE10FA8DED047ACDED73
:10CFB000057A0DD5B0EEC77AB4EEC67AF1EE10FA66
:10CFC00006D5F0EEE77AF4EEC67AF1EE10FAC4D4A4
:10CFD0009FED090A03A811F0D3F8B2EE040A03A8E2
:10CFE00011F0CEF894F82D200A2303A9204601F071
:10CFF0000FF9B2E7000000349A99193EFFF784BF99
:10D0000010B5044B044640F8043BFCF79DFC204659
:10D0100010BD00BF34740A0810B50446FFF7F0FFD6
:10D020002046FDF7F3FE204610BD0000F7B503686B
:10D030000F4616461BB90024204603B0F0BD00245D
:10D04000046008200193FDF7D9FE054620B1124B7C
:10D050000360019B4360019401A8FCF775FC002D5F
:10D06000E9D03420FDF7CAFE04460028E3D000F0E2
:10D07000E1FE0A4BA562236084F82C7084F82F60CF
:10D080002046FFF7A5FE05460028D5D12368204697
:10D090005B6898472C46CFE734740A081C740A086A
:10D0A0002DE9F74F046806460D4690469946002C38
:10D0B0006CD00B68002B49D0236820465B6A9847E8
:10D0C00003689B689847012328680DEB0302002141
:10D0D0000BF028F898B39DF80130EA2B2FD1DFF838
:10D0E000F0B04FF0060A28680023802206210AF0DB
:10D0F000F5FF20B3DBF80070B86A03680A215B68AB
:10D100009847002328681A4606210AF0E7FFB0B1C5
:10D11000B86A03680A215B689847012328680DEB09
:10D12000030206210AF0FEFF48B19DF8014014F009
:10D1300040042FD00AF1FF3A1AF0FF0AD3D1306829
:10D1400003685B6A98470368DB68984700241DE022
:10D15000022223460F2128680AF0C0FFB86A03683C
:10D1600001215B689847306803685B6A98470368E9
:10D17000DB689847336834604A46414601A801930A
:10D18000FFF754FF044601A8FCF7DEFB204603B07E
:10D19000BDE8F08F224623460F2128680AF09EFF43
:10D1A000B86A036801215B6898470223214630680A
:10D1B0000DEB03020AF0B6FF04460028C8D0B86998
:10D1C000024903681B689847B9E700BFF4730A086F
:10D1D000685F002090F82C10002200F02BBF0000A8
:10D1E00070B504468CB00426013E76B2731C4AD05A
:10D1F000A06A15236A465D210AF094FF0028F3D047
:10D20000A06A152306AA5D210AF08CFF05460028B6
:10D21000EAD0152206A9684680F01CF90028E3D15F
:10D220009DF8003084F82E309DF8073084F83030B7
:10D230009DF8143084F83A309DF813309DF8102092
:10D2400084F83B309DF80F3043EA0223A3879DF812
:10D25000013084F82F309DF8083084F83130039B7A
:10D260009DF80C20C3F30F2363869DF80B3043EA2F
:10D270000223A386049BC3F30F23E386019BC3F31E
:10D280000F23238707E0054B05491B68986903684E
:10D290001B689847002528460CB070BD685F0020C9
:10D2A00068740A082DE9FF4104460023806A8DF85E
:10D2B00007300368DFF868815B6A984703689B68FA
:10D2C0009847A06A03680A219B6C9847A06A0A22C3
:10D2D00004210AF0ADFE0425013D6DB26B1C32D075
:10D2E00000234B21A06A82220AF0F8FED8F80060E1
:10D2F0000746B06A036802215B689847002FEBD0AD
:10D3000001231A464B21A06A0AF0E8FE0746B06ADC
:10D31000036802215B689847002FDDD0A06A0123D3
:10D320000DF1070240210AF0FDFE0028D4D09DF83F
:10D330000720322A10D0002DCED1B06936490368BB
:10D340001D683223A847A06A03685B6A9847036890
:10D35000DB68984700255BE02046FFF741FF002887
:10D36000F1D0A06A0123172251210AF0B7FE00284C
:10D37000E9D05222A06A012311460AF0AFFE00282C
:10D38000E1D0A06A012338224C210AF0A7FE002830
:10D39000D9D0A06A03685B6A98470368DB6898473E
:10D3A000A06A05210AF05CFEA36A04F12C029968C8
:10D3B000204600F08DFE054650B3A36A94F82C1069
:10D3C0009A68204600F088FE94F8442094F82C10C7
:10D3D000204600F0B7FE94F845302BB194F82C109D
:10D3E0000122204600F08CFEA06A036802219B6C9B
:10D3F0009847A06A029403689E6A084B039304ABA3
:10D4000013E90C0044F21B11B04754F053FC2064A4
:10D41000284604B0BDE8F08190740A088DD5010853
:10D42000685F002070B5858F90F93B60AD03B5FB58
:10D43000F2F2A2F5804404FB04F2D51190F83A20F0
:10D440000498D201624306FB05225212A03002F575
:10D450008012424312134A43DB0003EB623000B2F6
:10D4600070BD000010B5448E53005C43B0F93830F5
:10D47000C91A838FD31AB0F93620B0F93400534358
:10D4800004F500449B10C3EBC13300EB2440044976
:10D4900093FBF0F04FF400420EF008FD00B210BD17
:10D4A0000080FFFF10B52DED028B8AB004460823E3
:10D4B000806A05AA42210AF035FE18B1BDF81A208B
:10D4C000D30719D4A06A0AF051FE54F0F3FB236C81
:10D4D000C31AFA2B0CD92064002382224B21A06AA4
:10D4E0000AF0FCFD0123A06A1A464B210AF0F6FD62
:10D4F0000AB0BDEC028B10BDBDF9141094F93030A8
:10D500000093920894F92E300392C9102046FFF739
:10D5100089FFBDF9161094F93130039A009308EE93
:10D52000900A94F92F30C9102046FFF77BFFBDF910
:10D530001810039A491008EE100A2046FFF792FFD0
:10D5400007EE900AF8EEE88AF8EEE77AB8EEC88AB5
:10D55000B3EE000A07A8CDED097ACDED078A8DED6F
:10D56000088A10F021FEB2EE040A07A810F008FEA7
:10D5700054F0A0FB94F82C2020640A23204607A92D
:10D5800000F046FEA06A0AF0F1FDB1E7FFF78ABF9E
:10D59000F7B503680D4616461BB90024204603B0B4
:10D5A000F0BD002707604820CDE90073FDF726FC99
:10D5B000044650B100F03EFC0E4B2360019BA36279
:10D5C000019784F8446084F8455001A8FCF772F98B
:10D5D0006846FCF76FF9002CDFD02046FFF762FEAB
:10D5E00005460028DAD1236820465B6898472C4618
:10D5F000D4E700BFC8740A0810B5044B044640F8CD
:10D60000283BFCF757F9204610BD00BFC8740A0834
:10D6100010B50446FFF7F0FF2046FDF7F7FB204664
:10D6200010BD000090F82C10002200F003BD000097
:10D63000F8B504460D4617461E4600F0FBFB094BA5
:10D6400023602B68A362002200232A6084F82D70D7
:10D6500084F82E6023656365A365E36523666366CE
:10D660002046F8BDE0740A08F8B51C460933164692
:10D67000DB086A46A2EBC30300AF9D46806AA31C89
:10D680006A460AF04FFD054628B122460DF1020117
:10D6900030467FF0EFFE2846BD46F8BD2DE9F34148
:10D6A00006460F46144654F005FB114BD3F8008094
:10D6B0000546D8F82800036801215B6898470123D4
:10D6C0000DF1070207213046FFF7CEFF60B19DF84C
:10D6D0000730DA0702D4B7EB531F05D054F0EAFA4B
:10D6E000431BA342E5D3002002B0BDE8F08100BF98
:10D6F000685F00202DE9F041DFF8608292B00446B7
:10D7000002AF002646F02002A06A0023D2B25021C8
:10D710000AF0E4FC002800F00C810325013D6DB205
:10D720006A1C00F00681D8F80030986A03684FF44C
:10D7300096719B68984701230DF1060255212046FA
:10D74000FFF792FF002800F0F4809DF8063013F0F8
:10D75000E00F40F0EE80DB07E0D502230DF106027A
:10D7600052212046FFF780FF002800F0E280BDF83C
:10D77000063001365BBA202E27F8023BC2D1BDF835
:10D7800024309DF826109FED6D7ADFED6D6A9FEDD8
:10D790006D6A43F30B0207EE902A1B0903F47063D2
:10D7A000BDF82620F8EEE77A0B4343F30B03C4EDF4
:10D7B0000C7A07EE903A02F470639DF82820F8EE98
:10D7C000E77A134343F30B03C4ED0D7A07EE903A67
:10D7D0009DF92230F8EEE77AC4ED0E7A07EE903A22
:10D7E0009DF92930F8EEE77A67EE877A07EE103A6E
:10D7F000B8EEC77A9DF92A30C4ED0F7A27EE267A63
:10D80000DFED517A84ED107A07EE103AB8EEC77A60
:10D810009DF92B30E7EE267AC4ED117A07EE903AA7
:10D82000F8EEE77A9DF9233067EEA67ADFED476AD6
:10D83000C4ED127A07EE903A9DF92C3007EE103ABB
:10D84000B8EEC77A9DF92E3027EE267AF8EEE77A01
:10D8500084ED147A67EE867A07EE103A9DF930303F
:10D86000C4ED137A07EE903AF8EEE77A9DF92D3081
:10D8700067EEA67AB8EEC77AC4ED167A27EE267A56
:10D8800007EE903A84ED157AF8EEE77A9FED307A5C
:10D890009DF92F3067EE877AC4ED177A07EE903A3C
:10D8A0009DF93130F8EEE77A06EE903A67EE877A26
:10D8B000F8EEE66AC4ED187ADFED267ABDF9383065
:10D8C000E6EE877A07EE103A9DF93230C4ED197A08
:10D8D000B8EEC77AF3EE077AE7EE067A07EE103A6B
:10D8E000DFED1D6AC4ED1A7AB8EEC77A27EE267A04
:10D8F00084ED1B7A9DF9333007EE103AB8EEC77A03
:10D900009DF9343027EE267A84ED1C7A07EE103A22
:10D910009DF9353007EE903AB8EEC77AF8EEE77A1F
:10D9200027EE267A67EEA67A84ED1D7AC4ED1E7A7C
:10D9300000E0002012B0BDE8F08100BFCDCC4C3E2D
:10D940000000803B0000003B0AD7233C0000003D64
:10D950000000803817B7D1B80AD7A33A685F002013
:10D9600073B501230E460DF1070206210446FFF7A9
:10D970007BFE18B90025284602B070BD9DF807301F
:10D98000013B012B0CD80023A06A1A4606210AF09D
:10D99000A5FB0028EED0062200212046FFF77EFEE0
:10D9A000A06A0023324606210AF098FB05460028AB
:10D9B000E0D0262231462046FFF770FEDBE700006C
:10D9C00013B501230DF1070207210446FFF74CFEB2
:10D9D00010B9002002B010BD9DF807301B070CD510
:10D9E0000023A06A1A4606210AF078FB0028F0D02E
:10D9F000062200212046FFF751FEA06A00230722DD
:10DA000006210AF06BFB0028E3D0132207212046F1
:10DA1000FFF744FE0028DCD0A06A0023052206217F
:10DA20000AF05CFB0028D4D0172205212046FFF71E
:10DA300035FE0028CDD001212046FFF791FFC9E730
:10DA4000F7B50446806A5B4F03685B6A98470368D2
:10DA50009B689847A06A03680A219B6C9847A06A54
:10DA60000A2204210AF0E4FA0525013D6DB26B1C7F
:10DA700000F09680A06A0023B6227E210AF02EFBD9
:10DA80000028F2D03B68986A036818215B686E46EC
:10DA900098470123324600212046FFF7E5FD002884
:10DAA000E3D09DF80030332BDFD12046FFF722FE74
:10DAB000002875D0A06A0023802250210AF00EFBB6
:10DAC00000286DD02046FFF77BFF002868D0A06AB1
:10DAD000002386222E210AF001FB002860D0A06AD4
:10DAE0000023242204210AF0F9FA002858D0A06A61
:10DAF0000023022206210AF0F1FA002850D0142255
:10DB000002212046FFF7CAFDA06A00230722052153
:10DB10000AF0E4FA002843D001212046FFF720FF55
:10DB200000283DD0A06A036803219B6C9847A06A37
:10DB300003685B6A98470368DB689847A06A172107
:10DB40000AF08EFAA36A04F12C029968204600F0CC
:10DB5000BFFA054608B3A36A94F82C109A682046C9
:10DB600000F0BAFA94F82E2094F82C10204600F019
:10DB7000E9FA94F82D302BB194F82C1001222046AC
:10DB800000F0BEFAA06A03689F6A0B4B00940193F1
:10DB900096E80C0042F21071B847284603B0F0BD79
:10DBA000A06A03685B6A98470368DB6898470025AA
:10DBB000F3E700BF685F0020B1DD010810B586B053
:10DBC0000C236A4631210446FFF74EFD002800F081
:10DBD000DF809DF801309DF80020DFED717ADFEDE8
:10DBE000715A1B0403EB02239DF8022003EB02632E
:10DBF0001B1206EE903A9DF804309DF803201B049A
:10DC000003EB02239DF8052003EB02631B1207EED2
:10DC1000103A9DF807309DF806201B0403EB022301
:10DC20009DF8082003EB02631B1206EE103A9DF8E4
:10DC30000A309DF809201B0403EB0223F8EEE66A84
:10DC4000B8EEC77A9DF80B2066EEA76A27EE277A12
:10DC5000B8EEC66ADFED547A03EB02631B1226EEC0
:10DC6000276A07EE903AF8EEE77A67EEA57AF5EEC6
:10DC7000C07AF1EE10FA40F38D80DFED4C5A77EE6A
:10DC8000E57AD4ED134A94ED0F5A94ED1C4AD4ED85
:10DC90001D3A94F82C20F7EE005A74EEA54AF0EEE7
:10DCA000632AA4EEA75A0A2303A9D4ED107AD4ED6F
:10DCB0000C4A77EEA57A2046E7EEA64AD4ED1A7A0A
:10DCC00075EE677A94ED145AF0EE646AD4ED174A53
:10DCD000E5EE276AB0EE655AA7EEA45AC6EE854A6D
:10DCE00094ED115AD4ED0D6A35EE255AE5EE076A2A
:10DCF00094ED157AE7EE876A94ED187AB0EE655ADE
:10DD0000A7EE875A86EE857A94ED125AD4ED0E6A04
:10DD100035EE255AE5EE066A94ED166A94ED195A29
:10DD2000E7EE866AB0EE656AA7EE856AF0EE657A80
:10DD300086EE863A94ED1B6AF0EE646AE6EE447A6B
:10DD4000E6EE476A86EEA75AF0EE476AE4EE646AAA
:10DD5000C6EEA75AD4ED1E6AD4EE262AE6EE636A12
:10DD6000B2EE046A27EE667A65EE066AA2EEA47A3F
:10DD7000CDED036A65EE866ACDED046AC7EE276ACB
:10DD800076EE837A67EE867ACDED057A00F040FA7A
:10DD900006B010BD44BFDFED055A77EEA57A70E7F7
:10DDA00047ABE73B5B9E803AF61BEB3B85EBCB41F9
:10DDB000FFF704BF30B51346026885B00D461AB9A7
:10DDC0000024204605B030BD002101607C20019375
:10DDD0000392FDF713F8044620B1019B2A4603A9DC
:10DDE000FFF726FC03A8FBF765FD002CE8D02046D2
:10DDF000FFF726FE05460028E3D1236820465B682E
:10DE000098472C46DDE7000010B5044B044640F867
:10DE1000283BFBF74FFD204610BD00BFE0740A0809
:10DE200010B50446FFF7F0FF2046FCF7EFFF204651
:10DE300010BD0000064B10B503600446FDF756FD0B
:10DE4000606004F1080052F0E9FD204610BD00BFFB
:10DE5000F8740A0873B50646144675687C2303FBFC
:10DE60000253C4EB441405EB8404084693F8A41051
:10DE7000019010F01BFA94F93C3001983BB973689B
:10DE800093F8251002B0BDE8704010F00FBA94F876
:10DE90004010F7E737B5446801917C2505FB024542
:10DEA00095F83F3004EB8304D4F84C325BB153F067
:10DEB00001FFC5F89C000199D4F84C0203B0BDE8FD
:10DEC000304003F0A7BF03B030BD00002DE9F04F94
:10DED000C2EB421447684FEA840881460E4607F1B8
:10DEE0003C0B08F108018BB015465944304610F040
:10DEF00013F9D9F8040029460BEB8404FDF79CFCC8
:10DF000038B17C2303FB057393ED1A0A304610F0F9
:10DF100037F97C2303FB057393ED146ADFED3A7A3E
:10DF2000D3ED156AB0EEC67AB4EEE77AF1EE10FAE8
:10DF30000FD5B0EEE67AB4EEE77AF1EE10FA08D536
:10DF400094ED077AB0EEC77AB4EEE77AF1EE10FA04
:10DF50001BD47C2303FB0573D86D196E5A6E9B6D21
:10DF6000029003910490079101A831468DED016A5A
:10DF7000CDED056A0692089209930EF095F986EDAB
:10DF8000000AC6ED010A86ED021A7C2303FB057721
:10DF90000023C7F88C30C7F88830C7F88430D9F828
:10DFA000040090F95C3208F13C0A08F14808DA44B0
:10DFB000D84463B15DB9414600F5167004F0E2FB48
:10DFC000414630460BB0BDE8F04F10F0A5B890F9CF
:10DFD0003430012B0BD190ED0E0A504610F07CF836
:10DFE00084ED120AC4ED130A84ED141AE8E7022B3B
:10DFF000E6D1FCF7E7FA002201A9FBF7B1FF002800
:10E00000DED09DED010AE8E70000003410B543685A
:10E010007C2404FB023407C904F1900383E8070061
:10E0200053F048FEC4F89C0053F038FEC4F8A0003A
:10E0300010BD0000F0B5074685B00D46164600F14C
:10E040000801A92203A80AF0C7FA7C687C2303FB15
:10E050000543D3F8B42022B903A80AF0DFFA05B0CB
:10E06000F0BDBEB196ED007AD3ED2A7A67EE877ADD
:10E07000C3ED2A7A96ED017AD3ED2B7A67EE877A93
:10E08000C3ED2B7A96ED027AD3ED2C7A67EE877A80
:10E09000C3ED2C7A7C2607EE902A06FB0541A831B9
:10E0A000B8EE670A0846019110F07EF801992A46F9
:10E0B0003846FFF7ABFF06FB05410023C1F8B0303F
:10E0C000C1F8AC30C1F8A8300023C1F8B430C3E7C0
:10E0D0004068FCF7ABBF0000F7B506464068019208
:10E0E0007C2707FB01000D466C3001A914462BF07C
:10E0F0004FFD716807FB05152C6703B0F0BD0000EC
:10E1000007B540687C2303FB010393F93C30022BE5
:10E110000BD000F13C03C1EB411003EB80000DF18B
:10E1200007018DF807202BF08DFC03B05DF804FB90
:10E1300043687C2202FB013191F93C00003818BF92
:10E140000120704743687C2000FB013181F8A42046
:10E1500070470000F8B5054608460F4610F082F8F3
:10E1600010B100242046F8BD384610F061F804468E
:10E170000028F6D16B6893F934637EB1384610F00D
:10E18000A9FB95ED087ADFED1F7AF0EEC76AF4EE91
:10E19000E76AF1EE10FA03D585ED080A0124E1E7FC
:10E1A00077EE407A30EE076AF0EEE77AC7EE866ADD
:10E1B000F6B207EE906A9FED146AF8EE677A26EEE3
:10E1C000866AF4EEC67AF1EE10FA48BFB2EE046A3F
:10E1D000DFED0E7A45BF6B6A66EE866AB0EE676A5F
:10E1E00087EEA66A46BF01336B620124F7EE007A20
:10E1F00077EEC67A20EE060AA7EE270A85ED080A12
:10E20000B0E700BF0000003400004843CDCCCC3D57
:10E210002DE9F74304460E4615461F46FFF71AFE42
:10E220002A4631462046FFF735FE314620462A462B
:10E23000FFF74CFE31462046FFF78CFF28B39B22A8
:10E2400004F1080101A80AF0C7F964684FF07C09DD
:10E2500009FB054808F1A808314640460FF05CFF6D
:10E2600009FB0542D2F8B4100131C2F8B4104FB125
:10E27000B94207D34908C2F8B410B0EE000A4046CC
:10E280000FF092FF01A80AF0C9F903B0BDE8F083CE
:10E2900010B50446FCF754FFC0B23C34C0EB40104C
:10E2A00004EB800010BD0000F8B50A4E044600F5EE
:10E2B000167704F5137555F8040B08B104F0DEF871
:10E2C000BD42F8D13368986A036801215B689847BA
:10E2D000EFE700BF685F002008B5FFF7E5FF00002B
:10E2E000F0B5144E00EB810773780446D7F84C0262
:10E2F0006FF3410387B00D467370C8B102F0ACFCF8
:10E3000068B1737843F0100373702C440023A37238
:10E31000D7F84C0207B0BDE8F04002F021BCD7F8B6
:10E320004C12684602F0C8FC009B012BEDD1E8E7D7
:10E3300007B0F0BD1460002070B506460D460024FD
:10E3400045FA04F3DB07E1B202D53046FFF7C8FF18
:10E350000134032CF4D170BDFF21FFF7EDBF0000A5
:10E3600030B500F5137587B000F5167455F8041B29
:10E3700021B9A542FAD1002007B030BD684602F0AD
:10E380009BFC009B013B022BF3D80120F4E700002B
:10E390002DE9F0472DED028B88B004460D469046DE
:10E3A000B0EE408AFDF790F930B90026304608B04B
:10E3B000BDEC028BBDE8F08729462046FCF7FEFF46
:10E3C00006460028F1D004EB8507D7F83C22D7F8A1
